:020000040800F2
:10000000F8FF0720290102087B4407086944070814
:100010007D4407088944070895440708000000004C
:10002000000000000000000000000000A1440708DC
:10003000A344070800000000F95A07084102022003
:1000400001000208294507083B4507084145070804
:10005000B7CC07080100020899C007089FC007082D
:10006000A5C00708ABC00708B1C00708ED7B0708AB
:10007000FD7B07080D7C07081D7C07082D7C070801
:100080003D7C07084D7C070801000208E5A1070830
:10009000A9A10708AFA10708B5A10708B7C00708BD
:1000A000554507085B4507086D4507087345070870
:1000B000794507087F45070885450708AD82070889
:1000C000C9820708E58207080183070801000208C2
:1000D00001000208350302203B03022041030220F5
:1000E000DBC007082F450708B1440708B1450708DA
:1000F000B7450708CF450708C94507085D7C0708CD
:1001000001000208D5D607088D450708010002083E
:100110001D03022023030220A5450708AB4507085D
:100120006D7C07087D7C07088D7C07089D7C07088F
:10013000AD7C070835AF0708354507080100020800
:10014000010002080100020801000208A544070896
:10015000BD7C0708CD7C0708DD7C0708470302202B
:100160000100020801000208010002080100020863
:10017000010002080100020801000208000000005E
:100180000100020801000208290302202F030220B7
:100190000100020801000208010002080100020833
:1001A0000100020801000208010002080100020823
:1001B0000100020801000208010002081D8307086F
:1001C000398307080100020800000000010002084E
:1001D00001000208010002080100020801000208F3
:1001E00001000208010002080100020801000208E3
:1001F0000100020801000208024800234030836029
:1002000000F03AB900400220054B012243F82010CB
:10021000044B1A604FF08052034B5A60704700BF86
:1002200080CC022088CC022000ED00E010F4FE7F9C
:1002300003D1024B0422C3F8002E704700E100E016
:100240000D4B10B51C6801341C604FF0E02304F026
:1002500003021B69094B53F822300BB12046984723
:10026000074B1B68A34205D106490020BDE810409A
:10027000FFF7CABF10BD00BFD8B102208CCC02204E
:10028000D4B10220DDA10608224B03EB800310B598
:10029000D3F89C41002C3BD06268D3699BB2E383C6
:1002A0009B0618D5618A00292DD0A38A9BB2013301
:1002B000B3FBF1F001FB1033E18A9BB2994222D0EB
:1002C000516AA2890A40A17A91B113490968914201
:1002D0000ED1FFF791FFE38B626803F01801116202
:1002E000A28B134214D0206ABDE8104000F0C0B8C1
:1002F000E17AA0690129A18A89B20CBF20F81120F6
:100300004254A382E7E7136823F020031360E2E777
:1003100010BD00BF00400220D80402200420FFF7D7
:10032000B3BF0520FFF7B0BF0720FFF7ADBF082020
:10033000FFF7AABF0120FFF7A7BF0220FFF7A4BF66
:100340000320FFF7A1BF0620FFF79EBF134B00223B
:1003500070B504469A61124D00F076F80646EB68D7
:10036000DA0307D4EB6813F0F20F0ED000F078F840
:10037000012003E0611CF2D00CB9032070BD00F035
:1003800063F8801BA042EAD9F7E7EB68DB0701D4EA
:100390000020F3E70123EB60FAE700BFDCB10220A5
:1003A000003C02402DE9F843DFF8988005460F46EF
:1003B00098F81430012B40D001234CF2503088F8CB
:1003C0001430FFF7C3FF0446A8B94FF0FF333B607A
:1003D0002B68012B15D16968287C00F03DF84CF2A0
:1003E0005030FFF7B3FF164A0446136923F4004365
:1003F00023F004031361002388F814302046BDE87D
:10040000F883AE68DFF83890D5E902231344B3428D
:10041000F1D9297C304600F027F84CF25030FFF734
:1004200095FFD9F8103023F0FA03C9F8103010B155
:1004300004463E60DFE70136E6E70224DEE700BF60
:10044000003C0240DCB10220014B1868704700BF3D
:10045000D8B10220000000005FF800F0E5FD0608BA
:100460005FF800F0CDFC06085FF800F021FE0608FA
:100470005FF800F0359C06085FF800F051E40208D0
:020000040802F0
:10000000FEE700000F490020D1F8883043F4700368
:10001000C1F888300C4B1A6842F001021A609860EF
:100020001A6822F0847222F480321A60074A5A60F9
:100030001A6822F480221A60D8604FF000638B6047
:10004000704700BF00ED00E000380240103000248F
:1000500030B5002495B02F4D2C22214609A8C5F8B3
:100060009040039449F078F82B6C4FF480004FF0E7
:10007000040C4FF4A05E43F080532B642B6C03F010
:1000800080530093009B244B1A6842F440421A604C
:1000900001221B680A9403F4404304940193019BDA
:1000A0004FF4A023CDE9072310230F220B93022343
:1000B0000292D8221193CDE90D30092307A812939B
:1000C0004FF48053CDE90FC2CDE905E34CF0CAFFF0
:1000D00010B1124853F072FD4CF036FF08B11048D1
:1000E000F8E7109B30210F9A02A8DB00B3FBF2F374
:1000F000B3FBF1F201FB12321199003AB3FBF1F1BB
:1001000018BF012255F0FCFD08B10648E2E715B022
:1001100030BD00BF0038024000700040E0EA070830
:10012000F2EA07080CEB07080446DFF82CD00B496D
:100130000B4A0C4B03E051F8040B42F8040B9A42B3
:10014000F9D300200849094A01E041F8040B914223
:10015000FBD3204653F086BEF8FF072010250A087F
:1001600080040220E40402200040022068410320B1
:1001700040F8044B40F8045B40F8046B40F8047B03
:1001800040F8048B40F8049B40F804AB40F804BBF3
:1001900040F804CB40F804DB68467047024B5A69CC
:1001A000026058610020704700400220024B5A69EB
:1001B00012685A61704700BF00400220024B9A69E2
:1001C000C0E900219861704700400220044A936909
:1001D0001968916110B15A6818461047704700BFFE
:1001E0000040022038B50446044DAB690BB1A34270
:1001F00000D338BD0120FFF7E9FFF6E700400220F9
:10020000C460056146618761C0F81C80C0F8209019
:10021000C0F824A0C0F828B0C0F82CD080ED0C8B1A
:1002200080ED0E9B80ED10ABC0F808E0FFF7B6BF85
:10023000124D6C6908B50CB953F000FE60602046A1
:10024000FFF7D0FF23686B612046C46805694669E3
:100250008769D0F81C80D0F82090D0F824A0D0F87E
:1002600028B0D0F82CD090ED0C8B90ED0E9B90ED3B
:1002700010ABD0F808E00120704700BF004002201A
:1002800010B50021044600F0FDFA18B914B120465B
:100290000DF0A6FE10BD002100F0F4BA10B501214A
:1002A000044600F0EFFA18B914B120460DF098FE9C
:1002B00010BDFFF7E5BF10B501220C4600F006FCAB
:1002C00018B914B120460DF08BFE10BD00F0FEBB36
:1002D00000F0BEBB484308B50830FFF7DCFF40B173
:1002E000044A936A03B118600021C0E900139062C8
:1002F000083008BD00400220034678B153F8042CB2
:10030000083812B153F8081C116053F8083C13B1B7
:100310005A6000F09DBB024B9A62FAE7704700BF3B
:10032000004002202DE9F0414FF0030C00252A4C3B
:100330008646D4F8CC02002101310EEB01039A0865
:1003400003F00303825C5B0042FA03F303F0030350
:10035000022BF1D0D4F8D802090100EB0E104FEABD
:10036000910E61B300EB8E0E03681A0724D1D4F806
:10037000D822991A9A424FEA9116C1F301124FEA14
:10038000111119D8D4F8DC7252009F4214D9D4F854
:10039000CC720CFA02F8BB5D43FA02F243EA08039E
:1003A00002F00302012A07D13F2DBB5504EB4503A0
:1003B0000CD80135A3F8EC1204307045D4D145B106
:1003C000013D04EB4503B3F8ECE2B2E7C4F8E822E0
:1003D000F2E7BDE8F08100BF0040022030B51C4CC0
:1003E0000122D4E9B553C01AC109C0F302134FEA80
:1003F000101C9A406B5C4FEA9C0E23EA02036B547C
:100400008309D4F8E0220325B2EB901FD4F8CC0284
:100410000CF0030288BFC4F8E032C15C52000CF15A
:10042000010C05FA02F30CF0030221EA0301530068
:1004300000F80E104FEA9C0ED4F8CC0210F80E1003
:1004400041FA03F303F00303022BE7D030BD00BFF2
:100450000040022021F00F01154A38B50B1A154C47
:100460000546013BC4F8DC12C4F8CC02DB00A2FB59
:1004700003235B0A9A00C4F8D032A1EB8311013345
:1004800007321D44C4F8D81203EBD2020021C4F88D
:10049000D45248F061FE002301214FF0FF32238146
:1004A000A4F86C13C4E9B833C4E9DC3238BD00BF2A
:1004B000F32C23FA00400220024A138902331381ED
:1004C000704700BF00400220024A1389023B13819B
:1004D000704700BF00400220024B1889003818BF47
:1004E0000120704700400220F8B51C4D00222B89E6
:1004F00005F1080405F50876C5F8E82243F0010384
:10050000C5F870232B8154F8043F1A0719D1D5F888
:10051000D822981A93424FEA9011C0F301124FEA81
:1005200010100ED3D5F8DC725200BB4209D2D5F8B8
:10053000CC7217F801C04CFA02F303F00303012B4D
:1005400002D0B442DFD1F8BD032393404CEA030C40
:1005500007F801C0FFF7E6FEF3E700BF0040022006
:1005600071B3F8B50F46051F0024164E55F8043F29
:100570001A0719D1D6F8D822981A9A424FEA901C35
:10058000C0F301124FEA10100ED8D6F8DC12520058
:10059000994209D9D6F8CCE21EF80C1041FA02F3C0
:1005A00003F00303012B03D00134A742DED1F8BDD1
:1005B0000323934019430EF80C10FFF7B3FEF3E743
:1005C000704700BF004002202DE9F043614C83B02A
:1005D000D4F8E832D4F8CC12C3B1D4F8D032002524
:1005E0009800C4F8E85288B10026B30806F0030268
:1005F000CB5C5200134103F00303032B20D00136E0
:100600008642F2D3D4F8E832002BEAD1D4F8E432AF
:100610004FF0000901274FEAD308D4F8D4324FEA4B
:10062000C90513F8096046B305F0030316F0010F7E
:100630004FEA95024FEA430314D176080135F3E7F8
:1006400030460136FFF76EFED4F8D032D4F8CC1223
:10065000B6EB830F4FEA8300C7D3D4F8E832002B00
:10066000BFD1D3E78A5C42FA03F303F00303012B03
:1006700009D0760805F10105D6D1C84509F1010375
:1006800025D09946C9E7D4F8D8022B016A4640F232
:100690001241C35800EB05105BB10CF031FE009B1A
:1006A0003BB10DF0E3FEDDE900010DF0B7FE0DF00A
:1006B000F3FEEB08D4F8D40205F00701C25C07FA98
:1006C00001F122EA0102C254D4F8CC12D1E74FF072
:1006D000000C03260227654662460EE0012905D17B
:1006E00006FA03F301252EEA030303700132D4F85E
:1006F000E4329A421FD8D4F8CC124FEA920E02F09C
:10070000030301EB920011F80EE05B004EFA03F1D7
:1007100001F0030102291AD00329DFD107FA03F3FC
:100720002EEA030E80F800E09446D4F8E432013259
:1007300000259A42DFD923890022C4F8E4C223F0BD
:100740000103C4F8E022238103B0BDE8F083002D4B
:10075000EAD0C5E700400220044B00211A89C3F803
:10076000E81242F001021A81FFF72EBF004002207A
:10077000434B00212DE9F041D3E9B6420F460E4626
:10078000121BD3E9B3540B4641604FEA840C0C466C
:1007900081610260C0E90211C0E904119A0803F006
:1007A00003080133AA5C4FEA4808ACEB030E42FA97
:1007B00008F2BEFA8EFE02F003024FEA5E1E012A24
:1007C00049D0022A39D0A2BB01369C4501F1010172
:1007D0001746866022D09A0803F00308AA5C4FEA05
:1007E000480842FA08F202F00302012A02DDBEF1D3
:1007F000000FD3D0A2F10108012FB8FA88F84FEA10
:10080000581824D0022F02D1426901324261826914
:10081000BA4238BF8761B8F1000F02D1BEF1000FB4
:10082000BCD0C2688A4238BFC1609C4519D0002143
:10083000B4E79C45CFD10322D7E701349C4507F1AB
:1008400001074460C7D1012F4FF00008DAD10269D7
:1008500001320261DBE701349C45446007D0174652
:10086000B9E724013601C0E90146BDE8F081076916
:1008700001370761876907B982610127D1E700BFA6
:10088000004002202DE9F84300F10F0636093FD061
:100890006E4C2389E3BBB4F86C230D46E2BBD4F85D
:1008A000E002D4F8D072B84232D24FF0010ED4F840
:1008B000CCC20138013F00216044CCF101086744FB
:1008C00018E04A1C964255D913F00C0F37D18A1CF8
:1008D000964240F2AA8013F0300F36D10132964290
:1008E00040F2A8803F2B23D8511C8E4240F2A780B3
:1008F000B8420AD008EB000910F8013F9A07E0D08F
:1009000013F00C0F16D10122E2E7BEF1000F23D045
:1009100000231846BDE8F883D4E9DC12914226D2C0
:10092000D4F8E002D4F8D072874215D99E46BEE7CB
:100930000021DDE713F0300F0CD10122CFE703F0E7
:100940003002B2FA82F25209CCE73F2B8CBF002171
:100950000121CDE70022C5E75AF0DAFDD4F8E00224
:10096000D4F8D0724FF0010EB842A0D3D0E75AF0BD
:10097000CFFD94E74FEA8909A9EB0201012A01F1B1
:10098000010704D109F101039B08C4F8E032D4F84F
:10099000E43207F0030EB80802314B454FEA4E0E21
:1009A00038BF4B468945C4F8E4324FF0010303FADF
:1009B0000EF31CF800E043EA0E030CF8003012D3EB
:1009C0004FF0020E01F003038808D4F8CCC20131C5
:1009D0005B001CF8008089450EFA03F343EA080324
:1009E0000CF80030EED2D4F870331201D4F8D8826B
:1009F000002133443E01C4F8703308EB0713184656
:100A000048F0AAFBEA07034683D50022D4F8D402B3
:100A1000F90807F0070748F806200122445CBA40AD
:100A2000224342541846BDE8F8834FEA890909F188
:100A30000109A1E74FEA890909F102099CE74FEA98
:100A400089090A4609F1030996E700BF0040022020
:100A5000034B1A89012A02D808B1FFF7BFBC7047BF
:100A600000400220034610F00F001BD1164AD2F8B6
:100A7000D812994215D810B4D2F8DC429C420DD954
:100A80005B1AD2F8CC42C3F301119A091B09A25C8C
:100A900049000A4102F00302012A05D05DF8044B27
:100AA000704770470020704701301A18910802F013
:100AB0000302615C520041FA02F202F00302022AD0
:100AC000F2D00001EAE700BF004002202DE9F84F14
:100AD0000F460646002800F0CC80744D2C89002972
:100AE00000F09280002C40F09380D5F8D8020F31AE
:100AF000D5F8D0C2301A09094FEA8C0A030903F16C
:100B0000010EBEEB8C0F80F0BA80A446D5F8CC92D3
:100B10004FF001084FEA9E040EF0030B19F8044051
:100B20004FEA4B0B44FA0BF404F00304022C2BD0D5
:100B30002CB90CF1010C0CEB08048C4226D3414576
:100B40005ED067D3C4448C4525D2002A60D0C20948
:100B5000D5F8D41203F007033846895C194101F037
:100B60000101FFF78FFE0446002851D04FEA08121A
:100B7000314648F0ADFA2B89012B02D83046FFF7F9
:100B80002DFC2046BDE8F88F08F101080EF1010E9A
:100B9000F245BFD1D3E75C1843449C4220D903F00F
:100BA000030298084FF0020C0133520019F800704C
:100BB0009C420CFA02F242EA070209F800200FD91F
:100BC00003F003029808D5F8CC720133520017F8ED
:100BD00000E09C420CFA02F242EA0E023A54EFD1D3
:100BE000D5F8E432A1EB080206EB081000219C4284
:100BF0004FEA021238BF1C46C5F8E44248F0ACFA8E
:100C000034462046BDE8F88F012C01D8FFF7E6FBFB
:100C10000024B6E75C184FF0030CA8EB010104EACE
:100C20000C07A008012904F101044FEA470719F84D
:100C300000E00CFA07F72EEA070709F8007010D059
:100C400003EB080E04F00302A708D5F8CC320134F8
:100C50005200D95D74450CFA02F221EA0202DA551B
:100C6000F0D1D5F8E0328342CAD93446C5F8E00263
:100C7000C7E701463846BDE8F84FFFF703BE012934
:100C8000BED029B14FF00108002A7FF460AFBFE762
:100C900003F003038009D5F8CC1203225B009A40CD
:100CA0000B5C23EA02030B54DBE700BF0040022089
:100CB00010B58AB0044603A8FFF75AFD039A094904
:100CC000DDE904300090204600F092FF2046069CAB
:100CD000079ADDE90831CDE90014034900F088FFE7
:100CE0000AB010BDE0700808047108082DE9F84347
:100CF000DFF8589107464749D9F8D82200F078FF25
:100D0000D9F8D01289006DD00025DFF8448115F0A4
:100D10003F0633D005F003067600AB08D9F8CC22A5
:100D2000D35C334103F00303022B63D0032B5FD06A
:100D3000012B4AD1D9F8D8222B01D25842455BD099
:100D4000354B9A425AD0354B9A425BD0344B9A423B
:100D500056D0344B9A4253D0334B9A4254D0334BF3
:100D60009A4251D0324B9A4252D0324B9A424DD095
:100D7000314B9A4214BF68224D2227E0A9421ED966
:100D8000D9F8CC022C4602E001348C4208D0A208EB
:100D900004F00303825C5B0042FA03F39B07F3D089
:100DA000621B7F2A0BD992092449384624F03F055B
:100DB00000F01EFFD9F8D032B5EB830F12D22A0112
:100DC0001F49384600F014FFA7E72E221D49384678
:100DD00000F00EFF0135D9F8D032B5EB830F4FEAA2
:100DE000830194D338461849BDE8F84300F053BB5B
:100DF0006D22EBE73D22E9E75422E7E74C22E5E7E5
:100E00005322E3E74422E1E74122DFE74222DDE724
:100E10004622DBE74C710808CCB608088CAE0808FF
:100E20009CBF0808CCBF080840AB0808B4AB080852
:100E300034B30808F8B3080860B8080868710808EF
:100E4000847108088C710808487108080040022065
:100E500014C108080346064A506A1A684168C1F37B
:100E60001E018A4202D3521A1A6070470068F5E7E1
:100E700000400220014441F20553884204D398B255
:100E8000012838BF0120704703EB431310F8012BF2
:100E90005340F2E7034B044A5A620022C3F824226B
:100EA000704700BF004002208C0C09082DE9F04774
:100EB00081460F46002942D0FFF7DCFF214B8246D6
:100EC0005C6A0CB9204636E094F907300025E668E4
:100ED000002B06F1FF3616DB013604F11808B54287
:100EE00015D32468EDE705EB06083A4648464FEA75
:100EF000580808F1060354F8231048F091F9002827
:100F0000CCBF45464646731B012BECD8E4E723696A
:100F100033F815309A4510D163695B5D9F420CD15F
:100F20003A46494658F8250048F042F928B9606821
:100F3000C0F31E002844BDE8F0870135CFE701204B
:100F4000F9E700BF004002202DE9F84380460F4634
:100F5000FFF7ACFF002840F09280FF2F03D94949EA
:100F600049480CF031FA494D7E1CD5F82432ABB11A
:100F7000D5E98A1232448A422CD9024631441846B5
:100F8000FFF7A4F9D5F824320446E0B90246D5F8B3
:100F90002C121846FFF79AF9C5F82442802E3446E1
:100FA00038BF80242046FFF776F90346C5F82402AF
:100FB000B8BB3046FFF76FF90346C5F8240278BB8B
:100FC00030460DF00DF8D5F828223244C5F8282215
:100FD000002BE3D0D5F82C2241464FF000089C1896
:100FE00032442046C5F82C223A4648F071F839467A
:100FF000204604F80780FFF73DFF8146686AD0E984
:101000000262B2422BD376000A2E38BF0A26C6EB04
:10101000C6001830FFF73FF948B9C5F82402CFE7FA
:1010200034460022C5F82842C5F82C22D2E700F148
:101030001802696A02EB86020160026102EB460255
:1010400042614A68C968C2F31E02C0F80C800A44B3
:10105000416862F31E014246C0E9011668620169F7
:10106000436921F81290911D9F546B6A43F8214007
:101070005868D968C0F31E0001311044D960BDE83A
:10108000F88300BF20EB070828B0080800400220C2
:1010900010B5044648F09EF801462046BDE81040D1
:1010A000FFF752BF07B5019001A8FFF7D3FE019AE1
:1010B000036933F8120003B05DF804FB07B5019033
:1010C00001A8FFF7C7FE019B4269D05C03B05DF841
:1010D00004FB07B5019001A8FFF7BCFE019B063396
:1010E00050F8230003B05DF804FB13B5019001A88C
:1010F0000C46FFF7AFFE019B4269D25C063350F805
:101100002300226002B010BD2DE9F8431D460023E4
:1011100007468846036016460B6013602B60154B2C
:10112000DFF854905C6A64B92B68326813442B6012
:10113000BDE8F883336812F8010B013303443360D0
:101140000DE04C45F0D03B6801333B60E268D8F8D5
:10115000003013446269C8F80030E368D1188A424D
:10116000E8D32046FFF77EFC2B68246803442B60FD
:10117000D9E700BF004002208C0C0908F8B50B4BE2
:101180000B4F5C6A0CB1BC4200D1F8BD04F11805EC
:10119000E36805EB8306B54201D32468F2E755F80E
:1011A000042B0449044800F023FDF4E7004002202A
:1011B0008C0C090825EB0708949E080830B500231D
:1011C000202511F8012F0AB9027030BD120600F176
:1011D00001041FD513B12023037020460B78124A57
:1011E00003F07F0363B9013A12F8013F044601306E
:1011F00013F0800F0BD003F07F0323700123E0E78F
:1012000012F9014B002CFBDA013BDBB2EAE700F8F4
:10121000013CE9E7012B04BF057020460B7800F87C
:10122000013B0223CDE700BF2CEB070838B543682C
:10123000054619440368994210D9037B1BB100216C
:1012400007480CF0C1F801F11004806824F007048D
:1012500008342146FFF72FF82C60A86038BD00BF86
:1012600028B0080870B504460E4611461546FFF72B
:10127000DDFF31462A46D4E90130184447F058FFD3
:1012800063682B44636070BD012938B538BF012104
:1012900004460025084621606560FEF7F1FF2573CE
:1012A000A06038BD38B505460C460131FFF7ECFFAC
:1012B0006C6038BD00230160C0E901320123037373
:1012C0007047000038B514460546FFF7DDFF024BB6
:1012D0002560636038BD00BF65120208037B10B54E
:1012E000044613B98068FEF7F3FF0023A36010BD26
:1012F00038B505461020FEF7C3FF04462946FFF720
:10130000C3FF204638BD10B5044648B1037B13B96E
:101310008068FEF7DDFF2046BDE81040FEF7D8BF2D
:1013200010BD000038B5037B04460D461BB10021FB
:1013300006480CF049F8016880682944FEF7BBFFB5
:101340002368A0601D441844256038BD28B00808F3
:1013500038B504460D46FFF769FFD4E901301D4456
:101360001844656038BDD0E9002310B59A420446A0
:1013700002D10121FFF7D6FF0021D4E90132D15477
:10138000A06810BD10B50C460121FFF7E1FF047005
:1013900010BD7F29F8B50C46CEB204D80121FFF765
:1013A000D7FF0670F8BD06F03F06B1F5006FC1F338
:1013B000871546F0800607D265F03F050221FFF74A
:1013C000C7FF46700570EDE705F03F05B1F5803FBA
:1013D000C1F3073745F0800508D267F01F070321E6
:1013E000FFF7B6FF457007708670DBE7A40C07F0C7
:1013F0003F07042164F00F0467F07F07FFF7A8FFA1
:10140000857004704770C670CCE738B505460C4649
:10141000084647F0DFFE214602462846BDE8384030
:10142000FFF720BFF8B5476804461646B94228BF03
:1014300039460D461146FFF7F9FEA368A8197A1B35
:101440005919184447F074FE6368A068334428446F
:101450006360F8BD43688B422CBF591A002141607C
:10146000704738B504461546084662688A4203D973
:1014700029448A4201D8606038BDA368521A1844D2
:10148000194447F055FE63685B1B6360F4E7084648
:10149000114648F04DBF70B5054608460E4647F068
:1014A00099FE044620B102466B6831462868984789
:1014B000204670BD2DE9F74F8A469DF830109146C1
:1014C0000D9A11F0DF0F0746A2EB090551D0302924
:1014D00053D1C3F34721002953D05F290BBF052601
:1014E00004262C482C4892FBF6F106FB112109B981
:1014F00001350132711E92FBF6F406FB14228A1AA2
:1015000000EB020813F020023ED005EBD573A5EBEB
:1015100063045D10002D3BDDAB465E4532467B68C3
:101520004146A8BF5A46386801929847019AABEBEA
:10153000020BBBF1000FF0DCB9F1000F05D04D44F8
:101540007B684A46514638689847002C0DDD254493
:10155000A642B1467B684146A8BFA1463868A4EBC5
:1015600009044A469847002CF2DC284603B0BDE83F
:10157000F08FDFF828801026C4E70DF1300801262F
:10158000C0E7DFF81C80F6E713F00104C2D02C4658
:101590000025D1E7A89E0808AD9E0808B39E08085C
:1015A0009C9E08082DE9F04F924693B0CA078046EA
:1015B0000D461C9C9DF874900593DDE91E760BD4B6
:1015C0008B0703D109687C4B994205D028460DF062
:1015D0008BFD450045F0010514F0210306D1B9F15A
:1015E000300F03D1B742B8BF37461E4628460DF12B
:1015F000280B10F0BAFF00281CDBA00716D52B2300
:101600008DF828300DF1290322079DF814101FD5FD
:10161000BAF1020F10D14FF0300C184600F802CB8F
:1016200001F1010C83F801C0034611E0610701D507
:101630002023E5E75B46E7E7BAF1080F5BD13020EE
:101640001870200649BF01F10E00013358700233B3
:1016500000200EAA012E1870A3EB0B030B924FF083
:1016600010020693C4F34723C8BF14438DF8270024
:10167000CDE90C2014F01002CDE90213059245D0FB
:101680002B460DAA0CA9CDE900A00BA810F030FE46
:10169000037882462D2B06D18DF8273000F1010A00
:1016A0000D9B013B0D93012E7ADD0D9D059BB542EF
:1016B000B8BF35462BB19DF8273003B10135069BE5
:1016C0001D4424F00103AF42079371DD14F00109BA
:1016D000A7EB05056DD1202301954A4637490093B4
:1016E00040464B464D46FFF7E5FE0446059B4FF04E
:1016F0003009C3B936E0BAF1100FA9D14FF0300C60
:10170000184600F802CB01F1170C8BE70AAB0DAAC3
:101710000CA90BA8CDE900A32B4610F0E9FD8246E9
:10172000C1E700252C469DF8273053B10023012244
:101730000DF127014046013FCDE90032FFF7BAFE27
:101740000444069B5BB10023012259464046CDE983
:101750000032069AFFF7AEFE069B0444FF1A012EE4
:10176000D8BF3E46079B51460D9A4046CDE90096AC
:10177000FFF7A0FE04444DB12023104940460195D7
:10178000009300231A46FFF795FE04440B980EAB16
:10179000984201D0FEF79CFD204613B0BDE8F08FC3
:1017A000059B0794002BBCD11D461C463E46D9E73D
:1017B000002500249AE700BFB4B50808375208088E
:1017C0002DE9F0430746900798468DB054BFC2F309
:1017D00080032B23164603A858BF5B010A464FF02F
:1017E0002101DDF8509058BFDBB20093159B0AF041
:1017F000A7FCF20504461FD52E2103A847F04CFD97
:10180000D0B9652103A847F047FDA8B96E2103A808
:1018100047F042FD80B9631C04F130022E210234EE
:101820006A44303302F8241C6B44302203F8242C21
:10183000A3186B4403F8240C73060ED504F1300290
:10184000631C00210DEB0204252204F8242C03F173
:1018500030021C466A4402F8241C16F010051DD004
:101860009DF80C302F2B4FF0000319D8012203A94B
:10187000384609F1FF39013CCDE90032FFF71AFE85
:101880000DF10D010546334622463846CDE9008963
:10189000FFF710FE28440DB0BDE8F08303A9F2E77E
:1018A00003A91D46EFE700002DE9F04F81468BB0FC
:1018B00014464FF000080B461D4613F8012B0AB1E1
:1018C000252AF9D1A94208D26E1AD9F80430D9F8DC
:1018D00000003246B044984729460B78002B00F0B0
:1018E0007F8120234A1C00270393134613F8016BC2
:1018F0003EB12D2E25D01ED8202E29D02B2E24D01F
:101900000026154612F8013BA3F13001092922D91E
:101910002E2B46D16B782A2B23D00023154612F8A4
:10192000011BA1F1300009281ED80A2000FB031B6F
:10193000ABF13003F2E7302EE2D147F01007039607
:1019400001E047F001071A46CFE747F00207FAE740
:1019500047F00407F7E70A2101FB0633A3F130063D
:10196000CFE7023554F8043B23EAE37B2B786C2B5A
:1019700008BF01352978002900F03281782906D87E
:10198000572911D8472959D8442900F21C81D9F880
:10199000043001222946D9F8000008F101089847CF
:1019A00085E04FF0FF3BE1E7A1F15803202BEED893
:1019B00001A252F823F000BF411A02088F19020851
:1019C0008F1902088F1902088F1902088F1902084F
:1019D0008F1902088F1902088F1902088F1902083F
:1019E000951A0208BF1A0208411A0208C71B02080A
:1019F000C71B0208C71B02088F1902088F190208AB
:101A00008F1902088F1902088F1902088F1902080E
:101A10008F1902088F190208411A0208D51A020804
:101A20008F190208FD1A02088F190208411A0208CC
:101A30008F1902088F190208411A02085029A6D1ED
:101A400001F0DF0354F804CB502B604668D16429C1
:101A50006AD1BCF1000F80F29D802D23CCF10000F3
:101A60000A228DF8173051230DF1280A0A3B0DF197
:101A7000180B8646B0FBF2FC02FB1C0160460929EC
:101A80008CBFC91830310AF8011DDA455CD07245A7
:101A9000EFD959E054F8043B019653B1039B04225B
:101AA000514900933B464846FFF704FD8044691CBA
:101AB00001E7039B05224D4900933B46F3E754F8A9
:101AC000043B012206A901968DF81830039B009370
:101AD0003B46E8E706A954F8040BFFF706FBBBF109
:101AE000FF3F014604D0069B9B4538BFCDF818B098
:101AF000039B069A00933B460196D4E754F804AB47
:101B0000504647F067FBBBF1FF3F024602D0584505
:101B100028BF5A46039B5146019600933B46C2E7B5
:101B2000642996D075292FD021F00F0300220F3B96
:101B30008DF817201022DBB2BCF1000F94D13023B6
:101B40000DF1270A8DF8273017F0100B9DF817308C
:101B50002DD0002B35D0039B01220DF117014846F3
:101B600000933B460192013EFFF7A4FC8346039B92
:101B70000AAA514648460093A2EB0A023B46019648
:101B8000FFF798FC584491E700230A228DF817309C
:101B90006123D1E7BB0705D52B238DF817300A2227
:101BA0005123C9E7C7F380035B01DBB2F5E7002BE4
:101BB000DDD006AA9245DAD90AF8013C0AF1FF3ACB
:101BC000D5E79B46D3E70734039B3A46484624F0C3
:101BD0000704CDE9006BB4EC020BFFF7F1FD65E7FC
:101BE00040460BB0BDE8F08F7C1B0808811B08083D
:101BF0000EB403B503AA52F8041B0192FFF754FE7A
:101C000002B05DF804EB03B070470346007893F927
:101C10000020002A0ADA00F07F004022104206D19C
:101C200013F8012F02F0C001802904D0704720EA88
:101C300002005208F2E702F03F0242EA8010EFE7AA
:101C4000431C18460133027802F0C002802AF8D003
:101C5000704703460020994200D8704711F8012DC3
:101C600002F0C002802A18BF0130F4E703460144A5
:101C7000002099421A4600D870471278013302F0CA
:101C8000C002802A18BF0130F3E700007F289DBF03
:101C9000024B185CC0F3400000207047C39E080848
:101CA0007F289DBF024B185CC0F3C0000020704726
:101CB000C39E08087F289DBF024B185CC0F38000BC
:101CC00000207047C39E08087F289DBF024B185C08
:101CD000C0F3801000207047C39E08087F2809D8F1
:101CE000064B1B5C13F00C0F06D1A0F15F035842AA
:101CF000584170470020704701207047C39E080874
:101D00007F289DBF024B185CC0F300100020704775
:101D1000C39E08087F289DBF024B185CC0F340108B
:101D200000207047C39E0808024608B5FFF7E8FF89
:101D300002EB401008BD08B50246FFF7EBFF40423A
:101D400020F01F00104408BD3038092884BF20F05F
:101D500020000738704702460144002010B5E524F2
:101D6000914203D8B0FA80F0400917E012F8013B25
:101D700030B103F0C003802B11D10138C0B2EFE7BE
:101D8000BF2B09D9F72B09D8DB0803F0060344FA67
:101D900003F303F00300E3E71B06E1D510BD0020C9
:101DA000FCE7023981420B4603D31A880239002A24
:101DB000F8D00233181A40107047B2EB131F70B5F9
:101DC00004464FEA13101BD901EB4001101A03F02F
:101DD0000F0326460246012A01F102010CBF31F829
:101DE000025C51F8025C013A25FA03F526F8025B21
:101DF000F1D104EB400434F8023C03B9013870BD62
:101E00000020FCE7F0B5059C0025121B2E46AC42D5
:101E10000FD101EB4403174600EB4404411A9FB96C
:101E200004EB420316B1023324F81260181A401072
:101E3000F0BD31F8157033F815C067443E4420F802
:101E40001560360C0135E2E71D88013F35445D52CF
:101E50002E0C0233E3E7F0B4049F00260D4634460F
:101E6000D11BB7420BD105EB47030A4600EB4707EE
:101E7000451B7AB907EB4101F0BCFFF792BF35F87B
:101E800016C033F816206444A41A20F8164024140F
:101E90000136E6E71E88013A34445C5324140233C9
:101EA000E7E72DE9F043079C0239DDF828E0154605
:101EB00084464FF6FF78A4EB0209DDE9087655B9B0
:101EC00000EB42011FB10123023120F81230BDE8BE
:101ED000F043FFF766BF31F8024F013D444426440A
:101EE00005EB0904A5422ABF33F8024B4FF6FF74F5
:101EF0004444744486EA040E360C17FA8EF74FEA0F
:101F0000144E2CF8027B3F0CD9E7022938B538BFB4
:101F10000221044680680D4618B12368B1EB930F87
:101F200007D96900FEF7C7F92368A06065F39F032E
:101F3000236038BD38B504460C20FEF7A1F90546EC
:101F400023682278C3F39D0023F0030302F001020B
:101F5000400013432B6063686B60FEF791F9A86043
:101F60002268A168C2F39D02520047F0B1F82846EA
:101F700038BD994210B511D313D800EB410002EBE4
:101F8000410209B9084610BD30F8023D32F8024D51
:101F90001B1B002B02DB04D10139F2E74FF0FF30AD
:101FA000F1E70120EFE710B5044638B18068FEF78D
:101FB0008FF92046BDE81040FEF78AB910BD70B514
:101FC0000C4602210546FFF7A0FF002C2B78B5BF79
:101FD000012200226142214662F30003AA682B70AD
:101FE000012388B21446090C1E4622F8020B03F1A5
:101FF0000103F6D16E60208070BD0023C0E900337C
:102000008360704728B103789B0702D48068FEF78D
:102010005FB9704738B504460D464968FFF775FF4C
:102020002A782378A06862F3000323706A68A9689D
:1020300062605200BDE8384047F04AB80A4629B904
:102040000178426062F3000101707047FFF7B7BF8B
:1020500008B5FFF7D2FFBDE80840FFF7EFBF9200D9
:1020600042F0020210B4026000225DF8044BC0E9A5
:1020700001211946FFF7E2BFF8B514461D469DF849
:10208000187004210646FFF740FF22462B4627B171
:10209000002D0CDA624265EB4503317867F30001ED
:1020A00031700021716052EA030102D1F8BD0027AE
:1020B000F3E7D6E901104C1C746020F81120120CD3
:1020C00042EA03421B0CEEE72DE9F84353EC102BD8
:1020D0001E46154603788046F20F62F30003037034
:1020E00047F6F07313EA16420AD198F8003023F04D
:1020F000010388F800300023C8F80430BDE8F883F5
:102100009A42F2D0C6F30A53A3F2FF34002CECDB60
:1021100004D10121BDE8F843FFF751BFA3F2EF3727
:10212000C6F31306332C4FEA271746F4801642DC19
:10213000C4F13402A4F11403C4F1140406FA03F345
:10214000D54026FA04F4D6401D4325430024A14679
:1021500039464046FFF7D9FEC8F80470B9F1000FC0
:1021600006D04FEA49020021D8F8080046F0F4FFF3
:10217000A4B105FA04F2D8F8083023F81920C4F104
:102180001003103409F10109A3F12002DD4006FA21
:1021900004F426FA02F2DE40254315434B469F42E3
:1021A000ACD0D8F8082022F813502D0C013345EAA2
:1021B0000645360CF3E70C34A3F2334304F00F0466
:1021C0004FEA2319C4E72DE9F8438F18C2F35B02E5
:1021D00004460D46511C9846089EFFF796FE23784C
:1021E000AC4600221FFA86FE68F300032370BC454C
:1021F0006046626002D3401BBDE8F88301780CF1B1
:10220000010CA1F13003092B05D9A1F14103192BD0
:1022100012D8A1F13703B342EDD2A06890468146AF
:10222000B8F1000F0FD100EB420113B1023120F8D9
:102230001230091A4A10DAE7A1F16103192BDAD832
:10224000A1F15703E7E7B9F8001008F1FF380EFBDA
:10225000013329F8023B1B0CE2E7F8B504461546AA
:102260001E46C1B1531E4FF0FF371E44E900204601
:102270000F310909FFF749FE2378002123F00103FC
:10228000616023700B4645B9A06800EB4101FFF780
:1022900088FD6060F8BD0127E8E700220F2B0ADC0B
:1022A0003078013D3E4400FA03F003F1080342EAAE
:1022B000000292B2F2D1A0680131103B00EB410064
:1022C000616020F8022CDEE738B5057804460B780B
:1022D00005F0010203F00103981A08D1D1E9013297
:1022E000D4E90110FFF745FEEB0748BF404238BD77
:1022F000884210B5044601D0FFF78CFE237823F006
:102300000103237010BD884210B5044601D0FFF7C9
:1023100081FE63683BB12378C3F3000282F00102BF
:1023200062F30003237010BD88421FB5044601D03C
:10233000FFF770FE626862B901212046FFF7E5FDF4
:102340000123A26813806360237843F001032370A4
:1023500010E02378D9070FD523F001032370012360
:102360000093A168ADF80E300DF10E030846FFF79B
:1023700072FD606004B010BD511C2046FFF7C5FD22
:1023800001230093ADF80E300DF10E03D4E90121C5
:102390000846FFF737FD6060D6E74B682DE9F04748
:1023A00005460E46144603B12AB931462846BDE813
:1023B000F047FFF72FBE02F10F014FEA111803EBB0
:1023C0001111FFF7A2FDA96814F00F044FF0000CE3
:1023D000D6E9012308BF102408EB020703EB4203F0
:1023E000C4F1100407F1004001384FEA400901EB45
:1023F00040001146864609BB6FF001032CFA04FC2D
:10240000C8F1010809F102095A43831820F802C0F3
:102410004FEA480203EB48035242184646F09CFE3E
:1024200003464B4417B133F8022D9AB12B786F60F5
:10243000327862F300032B70BDE8F08733F802AD09
:1024400001394AEA0C0C2CFA04FA4FEA0C4C2EF82B
:1024500002A9D0E7013FE5E72DE9FF410D464968B4
:102460000646144601B132B92946304604B0BDE8EB
:10247000F041FFF7CFBDFFF748FDB768D5F80880FA
:1024800023466A6838464146FFF797FC3378706008
:102490000246297861F300033370DB070AD5002375
:1024A00020096968ADF80E30994201D0834204D109
:1024B00081420AD804B0BDE8F08138F813509DB1CC
:1024C00001238142ADF80E3012D904F00F0401232C
:1024D00038F8101003FA04F4013C214206D1BDF88B
:1024E0000E30002BE6D003E00133DDE7ADF80E300F
:1024F000012312B93B807360DCE7009339460DF18C
:102500000E033846FFF77EFC7060D3E72DE9F341F8
:102510000D465768D1F8048014463B46926806463B
:102520004146A868FFF725FD01301FBF23462C4612
:1025300047461D4623782A785340DB0719D4791C77
:102540003046FFF7E2FC6B680093AB68B068D4E9F3
:102550000121FFF757FC70602378327800280CBF08
:10256000002303F0010363F30002327002B0BDE800
:10257000F08139463046FFF7C8FC6B680093AB68C2
:10258000B068D4E90121FFF766FCE4E72DE9F341E7
:102590000F464E68D2F8048014463146926843468E
:1025A0000546B868FFF7E5FC01301DBF23463C46F1
:1025B000B046012618BF1F46237818BF00263A7878
:1025C0005340DB0719D508F101012846FFF79DFCB0
:1025D0007B680093BB68A868D4E90121FFF712FC6F
:1025E000686018B1207800F0010070402B7860F32B
:1025F00000032B7002B0BDE8F08141462846FFF78A
:1026000084FC7B680093BB68A868D4E90121FFF7CC
:1026100022FCE5E74B682DE9F04F0C465168154662
:1026200085B08B42064621BF1946254613461C46F7
:102630002B78DB0722D4237813F001071ED1FFF794
:1026400064FCB068AD683B46D4E9011C99420CD1EA
:1026500000EB4101FFF7A5FB00237060327863F3C4
:102660000002327005B0BDE8F08F35F813203CF859
:102670001340224020F813200133E7E701313046B0
:10268000FFF743FC2F78237807F00109D5F804C041
:1026900087EA030147F30007B06803F0010AC94362
:1026A00043F30003A268834601F0010E41F30001E9
:1026B0009BB289B200930291B9B267460191A968B1
:1026C000A1F102086168A1EB0C0103918FB900EB45
:1026D0004C01BEF1000F03D00123023120F81C3061
:1026E000FFF75FFB706022782B78C2F30002134083
:1026F000B4E738F8021F013F019B5940039B89440E
:10270000D9198F4225BF32F8021B009B009959400E
:10271000029B8A4409EA0A014FEA1A4A4FEA194918
:1027200059401EFA81F14FEA114E2BF8021BCDE7FA
:102730002DE9F84F4B680D465168144606468B420A
:1027400021BF19462C4613461D462378DB0731D49A
:102750002B7813F001072DD1FFF7D7FBA068646831
:102760003B46D6F808C0D5E9012EA41A9A4213D1E7
:102770000CEB4203214600EB4202ACEB0000A1B996
:1027800003EB4403A3EB0C0358103378706061F340
:1027900000033370BDE8F88F30F813103EF8135083
:1027A00029432CF813100133E0E71588013915523D
:1027B0000232E4E701313046FFF7A7FB27782B7898
:1027C0004FF0010A616807F00108B06803F00109E1
:1027D000A46843F3000383469BB2A4F1020CD5E93D
:1027E00001E247F300050F46AEEB010EADB22FB983
:1027F00000EB4101FFF7D5FA0121C6E73CF8024F93
:10280000013F6C40A0440EEB0704A7422ABF32F8F8
:10281000024B1C465C40A14448EA09044FEA1949AE
:102820004FEA1848E4431AFA84F44FEA144A2BF8A2
:10283000024BDCE74B68F0B50D465168144685B095
:102840008B42064621BF194613462C461D46277863
:102850002B785F4017F0010736D1FFF756FBB068C1
:10286000D4E90121247814F00104D5E9015324D1DD
:10287000521BA54212D101EB4503144600EB45055E
:10288000411AACB905EB4201FFF78BFA0027337808
:10289000706067F30003337005B0F0BD31F8147059
:1028A00033F814C087EA0C0720F814700134E0E70D
:1028B0001F88013C5F520233E3E7CDE90277CDE99F
:1028C0000057FFF7EEFAE1E701310127FFF71DFBA3
:1028D0002B78DB4303F00103039323780197DB4359
:1028E00003F0010302936B680093AB68B068D4E90E
:1028F0000121FFF7D6FACAE74B682DE9F04F0446ED
:1029000085B00E4615460BB1536843B9237823F0C2
:10291000010323700023636005B0BDE8F08F81429E
:102920002DD1FFF707FBA542064607462ED06B6860
:10293000204671681944FFF7E8FA22680021A06870
:10294000C2F39D02520046F007FCB368D4F808E0D9
:102950000022D6F804900193F446AB680EEB4908C8
:10296000114602936B680393039B934233D0ACF1FF
:102970000200DDF804B00023CDF800901AE0824296
:1029800006D1FFF7D7FA05460746D0E70546CEE75A
:102990000027CCE730F802AF53443BF802AB1946AE
:1029A000029B33F8123003FB0A13009903800139AC
:1029B0001B0C009100990029ECD14146881C13B1F1
:1029C0000146A8F80030A1EB0E010CF1020C013217
:1029D00080464910C8E7616038462A78337853400A
:1029E000227863F30002227005B0BDE8F04FFFF7D4
:1029F000DABA4B6870B50546144613B11378DA0796
:102A000006D52B7823F001032B7000236B6070BD7B
:102A1000636823B90121BDE87040FFF7D0BA0846CA
:102A2000FFF788FA06462046FFF784FA012104469C
:102A30002846FFF7C4FA636883B1A3681B88DB07E5
:102A400004D5324629462846FFF756FF0123D4E92C
:102A500001210846FFF7B1F9606038B93046FFF749
:102A6000A2FA2046BDE87040FFF79DBA32463146D3
:102A70003046FFF741FFDEE72DE9F04F0C46516885
:102A80008FB09346013105460393FFF73EFADBF81A
:102A900004200021A86800260132520046F05CFBA9
:102AA0002B786E60204623F001032B70DBF80410B6
:102AB0000131FFF72AFA59462046FFF7ABFA039B8C
:102AC000D4F80890D4F8048048464146D3E9013749
:102AD00002933A46AB680493029BFFF74AFA002838
:102AE00033D10123049A606013806B60237862689D
:102AF000002A0CBF002103F0010161F300030399D8
:102B000023709BF8003009784B40DB0740F1FD80D3
:102B10006B682978003B18BF012363F3000129701B
:102B2000002A00F0F2800BA84FF0FF31FFF790FA77
:102B30000BAA29462846FFF7E9FC039A21462046BE
:102B40000FB0BDE8F04FFFF7E1BC013001D16E607E
:102B5000CCE7029B03F100423346013A4FEA420AB6
:102B600037F812100E0403F101004ED509EB4801AD
:102B70004FF0000C9BB208F101000191CE46C3F169
:102B80001006023129F818C0059660608E4540D3C2
:102B900037F812209A400592029A012A09D907EBC8
:102BA0000A02C3F1100132F8022CCA400599114300
:102BB0000591029A801A049A686000F10040013879
:102BC00002EB400207920AF102020992BA1E089231
:102BD000D4F804A0029A524529D30AF1004A0022EF
:102BE000C3F110000AF1FF3A09EB4A0AD14573D943
:102BF0006FF000416B682BB15A18049830F812201E
:102C0000002A73D06FF0004175E04900034689B295
:102C1000A8E7BEF8008008FA03F64CEA060C059E09
:102C200028FA06F82EF802CB1FFA88FCAEE7019AC4
:102C30000198118832F8022C42EA01420599B2FB50
:102C4000F1F20999411A0020069186460899069FDB
:102C50000E460199B9420DD809880844A8BB0799C6
:102C600021F80229019A0791023A01920AF1FF32F2
:102C70006260ADE736F8021FB7F80080994018FA95
:102C800080F841EA1E4E1FFA8EF151431FFA81FC73
:102C9000090CA8EB0C0CC1EB204127F802CB01EB8F
:102CA0002C40D6E738F8021F994041EA1E4EBCF886
:102CB0000010394411FA8EF10F0C2CF8021B019907
:102CC0006145EFD83844013AC8E70027DDF8208095
:102CD000DDF818C0BE46F2E7BAF8001041FA03F674
:102CE000814032432AF802298AB27FE7013B6B60B8
:102CF00080E7013B63606368002B3FF4F7AE5A182E
:102D000039F81220002AF4D0F0E60FB0BDE8F08FB9
:102D1000F0B51F464B6885B004460D4616464BB1CC
:102D20001378DA0706D47B68012B0BD1BB681B88AC
:102D3000012B07D1237823F0010323700023636064
:102D400005B0F0BD01212046FFF739F97368002B6B
:102D5000F6D02846FFF7EEF805463046FFF7EAF8CA
:102D6000002306460393CDE901337368B3B1B3681A
:102D70001B88DB070AD52A4621462046FFF7BCFD03
:102D80003B462246214601A8FFF776FE0123D6E9FD
:102D900001210846FFF711F8706058B901A8FFF744
:102DA00031F92846FFF7FFF8304605B0BDE8F0409E
:102DB000FFF7F9B82A4629462846FFF79DFD3B460E
:102DC0002A46294601A8FFF757FECEE7D0E90121A0
:102DD0000346002001EB420210B5914204D31B7858
:102DE000DB0748BF404210BD32F8024D44EA0040C4
:102DF000F3E730B5D0E90124002304EB420294420A
:102E000006D302780120D20748BF5B420B6030BD79
:102E1000B3F5004F04D232F8025D45EA0343EEE712
:102E20000020F4E7037813F0010310B510D1D0E9C6
:102E3000012404EB4202944202D301200B6010BD36
:102E4000B3F5803F04D232F8020D40EA0343F2E7C3
:102E50000020F4E72DE9F74FDDF830C006460F46B5
:102E6000019209B30CEB0300012400211A46A2468B
:102E70008E46D6E90189B8F1000F17D101990029D2
:102E800045D0002A43D1002B41D0002F3BD09CF8E5
:102E900000302CB1DB43347884EAD31404F001040D
:102EA000204603B0BDE8F08F6046DDE739F8025BED
:102EB0000EF1100E45EA0141BEF1070F02DC08F1E8
:102EC000FF38D8E796F800B08DB21BF0010F1FBF96
:102ED000ED435AFA85FA1FFA8AF5CAF3072A42B96E
:102EE0001CB1EDB2B5FA85F46409AEF1080E090A19
:102EF000E2E7EDB227B100F8015C0138013AF4E7EE
:102F000000F8015BFAE7634413F8013CC1E733784A
:102F100013F0010F14BFFF210021002F18BF6046DE
:102F200046F01AF9BCE70000D0E901329FED0C0B26
:102F30009FED0D6B02EB43039A4205D30378DB0749
:102F400048BFB1EE400B704733F8021D07EE101A70
:102F5000B8EEC77BA0EE067BB0EE470BECE700BFF8
:102F60000000000000000000000000000000F04031
:102F70000A292DE9F74F1546446814BF042203229D
:102F8000804689469DF830A00D9E0092A4B98DB16F
:102F9000013D324615F8011F134641B930221A701F
:102FA000002203F8012F981B03B0BDE8F08F02F850
:102FB000011BEFE73346F1E764000193B346204677
:102FC000FDF75EF92246D8F80810074646F080F86B
:102FD000019B304607EB040C3A3BACF102040021A4
:102FE000A742A6461DD930315C46392988BFC91889
:102FF00004F8011B39468C458E461DD83846FDF72E
:1030000067F965BB98F80030DB0744BF2D2304F84F
:10301000013B3346621E9A4233D80023A01B237023
:10302000C2E7BEF800E04EEA014EBEFBF9F124F81B
:10303000021909FB11E1D3E7BEF800200231002A92
:10304000D9D0BAF1000F08D0211A009A914204D1C8
:103050000BF102048BF801A02046A346BDE72846E9
:1030600046F0B8F829185A460B46AB4204D88D42B0
:1030700088BF00200444C5E713F8017D02F8017FF2
:10308000F3E71978107803F8010B02F80119C2E789
:10309000D0E9023293423DBF5A1C826018784FF04B
:1030A000FF3070470368013B033310B5044602D874
:1030B0004068FDF70DF92046BDE81040FDF708B95E
:1030C000F8B50C461F46164605461020FDF7D8F801
:1030D000054B8460C0E900743444C4606B60034BEA
:1030E0002860AB60F8BD00BF91300208A53002082F
:1030F00002690A2AF8B504461BD18369013383614A
:103100000123E3610026237D0A272361637D237564
:10311000256EB5B16B1CA26D2366555D626D934241
:1031200001D366652666237D0D2B14D0BDB1657570
:10313000F8BDC369092A04BF073323F0070301332D
:10314000DFE7D4E901039847431CECD0012838BFDE
:1031500001200546E7E70A2D2775D9D0E6E7237D4C
:10316000002BE4D00A2B18BF0A25E0E701690246CC
:10317000272901D0222912D1012024E0137D272BF9
:10318000FAD0222BF8D0722914D1662B16D1507D9B
:103190002728F1D0A0F12203584258417047A1F1ED
:1031A0006200132804D8084B034113F00100E5D056
:1031B00000207047662904D1722B00E0622B02D1F7
:1031C000E5E76229F8D07047EEFFF6FF38B5044610
:1031D0000D462069D0B10A2806D10DB1636AB3B19A
:1031E0002046FFF785FFF4E7FEF750FD0028F7D1F2
:1031F0002369232B08D12046FFF77AFF2369002B90
:10320000E7D00A2BF7D1E4E75C2B02D00025284653
:1032100038BD237D0A2BF9D12046FFF769FFDFE790
:10322000002301212DE9F04F044685B04364FFF7E8
:10323000CDFFA369276A6363002FE369A36307DAFD
:103240000723013784F83C30276205B0BDE8F08FD2
:1032500004D00623013F84F83C30F5E7002835D040
:1032600039462046FFF7B2FF0523E56984F83C3074
:10327000013DD4E90B3003F10042013A30F812204D
:103280009542E2D009D8013B30F81320954218D37B
:10329000DBD0022384F83C30D7E7A16A8B4207D306
:1032A00008314900FDF707F8A36A20630833A362D9
:1032B000E36A5A1CE26220F81350236A0133236246
:1032C000C3E7226AE362013A2262DCE7256915B9A5
:1032D00084F83C50B9E72046FFF748FF064600282F
:1032E00000F00B8284F83C702369722B6BD008D8F5
:1032F000622B0CD0662B70D0B9460025A8460B2354
:103300000DE0753BD3F1000949EB0309F5E7237D97
:103310000025722B69D0A8464FF001090C2394F8C0
:103320003C20002A6AD184F83C30B9F1000F08D063
:103330002046FFF7DDFEB9F1020F02D12046FFF76C
:10334000D7FE23692046222B0CBF2223272301937B
:10335000FFF7CEFE2369019A934240F08680237DD9
:10336000934240F0828020464FF00309FFF7C0FEF1
:103370002046FFF7BDFE35B1A36E23B9A44904F181
:103380006400FEF742F804F140034FF0000B029393
:103390002169002900F0A881B9F1010F02D10A29A1
:1033A00000F0A281CB4563D3594604F14000FEF7FB
:1033B00051F801212046FFF709FF2046FFF7D6FE0E
:1033C000002891D11CE0237D622B0DD0662B10D0FC
:1033D0000025B0464FF0010991E7237D3546722B59
:1033E00008D04FF00008F5E70025B0464FF002097D
:1033F00094E73546B0464FF0020980E79A4294D0F0
:10340000A36E002B3FF421AF292104F16400FDF7E6
:10341000B9FF236E04F15006002B40F06B810321AD
:103420003046FDF795FF23690370237D4370637D6C
:103430008370216E3046D4E91A572A46FDF7F2FF11
:103440002A46394645F044FE0023A26DA366236E4A
:10345000581C2066D15C2161991C03332166105CE5
:1034600023662075535C6375EFE64FF0010982E730
:10347000019B8B4209D1194602980BF1010BFDF714
:1034800088FF2046FFF734FE82E7002D60D15C29DB
:1034900040F0278120460391FFF72AFED4F810A0C0
:1034A0000399B8F1000F6CD00298D346FDF771FF75
:1034B000D2E004F1640B28215846FDF763FFD4F8ED
:1034C00068A00022216979B172BB3A290CD07D290C
:1034D0000AD0212928D1207D7238012829D8607D81
:1034E0003A2801D07D2824D1D4E91A21881810F86F
:1034F000010C3D2809D1A2EB0A02514404F140001D
:10350000FDF7B0FEA26E013AA266924558464FF012
:10351000290104BF042384F83C30FDF733FF2C213C
:103520005846FDF72FFF24E021F020005B280AD148
:103530000132C9B258460392FDF724FF2046FFF737
:10354000D7FD039ABEE75D2808BF02F1FF32F0E71E
:103550007B299CD120460391FFF7CAFD23697B2B71
:10356000A7D104F140000399FDF70CFF2046FFF7B7
:10357000BFFD7B2104F140004FF0000BFDF702FF7F
:1035800006E7BAF1780F09D8BAF15B0F0AD8BAF199
:10359000220F53D029D8BAF10A0F23D05C2104F1AD
:1035A000400082E7AAF15C021C2A73D8DFE802F02F
:1035B00046727272728A2A7272723A72727272727F
:1035C0007272347272720F722D3D37725C004FF05E
:1035D0000D0B94F83C300B2B77D1594604F1400089
:1035E000FDF7D7FE4FF0000B4BE7BAF1550F1CD09B
:1035F000D4D8BAF1270F21D0BAF14E0F4AD10548DD
:103600000AF0D2FE4FF0080BE3E74FF0090BE0E7BA
:10361000CC1B0808D51B08084FF00A0BD9E74FF060
:103620000B0BD6E74FF00C0BD3E794F83C200C2A99
:1036300006D15C2104F14000FDF7ABFED346C8E79C
:10364000BAF1750F14BF4FF0080A4FF0040A4FF09B
:10365000000BBAF1010A0AD2BBF5881FB9D34FF0AB
:10366000010384F83C30BDE74FF0020AEFE7204643
:10367000FFF73EFD226910460392FEF725FB002866
:1036800000F04F81039A4FEA0B1B1046FEF75CFBDC
:103690008344DEE7AAF1300BBBF1070F3FF67EAFA4
:1036A0004FF0030A06E02046FFF722FD2269303A78
:1036B00002EBCB0B227D303A072ACDD8BAF1010AB2
:1036C000F1D1C9E74FF0070B83E7BBF1FF0FC6D875
:1036D0000C2BC4D15FFA8BF104F14000FDF752FED0
:1036E00080E7C9B20298F9E7CB453CBF032384F8D1
:1036F0003C3059E6033B23669BE62846FEF7D0FAAA
:103700002169D8B95F2919D07F2917D80846FEF753
:10371000D1FA002855D123692E2B4DD00026834D98
:103720002F781FB12369BB4240F0A4802046FFF7E9
:10373000DFFC002F40F0A6800123ABE5082304F155
:103740004005C9B284F83C302846FDF71BFE2046F0
:10375000FFF7CEFC2069D8B92846754FFDF703FE68
:103760000025064657F8041B304645F041FD002869
:103770001CD10E35EDB2112D84F83C507FF465ADAF
:103780006C4BD3F83032002B14BF0E23102381E58D
:10379000FEF786FA40B920695F2805D07F2803D854
:1037A000FEF788FA0028D7D0217CCDE7FFF64DAD93
:1037B0000135242DD6D148E5207DFEF77BFA00287F
:1037C000ACD021692E292AD10A2384F83C30002567
:1037D00004F140060A273046FDF7DBFD2046FFF7DF
:1037E00087FC206900283FF430AD55BB20F0200352
:1037F000452B26D16521304684F83C70FDF7C9FD84
:103800002046FFF775FC21692B2901D02D29E8D12D
:103810003046FDF7BEFD2046FFF76AFCE1E70923CD
:10382000302984F83C30D2D1237D43F02003623B21
:10383000DBB2162BCBD8404DDD4015F00105C7D1CA
:10384000C5E7FEF72DFA28B121692E290DD184F89C
:103850003C70DDE72069FEF72DFA0028F4D12369DA
:103860002E2BF1D05F2BD6D0EFE421F020034A2B92
:10387000CED1ECE7652F01D0632F00D101350136A1
:1038800001354DE7212F08D123693D2B7FF454AF3B
:103890002046FFF72DFC3923FCE42E2F0FD123699E
:1038A0002E2B02D1237D2E2B01D05C23F2E4204667
:1038B000FFF71EFC2046FFF71BFC0D23EAE403354F
:1038C000334615F8027C632F18D0652F16D01B4A9B
:1038D000D35C84F83C30543BDBB2052B3FF6B5ACEF
:1038E000012202FA03F313F02A0F17D113F0150F78
:1038F0003FF4ABAC636A13446362A6E415F8012C91
:1039000001362169914207D12046FFF7F1FB33468A
:10391000652FDCD00235D4E7632FFAE7636A013BF9
:10392000EAE70123834684F83C3052E6871B080807
:10393000449F08080040022001204000D49F08084E
:103940007FB501AD0646742085E80E00FCF798FCB3
:103950000446034695E8070043F8046B002583E816
:10396000070001236FF001021420C4E906320A2285
:10397000C4E90855C4E90A23FCF782FC202120632E
:1039800004F14000FDF780FC294604F15000FDF7EA
:103990007BFC294604F164002566FDF775FC236B6A
:1039A00020461D802561A582FFF7A2FB2046FFF778
:1039B0009FFB2046FFF79CFB2046FFF731FCA36BE3
:1039C000012B06D094F83C30052B1CBF062384F84D
:1039D0003C30204604B070BD30B585B0054601AC22
:1039E0002046FFF76DFB284694E80E00FFF7A8FF7E
:1039F00005B030BD30B585B00446014601AD28465E
:103A000023F044FA204695E80E00FFF799FF05B031
:103A100030BD10B50446B0B1C3684068984704F1A2
:103A20004000FDF75BFC04F15000FDF757FC04F18A
:103A30006400FDF753FC206BFCF74AFC2046BDE810
:103A40001040FCF745BC10BDD0E90432013B0361D6
:103A500052F823007047036942695B1A013B52F830
:103A600023007047F8B5446A06460D46B4B1D4E960
:103A700000030B44834222D908310022014420462E
:103A8000FCF724FC0246B8B9616820460831FCF70F
:103A90001DFC63682360336A63603462802D2F46A7
:103AA00038BF802707F10800FCF7EAFB0023076016
:103AB00004464360706202E023682B442360606820
:103AC0000834054444F8045C2044F8BD38B50D467C
:103AD0000C211446FFF7C6FF4FF49D720560C0E944
:103AE000012438BD38B5D0E9033204460D469A4268
:103AF00008D3103340699900FCF7DDFBE36860618F
:103B00001033E360D4E90432591C216142F8235098
:103B100038BDF8B504461D460F461646D0E90003E9
:103B2000834208D31030C100A068FCF7C4FB2368AF
:103B3000A06010332360D4E90103421C626003EBF0
:103B4000C00253F8301067F3170143F83010D670F5
:103B50005560F8BD10B48469CAB20023616B5DF88A
:103B6000044BFFF7D6BF0000F0B593B004460E46F5
:103B7000174668461D46FCF743FB10B1002013B002
:103B8000F0BD3A46314620460AF046FA0446FCF7B4
:103B90000DFBA30703D12268024B9A42EED001200D
:103BA0002C60ECE7A0AC080810F00102034604D03A
:103BB00040F001030B6001207047A8B110F0030032
:103BC00013D11A793A2A11D19B6813F001000B60C6
:103BD000F1D19A070AD11868054B9842EBD0054BF2
:103BE000C31A58425841704770471046704700BF8B
:103BF000B4B5080834B3080810F001021CD110F065
:103C000003030CD000F00F03062B15D00A2B11D1A3
:103C100000090D3803288CBF00200120704770B1C7
:103C200002793A2A08D02D2A08D18068B0FA80F0AB
:103C3000400970471046704701207047184670478A
:103C4000C20702D540F001007047830710D0030976
:103C500000F00F00062803D1D80040F002007047A2
:103C6000A3F10E00022809D8064B53F82000704734
:103C700030B103793A2B03D180687047024870470E
:103C80000248704700A00808A4BC0808D8C008086B
:103C900038B505460C46FFF7AFFF38B12846FFF7A9
:103CA000CFFF0BF06DFB031B5842584138BD2DE987
:103CB000F0410F4605461446114689B9204612F0D8
:103CC0005DFF014600F10808A4B90A4628463946B6
:103CD000FFF7FCFE01462846FFF704FF012007E03E
:103CE00001392846FFF7B7FEFFF786FF0028E4D129
:103CF000BDE8F0812846013CFFF7A6FE0646FFF727
:103D00009FFF48F82400002EDED0B307DCD1686A9C
:103D100000F108039E42D7D3426813449E42D3D297
:103D200073681B0A0233A2EB83024260CCE70000F7
:103D3000F7B5866905460F4696F83C20A2F10803C0
:103D4000042B52D8DFE803F003232B384C00D6E9CC
:103D50001110FDF7F9F8902F04460ED1C100002292
:103D600005F1280041F002010AF0B8FE28B14268CE
:103D7000D3071CD542F0010002E0200140F0020010
:103D80000146284603B0BDE8F040FFF7ABBE002275
:103D90003346D6E9111008F051FC0246E8E70096D8
:103DA00000230122D6E9111008F0A6FD0246716B2E
:103DB0002846FFF78BFEE3E7D6E911100A2906D85B
:103DC000FDF7C2F830B1000140F00600D8E7FDF77A
:103DD0006DF8F7E7D6E91121064810F0B7FFE5E7DF
:103DE000D6E9111011F092F8E0E7120142F00A0052
:103DF000C6E700BFCCBF080810B5FFF7D5FE50B12D
:103E00000B6813F0010007D19A0704D11868034B1F
:103E1000C31A5842584110BD0120FCE7B4B5080848
:103E20000021FFF735BF0121FFF732BF2D2A2DE911
:103E3000F04F044685B0884616461D460BD100213A
:103E4000FFF709FEC0B1820702D10379922B13D08C
:103E500005B0BDE8F08F922A2ED10021FFF7FBFDBF
:103E6000014648B1830707D14768FBB2952B18D1AB
:103E7000013D2046FFF7E8FDA6F12303DFB2092F3D
:103E800000F2EB80092B00F2CF80DFE813F0ED00A9
:103E9000ED00ED001F011F011F014601ED00CD00E7
:103EA0009001962BE8D127F0FF072046FFF7CCFDC5
:103EB00047F092074F60CBE7962A13D10135D0E93E
:103EC000012303EBC20313F8153C2D2B40F0AD800A
:103ED0002A46FFF7ECFE002800F0A7806368023B4B
:103EE0006360B5E7A2F11E03012B5FD9202A00F021
:103EF0008380052AC0D10021FFF7ADFD07460028C9
:103F000000F0938010F0030A05D1436803F0FE032C
:103F1000562B00F08A8001212046FFF79CFD00F01F
:103F20000F03022B40F08180BAF1000F7DD13B7965
:103F30002C2B7AD1BB6803F00F02022A75D11B0922
:103F4000482B72D1FB68002B6FD09A076DD11A797C
:103F5000302A6AD1D3F808B04FEA10195846FFF753
:103F60004BFE002840F0FE80B749B8480DF032F90A
:103F7000A169054653463A6809680DF00DFA2846CE
:103F8000FCF756F91E2E0AD1FFF74DFF18BB384635
:103F9000FFF746FF00B9D3460BF1FF3A0BE0FFF7FE
:103FA0003FFFC0B93846FFF73EFFF3E705F1FF3AA0
:103FB0008DB1AB46A94609F1FF3920464946FFF7C6
:103FC0004AFD236962690746A3EB0B0342F823000D
:103FD000B9F1000FD6D10021514508D16D1A012D3C
:103FE0003FF436AF362E00F04281332E3DE12046BD
:103FF0000131FFF729FDEFE70021FFF72CFD074610
:10400000FFF70EFF68B93846FFF70DFF68B1EA21E8
:104010002046FFF719FD204605B0BDE8F04FFFF739
:1040200061BD4FF48571F3E72B26A91C204689005A
:10403000FFF718FD074646EA052300F10801C0F81E
:1040400000804360002D40F01B81962E03D139463D
:104050002046FFF747FD3946DDE7922E00F0FE804F
:10406000062E00F00481BDE7691E2046FFF7F3FC31
:1040700001A9FFF799FD0028B7D0022FA5F102078B
:1040800096BFA6F10D094FF022095FFA89F9002FBA
:1040900009DA002D40F0CD80019AD30740F1CE809F
:1040A00042F00101B7E739462046FFF7D4FC02A9E8
:1040B000FFF77AFD002898D001AB4846DDE90112F0
:1040C000FFF752FD002890D0013FE0E7691E20462F
:1040D000FFF7C1FC01A9FFF767FD002885D0AF1EDF
:1040E000002FD6DD791E2046FFF7B5FC02A9FFF7A9
:1040F0005BFD00283FF479AF39462046FFF7ABFC63
:1041000001AB00092438DDE90112C0B2FFF72CFD34
:1041100000283FF46AAF023FE2E700212046FFF7A4
:104120009AFC01A9FFF740FD00283FF45EAF012192
:104130002046FFF790FCC0F30710019933280BD1FC
:10414000CF0707D488077FF450AF0A68404B9A42E4
:104150007FF44BAF022001E03F38C0B209F08EF986
:10416000019096E75846FFF76BFD07464FEAC903F3
:104170000A4604F1280043F002010AF0AFFC476050
:104180004846FCF7A6FF037820465F2B08D10025A0
:10419000FFF75AFC20460826A846FFF755FC6BE6B9
:1041A000FFF752FC59462046FFF79CFC3DE70121F2
:1041B0002046FFF750FC00F00F030746022B7FF468
:1041C00014AF00212046FFF746FC00283FF40DAF56
:1041D00010F003027FF409AF0379322B7FF405AFAF
:1041E0003909D0F808901B48C90041F002010AF0D3
:1041F00075FC00283FF4F9AE02AA4FEA1911406895
:1042000009F07EF8029B002B3FF4EFAED9070AD4E9
:104210009A077FF4EAAE1A680D498A4203D00E4924
:104220008A427FF4E2AE039A002A7FF4DEAE019365
:104230002FE72046013DFFF707FC2AE729462046E5
:10424000FFF744FC0146E6E65E1C0808E0AF0808FC
:10425000B4B508080CA0080834B30808D4E9012351
:1042600003EBC20313F8053C2D2B7FF4DEAE2A4688
:1042700041462046FFF71BFD00287FF4E9ADD4E658
:10428000013D2046FFF7E0FB41F82500DAE600BFDC
:104290000346006830B550B184070AD14468E5B2DE
:1042A0008D4206D100F10803200A136030BD034699
:1042B000FBE70120F9E700002DE9F04FA94B97B08B
:1042C0000D460024029005A80192CDE90731A649C8
:1042D000FBF774FF40234FF40070CDE90934FBF77E
:1042E000CFFF20230B908020CDE90C34FBF7C8FFD3
:1042F0002146CDE90E0513A8CDE911440AF0B8FB1B
:10430000019B002B48D0022B0CBF3F2222460023EA
:10431000696B09A8954FFFF7FCFB00230A9C002C52
:1043200000F06481013C0B99914801EBC40251F803
:1043300034100A94D678C1F3170A8E49632E526856
:1043400011F806B08C490BF00F09895D88BF41F464
:10435000807100EB41080BF0300110291ED020299C
:104360004BD0002B00F01B81B9F1020F40F00A8105
:10437000012A40D000211BF0010F02F1FF3306D0CB
:10438000B8F802003840B0F5805F08BF5308012B31
:1043900040F0E580E1B1E2E03D22B8E702B1BBB117
:1043A00008EB420825E0C34638F8023B03EA070160
:1043B000B1F5805F0ED195F83C10C3F30B03994221
:1043C00016D109A83146FFF7B3FC2846FEF728FFAF
:1043D0000023A3E7531C4B4504D23246514609A89B
:1043E000FFF797FBBBF8001009A8FFF7B3FBEFE757
:1043F00001329145D7D8012390E773B102F1004310
:10440000013B38F813303B40B3F5405F21D1002128
:1044100009A80392FFF766FB039A08EB4204914553
:104420002BD8019B83B1052E0ED1002109A8FFF7DF
:1044300012FB48B9012109A8FFF70DFB830744D0FF
:1044400000F00F00022845D1002408EB4903A146E3
:104450005AE0012ACFD995F83C30062B40F0F48081
:10446000464947480CF0B6FE044600236A6B2968AB
:104470000CF092FF2046FBF7DBFE039434F8021B9E
:1044800001EA0700B0F5805F16D1C9B295F83C008B
:1044900088420ED1082805D1314609A80392FFF7BA
:1044A00047FC039A28460392FEF7BAFE039A0132AC
:1044B000B5E7002A9FD0CEE7531C5146324609A8E3
:1044C000FFF727FB039B19888EE70028BCD00379F0
:1044D0003A2BB9D109A8FFF7B7FA09A8FFF7B4FA40
:1044E00000230822514609A8FFF7A0FC70E733F823
:1044F000022D02EA0701B1F5805F10D1D2B2082A7D
:1045000002D1013409F101094345F0D1B9F1010F9C
:104510001CD11BF0400F19D00026314610E0214677
:1045200009A80393FFF797FA039B08B109F1010962
:104530000134E9E7FFF788FA0136002818BF014681
:10454000A64209A8F6D1FFF7CDFA41E71BF0800F8C
:1045500004D00134002109A8FFF7C4FA23463246EB
:10456000C0E700BF133A020803D2020800F0FFFFC1
:10457000F8A0080880A4080848A008086A1C0808D1
:10458000BCAF0808012A3FF436AF12F001013FF436
:10459000F2AEB9F1030F7FF45EAF0121EBE609EA59
:1045A000020303F0010338F8134004EA0701B1F5F0
:1045B000805F13D1C4F30B0495F83C10A14202F1C3
:1045C000010409D11BB9314609A8FFF7B1FB284600
:1045D000FEF726FE2246E2E72246C5E6531C514678
:1045E000324609A8FFF795FA2146FDE613A80AF01E
:1045F00053FA129850B1416822460831FBF766FE23
:10460000129B5A681A60119A5A60119395F83C30BF
:10461000002B7FF420AF0D9B002B3FF41CAF0E9BB3
:104620000B981B681093FBF753FE0E98FBF750FE98
:104630000120FBF7CBFD029BDDE9100183E80300BD
:10464000184617B0BDE8F08F022B01D1034908E7E7
:10465000042B03480CBF0349034903E7731C0808F4
:10466000E0AF08089A1C0808AD1C080838B50446D5
:10467000406808B9606038BD4568FBF729FE2846E8
:10468000F7E70000F8B5054630200E461746FBF761
:1046900010FE072D04460570C66001D0012D0FD114
:1046A000B368C3F30F13A38208F00AFA042320614E
:1046B00020202783E384FBF7E3FDE0622046F8BD7A
:1046C000014B5B5DEFE700BF30A5080810B504465D
:1046D000C06AFBF7FDFD2046BDE81040FBF7F8BDC2
:1046E00030B500220446058D954201D8002030BD2A
:1046F000E36A03EBC20043688B42F8D00132F3E770
:1047000070B504460D461646FFF7EAFFC0B9E38CC4
:10471000228D9A4208D30633E06AD900FBF7CBFD1D
:10472000E38CE0620633E384238DE26A591C02EBDA
:10473000C300218502F83360002345604370438045
:1047400070BD034618465B68002BFBD1FFF7C8BF5E
:10475000F8B544680E462CB9F8BD042BFCD10523EE
:104760000370F9E7254628466D68002DF4D0776878
:104770003946FFF7B5FF0028F5D00378043B022B3C
:10478000EAD806253570002239462046FFF7B8FFE3
:104790000378002BE1D105706468F4E7036A1B8B92
:1047A000012B1EBFC3685B18C3607047836A10B5D6
:1047B00004469B6F406A9847238B226A0133918C91
:1047C0009BB29942238338BF938410BD038B013B76
:1047D00010B503830446836A406AD3F8843098474F
:1047E00020460121BDE81040FFF7D8BF2DE9F04F6A
:1047F00085B004460D46984603921BB1CB8A43F020
:104800000803CB82039BEB83236ADA8A42F03002EF
:10481000DA821B78002B46D1A36A2946039AD3F883
:10482000B4604346606AB44605B0BDE8F04F6047E7
:10483000DB6A03EBC60B13F83630053B012B1DD8A2
:104840004FF0000917E0EB6A03EBC90213F83930A7
:10485000062B0ED1DBF804105368994209D1A36AE4
:104860000AF1010ABBF802201B69606A1F46002397
:10487000B84709F101092B8D4B45E4DC0136236A69
:104880001A8DB242D4DCBAF1000FC5D0A36A5246E9
:10489000CDF800802946D3F8B860606A039BB04722
:1048A00005B0BDE8F08F0026B246E8E7836A002134
:1048B00010B50446D3F88830406A9847A36A606A06
:1048C0000F211B6B9847A36A606A0121D3F8CC3093
:1048D000984720460321BDE81040FFF75FBF38B579
:1048E000836A04460022406A5B6C9847A36A606A48
:1048F000D3F8C05000231A461946A8472046BDE801
:104900003840FFF7D3BF836A002289681B6D09090D
:10491000406A1847836A8968DB6B406A184710B59C
:104920000446084611461A46FFF7ACFE236A436068
:1049300000238360E3690BB9E06110BD1A469B68F0
:10494000002BFBD19060F8E72DE9F04F87B00546CA
:104950000C4600AF11B90121116013E011F00306FC
:1049600019D10B79682B19D1CB681B0913608C689E
:10497000002CF0D0012604F00F03022B0DD12109E9
:10498000002EE9D0AB6A0022686ADB6A98471C37C0
:10499000BD46BDE8F08F0026EDE716B9A3681B09F8
:1049A0001360A04658F8043F4FEA132AC14608EBAB
:1049B0008A030AF1FF3BBB6059F8040F0009FCF7BA
:1049C0007DFBBB6883449945F6D10BF1070323F0C7
:1049D0000703ADEB030D0023E946C7F80CD058F8E8
:1049E000040F07F114013B600009FCF77EFB7A69B4
:1049F000014648467A6044F06BFB3B687A680133B5
:104A00004A449A4505D091464FF02E0209F8012BF1
:104A1000E5E75946F868FCF797FAAB6A01460022C9
:104A2000DB6A686A9847002EB1D00834BB689C42A4
:104A3000ADD054F8041F0022AB6A0909686A1B6DE7
:104A40009847F3E731B101F003038268134304BFD1
:104A50000B68836070472DE9F04107461E4659B147
:104A600011F0030510D14B68D8B290420CD14FEA37
:104A700013280C1D454501DBBDE8F08154F8041FE7
:104A800038460135B047F5E738463346BDE8F041D2
:104A900018470000F8B50E4611461A460023044692
:104AA00085780769837003610E4BFFF7D4FF636855
:104AB000BBB9618A51B1228A42B9A36A606AD3F84C
:104AC000A0309847A36A606A1B6C9847238A3146D6
:104AD000628A2046FFF78AFE003D276118BF012544
:104AE000A570F8BD3D53020870B5437805460C46E5
:104AF000012B06D1036A0A4602211B8BFFF70FFF29
:104B00002061A268284621694C23BDE87040FFF768
:104B1000C1BF70B51346427805460C46012A04D140
:104B20000A460721FFF7FBFEA061A6692846462337
:104B3000E2683146FFF7AEFFB08A70BD024B9D229E
:104B40008968FFF788BF00BF49580208024B6B22F3
:104B50008968FFF780BF00BFE173020838B543687A
:104B60000D46044611464BB905480CF033FB294667
:104B700060602046BDE83840FFF764BF38BD00BF25
:104B8000E0AF0808014AFFF7E9BF00BFB11C080801
:104B90000B79092B4FF6FF7370B508BF858A044661
:104BA00018BFC58A9D4202D1064AFFF7D7FF218B65
:104BB000628BA36A8A1A606A29465B6FBDE87040FF
:104BC000184700BFBE1C080838B5054679B101F08A
:104BD0000F03022B0DD10C09204609F0C5FD00285A
:104BE00006DA2246054906480CF08AFB6860002078
:104BF00038BD044AFFF7B2FFF9E700BFD71C080829
:104C000074AF0808DC1C080870B5144605460E464B
:104C1000127883B132B1032A04D0104ABDE8704043
:104C2000FFF79CBF032661682670286AFFF789FD9D
:104C300000B1067070BD62B9012321462370006A7D
:104C4000FFF786FD2378012BF4D1054A314628462B
:104C5000E4E7062AEED0034AE0E700BFEC1C0808B0
:104C6000F91C0808061D08082DE9F341437804469D
:104C70000D46012B1AD10B79102B0CBF4FF00108F8
:104C80004FF0000808D0036A1B782BB9114A02B014
:104C9000BDE8F041FFF762BF01AA6D2105F10800F0
:104CA0000026FFF7F5FA0746B74202D102B0BDE889
:104CB000F081019B0022206A53F826100136090971
:104CC000FFF71EFD4346024629462046FFF79CFF9C
:104CD000EAE700BF0D1D080842780B46012A02D101
:104CE000006A02F00FBE816A026A2031406A02F057
:104CF00018BE42780B46012A02D1006AFFF700BDB8
:104D0000816A026A1031406A02F00BBE70B5054636
:104D10000C4600292DD0CA0706D5836A49105B6B63
:104D2000686ABDE8704018478B0716D004F00F047E
:104D30000909022C0AD0062C0CD0052919D0836A47
:104D4000C9B2406A1B6BBDE870401847BDE87040AF
:104D5000FFF7CFBF836A9B6BE2E7836A0968DB6872
:104D6000406A98472279034B2146284653F822305F
:104D7000D7E770BD38A508082DE9F74F05460C4662
:104D800016461F462046FFF74BF840B16EB9AB6A96
:104D900039469B6E686A03B0BDE8F04F184720465D
:104DA000FFF741F820B1002EF1D103B0BDE8F08F3C
:104DB000002C48D0A30746D163684FEA132BDBB21F
:104DC0001E2B18D1DEB1043404EB8B0B5C45ECD008
:104DD0003B46324654F8041F2846FFF7CDFFF5E75F
:104DE00043465AF8041F2846019209F10109FFF7CA
:104DF000C3FF019A11E01F2B1FD1002EE3D0D5F87D
:104E00000C8004F1040A4FF0000986F0010208F159
:104E10000103EB600BF1FF330093009B4B45DFDC9C
:104E20000BF101013B463246284654F82110FFF7AA
:104E3000A3FFAB6A41469B6AACE7202B03D1A46871
:104E400086F001069EE721462846FFF75FFFAB6A22
:104E50003A463146DB6E686A03B0BDE8F04F18474A
:104E6000026A38B5127804460B46072A06D0022A91
:104E700004D0154ABDE83840FFF770BE9D6885B97B
:104E8000A36A0F21606A1B6B9847A36A0021606ABE
:104E9000D3F8CC30984720460121BDE83840FFF7D1
:104EA0007DBCAB070BD12B79AF2B08D12046A9686D
:104EB000FFF72CFF2046BDE83840FFF7F7BC294636
:104EC0002046FFF723FFE0E71F1D080870B5437871
:104ED00004461546CE68012B06D1036A0A462946C8
:104EE0001B8BFFF71CFD70610023716920461A4679
:104EF000FFF77CFCF1682046FFF708FF062D05D17F
:104F0000A36A0021606AD3F888309847A36A012118
:104F1000606AD3F8BC500023AC461A46BDE8704026
:104F2000604738B505460C46C968FFF7EFFEA16833
:104F30002846BDE83840FFF7E9BE0B79342B70B541
:104F400004460D4610D18968FFF7E0FEED68AD68B4
:104F500085B9A36A0F21606A1B6B9847A36A042274
:104F60000221D3F8A0301AE0836A0F21406A1B6B3C
:104F70009847ECE7AB071FD12B799A2B13D1A36A83
:104F80000F21606A1B6B9847A9680029E6D020466C
:104F9000FFF7BCFEA36A04220321D3F8A030606AA5
:104FA000BDE8704018479B2B06D1A9682046FFF743
:104FB000ADFEEB689968E8E729462046FFF7A6FEB4
:104FC000CCE710B504468968FFF7A0FE0021A36A6C
:104FD000606ADB6CBDE81040184700002DE9F7431C
:104FE0008D68044616465DB9002A75D0836A022290
:104FF0002946D3F8A030606A03B0BDE8F0431847F3
:1050000015F0030740F08A802B79372B13D132B18A
:10501000836A02220121406AD3F8A03098472046D3
:105020002946FFF773FEA36A606AD3F8A43003B081
:10503000BDE8F04318479F2B70D1EB681A79A12A7D
:105040005AD1A22101AA03F10800FFF721F9A968AA
:10505000804621B38B0722D10B79372B1FD136B174
:10506000A36A411C0222606AD3F8A0309847A9685D
:105070002046FFF74BFEA36A4FF00109606AD3F8A0
:10508000A4309847474510D1B9F1000F24D1A36A45
:105090000322791C606AD3F8A03098471CE02046B0
:1050A0004FF00009FFF732FEECE7019B53F82710A1
:1050B000A9B18E0713D10E79A6F1370046424641B9
:1050C0002046FFF723FEB9F1000F11D04EB9184A60
:1050D00029462046FFF742FD03B0BDE8F0830026D5
:1050E000EEE7A36A606AD3F8A43098470137C9E7AE
:1050F000002EFBD00F4AEBE7AB685BB19A0709D1F2
:105100001B79372B06D10422294603B0BDE8F043B2
:10511000FFF7DCBE052229462046F6E72946204651
:10512000FFF7F4FDA36A03220121D3F8A03062E760
:105130002A1D08083B1D08080122FFF74FBF70B564
:105140000D46C9680446FFF7E1FDA968A36AC1F3EB
:105150000711606AD3F89830332916BF3F3902210E
:10516000C9B2BDE870401847F8B54F680C46002634
:1051700089683F0A0C340546FFF7C8FD023608343B
:10518000B74200DCF8BD54F8041C2846FFF7BEFD0A
:1051900054F8081CAB6A0909686AD3F89C302439B2
:1051A000C9B29847EAE72DE9F0414E680C4601275D
:1051B0000546A6F10D08360A54F8081F5FFA88F86C
:1051C000FFF7A4FDB74201DBBDE8F08154F8041FEE
:1051D0002846FFF79BFDAB6A4146686AD3F89C30CE
:1051E00001379847EEE72DE9F0414E680D46896892
:1051F0000446360A0127FFF789FD032E89BFD4F83C
:105200000C804FF0000808F10103E3607B1C9E4214
:1052100022DC032E55D9E568606A6B1C2946E360E1
:10522000A36A9B6E9847A36A4146606A9B6A984747
:10523000A36A0121606A9B689847A36A606A1B6E33
:105240009847A36A606ADB6D9847A36A2946606A3B
:105250009B6ABDE8F0411847023729692046FFF7ED
:1052600055FDB74207DAA36A606A5B6D9847A36A87
:10527000606A5B6E9847EB68A26A03F00F01606A90
:10528000D2F89C200A2911D1C3F30713252B16BF8E
:10529000343B0621D9B29047B74205DAA36A4246A9
:1052A0000021606A1B6F98470835AFE71979852997
:1052B00001D13221EFE79B680BB90721EBE73321DE
:1052C000E9E7BDE8F08110B504468968FFF71EFDE7
:1052D0000321A36A606AD3F89830BDE810401847EC
:1052E0002DE9F0470D46D0F80C800446002755F80C
:1052F000046F5FFA86F9360AA9F11E03D3F100099B
:1053000049EB030908F10103C360B74206DBA36A56
:105310004146606A9B6ABDE8F0471847013755F877
:10532000041F2046FFF7F2FCB742F0DAA36A4246B8
:105330004946606A1B6F9847E7E7000001F00F03DA
:10534000022B70B5044612D00B79492B09D0483B8B
:10535000082B18D8DFE803F00817071717171705E9
:1053600007000123A37070BD8E680D6975B9A3781D
:10537000002BF8D1638A002BF5D020461D4ABDE8EA
:105380007040FFF7EBBBD1E90265EFE7A3783BB3D1
:10539000238A01339BB2012B23820ED1618AD4E987
:1053A0000903D1B1D3F8A03000229847A36A0222A2
:1053B0000021606AD3F8A030984729462046FFF7BD
:1053C000A5FCA36A606A31099B6B9847A36A606A6F
:1053D000D3F8A430BDE8704018471B6C9847E5E748
:1053E000638A2946204601336382BDE87040FFF797
:1053F0008DBC00BF481D08082DE9F041C568044672
:10540000D1F80C800E46AB1C0022D8F808106F1C97
:10541000C3602B46FFF7B0FCB1682046FFF776FC6F
:10542000A36A3946606A9B6E9847A36A2946606AF8
:105430009B6A9847A36A606A4FF0FF319B68984760
:10544000D8F80C102046FFF761FCA36A3946606A61
:105450009B6ABDE8F04118472DE9F047C66804464D
:10546000D0F814A00D46B31C06F10108B0F81A904C
:10547000C360038B8682A0F8168043838868FEF79A
:10548000CFFCF8B9E768A8687B1CE360FEF7CBFCAB
:1054900020B9A36A4146606A9B6E9847A36A394661
:1054A000606A9B6A9847E9682046FFF72FFCA36A69
:1054B0004146606A9B6A98473B460122A96820469C
:1054C000FFF75AFC29692046C4F814A0A4F81A90E2
:1054D000FFF71CFCA36A3146606A9B6ABDE8F0478F
:1054E00018472DE9F347C66804460D46731CC36090
:1054F0008868FEF795FC0246E8B9E7682046A96887
:105500007B1CE3603B46FFF737FC2046E968FFF76A
:10551000FDFBA868FEF787FCD8B92B690BB96B694E
:1055200023B1A36A3146606A9B6E9847A36A3946E5
:10553000606A9B6A984701AA712105F11000002753
:10554000FEF7A6FE81464F450BD169692046FFF75D
:10555000DDFBA36A3146606A9B6A984702B0BDE8EA
:10556000F087019B53F82780D8F80800FEF758FC15
:10557000024600BBD4F80CA02046D8F808100AF167
:105580000103E3605346FFF7F7FBD8F80C10204601
:10559000FFF7BCFBD8F80800FEF745FCD4E9092367
:1055A0000028D6D19B6E314610469847A36A5146D3
:1055B000606A9B6A98470137C5E70000184B2DE9E0
:1055C000F041D3F8307204460D463FBBC668012255
:1055D0008968731CC3603346FFF7CEFBA36A1F21A3
:1055E00001225B69606A9847E96851B12046FFF77C
:1055F0008DFBA36A3A460121D3F8BC503B46606A52
:10560000A847A36A0121606AD3F8C8309847A36A03
:105610003146606A9B6ABDE8F0411847BDE8F081F9
:105620000040022070B58D6804463DB9836A294662
:10563000D3F8C830606ABDE870401847AB070ED198
:105640002B795E2B0BD1A968FFF760FBE968204638
:10565000FFF75CFBA36A0221D3F8C830EAE72946CA
:105660002046FFF753FBA36A0121D3F8C830E1E7D6
:1056700010B504468968FFF749FBA36A606ADB6DD1
:10568000BDE8104018470000026A2DE9F041127889
:105690000446072A04D01B4ABDE8F041FFF75EBA72
:1056A0008D685DB9836A0F21406A1B6B9847A36AB6
:1056B000606AD3F8C430BDE8F041184715F0030222
:1056C0001DD12B791B2B1AD1C668EF68731CB968E2
:1056D000C3603346FFF750FBA9682046FFF716FB6F
:1056E000A36A606AD3F8C4309847A36A3146606AF7
:1056F0009B6A9847F9682046FFF708FBD7E72946D9
:10570000F9E700BF661D08082DE9F0410C46054683
:1057100054F8046F360A04EB8607BC4208D1AB6A22
:105720003146686A0022D3F8A030BDE8F04118473E
:1057300054F8041F2846FFF7E9FAEEE789680346A4
:1057400010B441B9826A406AD2F8A0400A462346A2
:105750005DF8044B18474A68120A022A0BD1CA683E
:105760004AB1940707D11279AC2A04D106225DF818
:10577000044BFFF7ABBB18465DF8044BFFF7C4BF03
:105780002DE9F0410E4605460F46002456F8043F29
:105790004FEA1328444501DBBDE8F08156F8041FA9
:1057A0002846FFF7B3FA6B683BB10234284657F836
:1057B0002410BDE8F041FFF745B90134EAE710B520
:1057C0000446FFF7DDFF2221A36A606AD3F89C300C
:1057D000BDE81040184770B58D68044645B9836A26
:1057E00001222946D3F8A030606ABDE8704018470E
:1057F000A9071ED16B68DAB2922A1AD11B0A022BB2
:105800000CD1EB6853B19A0708D11B79AC2B05D1A9
:1058100029460322BDE87040FFF758BB29462046C1
:10582000FFF7AEFF6968A36A0122090AD3F8A03026
:10583000DAE729462046FFF769FAA36A0122D3F87E
:10584000A0301146D0E7000001F00F03022B2DE934
:10585000F04705460C4604D10909BDE8F047FFF7BB
:105860003BBA002955D011F0030652D10B792C2BED
:1058700038D18968FFF74AFAE668002E49D016F059
:10588000030846D177683346FAB28E2A09D13F0A17
:1058900006F1040907F1FF3AC24510DC013756F85A
:1058A00027301A79312A12D199682846FFF72EFA43
:1058B000AB6A686A0221DB6CBDE8F047184759F80B
:1058C000041F284608F10108FFF720FAE4E7322A0E
:1058D0001FD199680222AB6A686A09091B6DBDE88D
:1058E000F04718472D2B14D18C6894B163681B0ABC
:1058F000022B06D0271D6368B6EB132F10D3BDE82B
:10590000F087E368002BF5D09A07F3D11B79AC2B15
:10591000F0D121462846064ABDE8F047FFF71EB9F8
:1059200057F8041F28460136FFF78EFFE3E700BF54
:10593000721D08082DE9F8430446006A17460D4613
:10594000C68AB20706D5374A29462046BDE8F8433D
:10595000FFF704B901F00F02022A18D1A378090950
:105960008BB1838B013383834FF000094FF0010823
:10597000002954D00022FEF7C3FE03780646002B10
:1059800037D0294AE0E7438B01334383ECE70A79B8
:105990008946BA420BD18968A37809091BB1838B68
:1059A00001338383E2E7438B01334383DEE79A428B
:1059B00017D1A378002BC6D10122A270896871B3D8
:1059C00001F00F0246F004064FF00308022AC682D7
:1059D00013BF894609099946D9F8081018BF090963
:1059E000C6E7896846F002064FF005080909C68235
:1059F000BEE7042380F801800370236A1B8B032B0E
:105A00000DD1482F0BD1B9F1000F08D0D9F80C10E7
:105A10002046FFF7D9F8737843EA00137370BDE8A6
:105A2000F88300BFAD1C0808861D080849234822DA
:105A3000FFF780BF4F234E22FFF77CBF2DE9F04FC9
:105A40000E468DB00162002142700446C1601546C9
:105A50003378072B05D08B4A0DB0BDE8F04FFFF728
:105A60007DB8012A05D0036B021D2946C06A1B6858
:105A700098476378D6F80C80032B10D10BAA4621E7
:105A800008F10C00FEF704FC236B01460B9A9B689F
:105A9000E06A984763687083002B40F0BC80D8F8B8
:105AA0001010C1B101F00F03022B10D10B09752B9F
:105AB0003FD006D83E2B3ED05E2B0CD0724A2046FB
:105AC000CAE740F22F629342F8D1032304E06F4A01
:105AD0002046FFF743F8022304934FF00009D8F85B
:105AE000143009AA192108A80893FEF7D1FB0690E3
:105AF000069B994521D16378012B16D9236B049914
:105B00005B68E06A98476378042B0ED1206A052110
:105B1000049BE26A0393438B02930023CDE9003395
:105B2000D2E90232006906F0DBFF6368002B72D114
:105B300014E00023D0E70123CEE7099B4FEA890B4D
:105B400053F829100B79082B02D109F10109CFE78D
:105B5000052B06D04E4A2046FFF700F80DB0BDE8F1
:105B6000F08F8B68002BF5D09A07F3D1CA68002A12
:105B7000F0D11A792C2AEDD19E6806F00F02022A84
:105B8000E8D1D3F80CA0BAF1000FE3D01AF0030F5C
:105B9000E0D19AF80430302BDCD10AAAA4210AF112
:105BA00008003609FEF774FB40F21A5307469E427E
:105BB0001BD1012805D10A9A136803F00F03022BA9
:105BC00004D0344A099B53F80B10C4E7E168012D57
:105BD00001F10103E3601AD01268236B1209E06A35
:105BE000DB68984798B92C4AECE740F235439E426F
:105BF00015D1012803D10A9B1968CB0701D4274A84
:105C0000E0E7012D03D04910E06A02F0BBFB6368B6
:105C1000002B9AD0D046D8F80030A3609EE740F21F
:105C200085439E4223D1012804D90A9B1A6812F0A9
:105C3000010601D11A4AC5E7012DE8D05310079398
:105C40000A9A0BA952F82600FEF7D6F808B9154AA9
:105C5000B8E7E36A01360B9805930CF090FD0799BD
:105C60000246059802F095FBB742E9D1CFE7012D36
:105C7000CDD0236B02463146E06AD3F810B00A9BC0
:105C8000D847C4E7901D0808A61D0808AA1D0808E3
:105C9000BB1D0808C91D0808D51D0808DD1D08081A
:105CA000E91D0808FB1D080842780B46012A02D1AD
:105CB000006A01F027BE816A026A1831406A01F069
:105CC00030BE00002DE9F14F8F0704460D46164601
:105CD00012D001F00F03022B17D102F0FD060909C3
:105CE000012E04D001B0BDE8F04FFFF7DDBF01B0D9
:105CF000BDE8F04FFEF7FDBF4968CBB22D2B7FD03A
:105D00000BD8062B0ED02C2B13D0514A29462046F7
:105D100001B0BDE8F04FFEF721BF2E2B00F08480CC
:105D20009D2BF2D1002EF0D105F10802090A204680
:105D30007FE0022A02D0A968FEF7E8FFEF68002F93
:105D4000E3D017F00309E0D17B68B846DAB28E2AB7
:105D50000DD1022E4FEA132805D007F1040A08F1ED
:105D6000FF3BD94515DB08F1010857F8288098F862
:105D70000430312B27D1022E13D1A36A606A5B6EE7
:105D80009847A36A0121DB6C606A01B0BDE8F04F5F
:105D900018475AF8041F204609F10109FEF7B6FF1B
:105DA000DFE72046D8F80810FEF7B0FF012ED4E94F
:105DB000090305D19B6D9847A36A0021DB6CE3E7DB
:105DC000DB6C0121E1E7322B9FD1012ED4E90903DD
:105DD0000CD15B6D9847A36AD8F8081000221B6DA0
:105DE0000909606A01B0BDE8F04F1847022E01D1E1
:105DF0001B6E9847A36A0122D8F808101B6DEFE7C5
:105E0000AA68002A81D0002E7FF47FAF5168090A6A
:105E1000022907D1D3682BB1980703D11B79AC2B8A
:105E20003FF473AF083282E7002A7FF46EAFA968AF
:105E300021B901B0BDE8F04F00F072B88E0703D170
:105E40000B790A46922BE1D005F1080201216EE799
:105E5000061E08082DE9F047C7681E4604460D4691
:105E6000BB1C3946904607F10109C360836A406A4A
:105E70009B6A9847A36A4946606AD3F88C30984772
:105E8000A96800222046FFF71DFF2D6965BB41462A
:105E90002046FEF73BFF236A19780629D4E9090357
:105EA0001CD1D3F8CC302946984720460121FEF773
:105EB00075FCA36A606ADB6D9847A36A3946606A1D
:105EC0009B6E9847A36A606A49469B6A9847A36A93
:105ED000606AD3F89030BDE8F0471847B200D3F8B5
:105EE000A83005329847E8E72B79AD2B07D1A96890
:105EF0003B4600222046FEF73FFFED68C6E7E96813
:105F00002046FEF703FFA36A606A0121D3F88830B8
:105F10009847731C424629462046FFF79BFFCCE773
:105F20002DE9F84304460D46904601F1FF3900265D
:105F30004FF0FF37B9F1FF3F0CD17B1C05D1A36AAD
:105F40002946606AD3F8AC3098470026AE421DD18E
:105F5000BDE8F88358F8261071B18A070CD10B7987
:105F6000222B09D101370BD1A36A37464A46314665
:105F7000D3F8B030606A9847013609F1FF39D9E7A4
:105F80002046084ABDE8F843FEF7E8BD58F8261059
:105F9000B7424FF00002204608BF89680136FFF77C
:105FA00091FED3E71A1E08082DE9F04704469046F3
:105FB00099460F4621B91946BDE8F047FEF7A6BE3F
:105FC000C668731CC360156835B315F0030A23D186
:105FD0002B797B2B20D1A968FEF798FE52463146DB
:105FE0002046FEF7E3FB5246E9682046FFF76AFECB
:105FF0004B4608F10402791E2046FFF7D5FFA36A3D
:106000003146606ADB6F984720460321FEF7C6FBE6
:10601000BDE8F047FEF7DABB29462046FEF776FEDC
:10602000204600223146FEF7C1FBA36A606ADB6DA1
:106030009847DDE737B50C46054601AA7A2104F1F9
:106040000800FEF725F9E3680146019A2846FFF7A4
:10605000ABFF03B030BD8B6803F00F03022B2DE9BB
:10606000F04F044689B00D4640F00181CB68002B0B
:1060700000F0FD80980740F0FA801A792C2A40F051
:10608000F6809A6802F00F01022940F0F0801209B0
:106090007C2A40F0EC80DB681A79302A40F0E780F7
:1060A0009B6807AAA42106A80693FEF7F1F8431EF1
:1060B000022B00F2DC80079B01281A6800F0CA80DE
:1060C000022800F0C5809E68F10740F1D080710879
:1060D00000F0CD80D3F8049032B1930704D1117948
:1060E000A639022940F2C380B9F1000F08D019F097
:1060F000030F05D199F80410A639022940F2B780A0
:10610000AB6819F001086F6901932B69218B029329
:106110006369E5680493638B05F1010B618305F105
:106120000401039305F1020305F1030AA582059317
:10613000A4F816B0E16005D1494620460592FEF765
:10614000E5FD059A11462046FEF7E0FDA26A51469C
:10615000606A926E9047A26AA91C606A926A904730
:10616000A26A606A526D9047002201992046FFF7AB
:10617000A9FD02992046FEF7C9FDA26A5946606A48
:10618000926A904731462046FEF7C0FDA26A0E2172
:10619000606AD2F89C209047A26A606A5146926A6F
:1061A0009047D4E90902B8F1000F57D1936D984791
:1061B000A36A606A1B6E9847002EA36A606AACBF30
:1061C00000210121D3F89C309847A36AAA1C012121
:1061D000DB6E606A9847049B6361039B6383002FB7
:1061E00043D0A36A606ADB6D9847B8F1000F03D112
:1061F000A36A606ADB6D984739462046FEF786FD44
:10620000E668606A731C3146E360A36A9B6E984738
:1062100088F00101A36A0131606A9B689847A36A0C
:106220002946606A9B6A9847A36A606ADB6D984753
:10623000B8F1000F03D1A36A606ADB6D984727B1FC
:10624000A36A3146606A9B6A984709B0BDE8F08F3F
:1062500003263FE791460326024645E7526D9047E5
:1062600049462046FEF752FDA6E73E46D7E7E668D8
:106270002046238BB4F81A90771C63836FEA464359
:10628000D4F814A006F102086FEA5343E968E782E4
:10629000A382F31CE360FEF739FDA36A606A012163
:1062A000D3F888309847A36A3946606A9B6A984752
:1062B000A36A4146606AD3F88C3098470022A968E7
:1062C0002046FFF7FFFC29692046FEF71FFDA36A61
:1062D0003946606A9B6E9847A36A4146606A9B6A2A
:1062E0009847A36A606AD3F8903098476969204656
:1062F000C4F814A0A4F81A90FEF708FDA36A31466A
:10630000606A9B6A09B0BDE8F04F18472DE9F74F66
:106310000446174698460E4629B9194603B0BDE80B
:10632000F04FFEF7F3BCC5682B1D05F1010A05F11E
:10633000020B05F10309C3601368002B00F0D28043
:1063400013F0030240F0CE8019797B2940F0CA8017
:10635000996801920093FEF7D9FCA16A606A496DC1
:10636000884740F20B412046FEF7B9FA2046DDE9A6
:106370000032D968FFF7A6FC022229462046FEF724
:1063800015FAA36A606A03219B6898473A1D434641
:10639000711E2046FFF7BAFFA36A606A6FF0020120
:1063A0009B689847A36A2A465146D3F880605B46AB
:1063B000606AB047A36A606A5B6D9847A36A606AC7
:1063C0005B6E9847A36A606A1B6E9847A36A0022B7
:1063D00040F20C41606A5B6C9847A36A606A5B6E2E
:1063E0009847A36A606A5B6E9847A36A606A5B6DB0
:1063F0009847A36A00220A21606A1B6D9847A36A26
:10640000606A1B6E9847A36A606A0F211B6B9847EE
:10641000A36A0321606AD3F8C05000231A46A84734
:106420002046FEF743FAA36A4A460021606ADB6E03
:106430009847A36A606ADB6D9847A36A606A0F2178
:106440001B6B9847A36A4946606A9B6E9847A36A8C
:10645000606A02219B689847A36A5946606A9B6AF2
:106460009847A36A606A5B6E9847A36A606A5B6E2E
:106470009847A36A5146606A9B6A9847A36A0022BC
:10648000606A5B6C40F20C419847A36A0F21606A16
:106490001B6B9847A36A606A5B6D9847A36A606A42
:1064A0005B6D9847A36A0321606AD3F8C05000234C
:1064B0001A46A8472046FEF7F9F9A36A606ADB6D21
:1064C0009847A36A606A4FF0FF319B689847A36AB8
:1064D000606A49469B6A9847204603B0BDE8F04F82
:1064E000FEF774B919462046FEF710FCA36A606AED
:1064F0005B6D9847204640F20B41FEF7F0F9A36A26
:10650000606ADB6D984737E72DE9F041CD680446B6
:106510000E4665BB0378C3B1036A1D78ADB940F27E
:106520001941FEF7E6FBB1682046FEF7EFFBA36AD0
:106530002A460121D3F8BC602B46606AB047A36AA3
:10654000606ADB6DBDE8F0411847B1688B0707D082
:1065500001F00F03022B08D12046FEF7D7FBEEE730
:106560000029F9D00B793A2BF6D1BDE8F081AF07BD
:1065700040F0AF806B68DAB25B2A11D1ED68002D74
:106580004AD1006A0378072BEFD1896801F00F0325
:10659000022BEAD10422BDE8F041D140FEF7B0B8A9
:1065A000562A13D101228968FFF78CFBE96820463F
:1065B000FEF7ACFBA968A36A0909606AD3F89C30AE
:1065C0003E39C9B298470222B1687DE0572A25D1E9
:1065D0001B0A5F1E013355F82310FEF797FB002FAF
:1065E00003DDA36A606A5B6D9847B16804350026D5
:1065F00000222046FFF766FBBE42B6DA0136BE42F5
:1066000003DAA36A606A5B6D9847002255F8041F9D
:106610002046FFF757FBEFE7A9075AD16B68DAB2BC
:10662000062A56D1B768002F53D0BA0751D17A68DD
:10663000D1B206294DD11B0A4FEA1228B3EB122F13
:1066400047D1A8F10203012B43D8BB6823B19807B7
:1066500002D11B79222B3CD0FB6823B1990702D1D0
:106660001B79222B35D0B8F1020F06D03B6923B13C
:106670009A0702D11B79222B2BD0A9682046FEF75E
:1066800045FBE9682046FEF741FBB8F1030F07D14F
:1066900020462969FEF73AFBA36A606A5B6E984759
:1066A000A36A606A1B6E98470022B9682046FFF70C
:1066B00009FB0022F9682046FFF704FBB8F1030F3D
:1066C0007FF453AF002239692046BDE8F041FFF75F
:1066D000F9BA29462046FEF719FB002274E70000AC
:1066E0000023032A2DE9F04104460D461646427068
:1066F0000162C36080F8342002D1C08E50BBA06319
:106700004FF00008A36A3146606A1B682A46A4F865
:106710003680984706212046FEF740F86778EE68F5
:10672000012F04BFA5F82280A5F82480B6B1B207D6
:1067300014D133793F2B11D1B168FEF7E7FAA36A80
:10674000606AD3F8C4309847A36A606A5B68BDE8A2
:10675000F04118478000F9F7ACFDD0E72B78072B04
:1067600000F29380DFE803F0049125414141410E9E
:1067700031462046FEF7CAFAA36A0F21606A1B6BF6
:106780009847DCE7012F12D1002346222046A37050
:10679000564BF168FEF75FF92B8B032B07D131695C
:1067A0002046FEF711FAEB8A43EA8013EB82716907
:1067B000DFE7A36A3168DB68606A98476378012B7A
:1067C00007D100234C222046A370494BB168FEF745
:1067D00042F9F1682046FEF799FAEB8ADB07AED55D
:1067E000A36A606ADB6D9847C6E7012FD6F80C8074
:1067F00005D104223946206AFDF782FF6F83A36A20
:106800003168DB68606A98472B78032B24D1A36A30
:106810000122D3F8A0300021606A98472B78062B1C
:1068200028D1A36A606A1B6C984701212046FEF7B5
:1068300060FAA36A606A1B6C9847A36A606A1B6C63
:1068400098470023B26841462046FFF703FB2B78A8
:10685000062B7FF474AF8FE7042B04D1A36A0222C6
:10686000D3F8A030D7E7052BD8D1A36A0322D3F8F9
:10687000A030D0E720460121FEF73BFAA36A0121B0
:10688000606AD3F888309847DBE7012F04D10422EF
:106890000A212846FDF734FF17212046FEF729FA82
:1068A00016212046FFF700FAB168A36A0909606A59
:1068B0009B6B98471A212046FFF7F6F9316920466D
:1068C000FEF724FA0A212846FDF70AFF024611784E
:1068D0000429D4E9090302D11B6B0F2150E71D697C
:1068E0000A2100235288A84729E700BF2D5A020831
:1068F000355A0208036A10B504461A8BFEF709F9E7
:1069000001462046BDE81040FFF7CEB92DE9F04F13
:106910008D6885B004462B79032B0AD12946FFF7F1
:10692000E9FFAA69D38A43F00103D38205B0BDE829
:10693000F08F026AD28AD20706D4624A294605B08D
:10694000BDE8F04FFEF70AB9162B40F0AD80C668DF
:10695000E968331D06F1010B06F1020906F1030A8D
:10696000C360FEF7D3F9A36A606A00225B6C40F251
:106970000D419847A36A606AD3F8C07000231A4695
:106980001946B8476369E7680093638B07F101080C
:10699000606A0193BB1C4146A782E360238BA4F885
:1069A00016806383A36A9B6A984701225946204652
:1069B000FDF7FCFEA36A606A5B6D9847204640F2D3
:1069C0000F41FDF78CFFA96820460022FFF77AF9F6
:1069D000A36A00224946606AD3F894309847A36AB4
:1069E0005946606A9B6A9847A36A606AD3F8D030B8
:1069F0009847A36A606A5B6D9847A36A0122606A40
:106A00005B6940F293319847A36A606A0821D3F822
:106A10009C309847A36A52460021606ADB6E984713
:106A2000A36A606ADB6D9847A36A01223146606AF7
:106A3000D3F894309847A36A5146606A9B6A984796
:106A4000A36A0121606A9B6898472046FDF7BEFE55
:106A5000A36A606AD3F8D4309847A36A4946606A4B
:106A60009B6A984729692046FEF750F9A36A414678
:106A7000606A9B6E9847009B3146606A6361019B28
:106A80006383A36A9B6A984769692046FEF73EF9CB
:106A9000A36A606A39469B6A9847A36A606ADB6D9D
:106AA00005B0BDE8F04F184703AA7A2105F10800A8
:106AB000FDF7EEFBEB680146039A2046FFF726FC44
:106AC00034E700BF211E08082DE9F04F85B0C568E6
:106AD0001E4604460E9B0F469346294603936B1CA5
:106AE00001220293AB1CC360FDF760FE39462046CD
:106AF0000027FEF70BF9A36A0022691CD3F8943033
:106B0000606A9847A36A2946606A9B6A9847A36AA5
:106B1000606AD3F8D0309847D4F80C9009F101039B
:106B2000E3605F4518DB2046FDF750FEA36A606A0C
:106B3000D3F8D4309847A36A02999B6A606A984751
:106B400003992046FEF7E2F8A36A4946606A9B6A09
:106B500005B0BDE8F04F18473346D4F80CA0043612
:106B600001371A6801920AF10102E260019AD2F833
:106B70000880B8F1000F4FD1BB4542D10025A36A70
:106B8000606AA846DB6D9847019B2046D968FEF7EE
:106B9000BDF825B3A36A0F21606A1B6B9847A36AEF
:106BA0004146606A9B6A9847A36A0121606A9B68B4
:106BB0009847A36A0F21606A1B6B984729462046B5
:106BC000FFF772F829462046FEF786F8A36A606A46
:106BD0004FF0FF319B6898472046FDF7F7FDA36A09
:106BE00001224946606AD3F894309847A36A514617
:106BF000606A9B6A9847A36A0121606A9B6898470C
:106C00008FE720461E4A1968FDF7A8FF204605B009
:106C1000BDE8F04FFDF7DABD18F003052DD198F867
:106C200004204346762A03D1DD68D8F808802D0970
:106C3000A36A606A5B6D984741462046FEF766F896
:106C4000A36A0821606AD3F89C309847A36A524629
:106C50000021DB6E606A9847002D8FD029462046C0
:106C6000FFF722F8D4F80C800222204608F1010335
:106C70004146E360FDF79AFD86E70025D8E700BFAF
:106C8000381E08082DE9F347C768984616460D4692
:106C90007B1C022239460446C360DDE90AA9FDF7E0
:106CA00085FD002E2DD1A36A0321606A9B68984759
:106CB00029462046FEF72AF8A36A6FF00201606AAF
:106CC0009B689847A36A0F21606A1B6B9847A36A69
:106CD0003946606A9B6A9847A36A606A01219B688B
:106CE000984749462046FEF711F8A36A606A4FF0BC
:106CF000FF319B689847204602B0BDE8F047FDF79A
:106D000065BD4346324629462046CDF800A0FFF730
:106D1000DBFED7E7F0B5CE6885B005460C46337983
:106D2000782B09D1B3680193002300931A46896830
:106D3000FFF7A8FF05B0F0BD742B03AA4FF0770151
:106D400013D106F10800FDF7A3FA37690246A168DE
:106D5000039BF06827B900902846FFF7B5FEE9E7E6
:106D6000BC68CDE900042846E2E704F10C00FDF719
:106D70008FFA002302460093039BA168ECE7000012
:106D800001F00F03022B70B504460D46164602D0E3
:106D90001E4AFDF7E3FE31462046FDF7B7FFA36A22
:106DA000606A2E095B6D98476378012B10D1226AC7
:106DB0001378033B032B0BD85068314600F0A2FD3B
:106DC0000346206A1A78032A08D13146FDF798FC59
:106DD00031462046BDE87040FEF766BF00223146CE
:106DE000FDF78EFC236A02465B685B68002B0CBFD4
:106DF0000123002304D00178012904BF0021017080
:106E000029462046FDF700FFE2E700BF061E0808FE
:106E10002DE9F04F002687B04FF0010B0446B14634
:106E20003746B04603A81D46CDE9022105AAA42194
:106E3000FDF72EFA0190019B9E4211D127B1A36A62
:106E40004946606A5B6B9847029AD4E90903002AB5
:106E500076D0D3F8C0403B4642462946A04713E0CF
:106E6000059B53F826A0BAF1000F5BD01AF0030F70
:106E700058D19AF80420A62A1AD1B80707D5324A61
:106E800051462046FDF76AFE07B0BDE8F08F1D2E83
:106E900001D92E4AF4E70BFA06F201350127DAF898
:106EA0000810204649EA0209FDF730FF0136C2E723
:106EB000A72A0DD1A26A47F00207606A126C9047B8
:106EC000DAF80810204608F10108FDF71FFFEDE78A
:106ED000A82A27D1DAF80C2072B191070CD11179C8
:106EE000AA2907D192682046DAF80810FFF748FF70
:106EF0000135DBE7AC290FD0DAF8081001F00F02FA
:106F0000022A01D0124ABBE7A26A0909606A926BA1
:106F10009047DAF80C10D5E7062251462046FDF7D7
:106F2000D5FFE5E7BB0701D50A4AA9E7B8F1000F8D
:106F300001D0094AA4E751462046FDF7E7FED7E70E
:106F4000D3F8BC4087E700BF501E0808571E08084A
:106F50005F1E08086C1E0808731E080870B50D46F1
:106F6000417804461346012903D12A46FDF7D7FC90
:106F70006861A36A606A9B6C98476E69002320462B
:106F800031461A46FDF732FCA36AB18A9B6B606AF0
:106F90009847E96829B18B0703D10B79A32B08BF68
:106FA0000021204602230022FFF732FFB08A70BD85
:106FB000002389681A46FFF72BBF00002DE9F8432C
:106FC0000C4689680546FDF7A1FEE668002E56D0FE
:106FD0007768296AFBB209788E2BA36819BF04F180
:106FE0000C0601273F0A0836072903F00F024AD191
:106FF000022A46D11A099A2A47D133681A79302AC7
:107000003FD19B68002B3CD10A212846FDF771FE39
:107010002A6AD36A128D32B9316828463F4ABDE8E0
:10702000F843FDF79BBD5978C9070FD55968284625
:10703000FDF75FFE022FD5E909030AD8D3F8BC405B
:10704000002302211A46A047012416E0013A083322
:10705000E1E7726811793229F0D1B46821793029D9
:10706000ECD1916801225B6C09099847A16803245F
:10707000002301222846FFF7CBFEA74226D8BDE811
:10708000F8830024F9E7022AFBD140F2D622B2EBC2
:10709000131FF6D133681A79302AF2D19B68002B7E
:1070A000EFD013F00304ECD11B792F2BE5D1AB6AA1
:1070B00022462146686AD3F8BC802346C04733681D
:1070C000224628469968FDF789FFBDE704F10108CB
:1070D000A30056F82410B8451AD20A79322A17D1DB
:1070E0003344D3F8049099F80430302B10D18968D8
:1070F0000022AB6A0909686A5B6C98470023012289
:10710000D9F808102846FFF783FE08F10104B4E718
:107110002846A046FDF7FAFDF7E700BF7A1E0808EB
:10712000026A0B4610B512780446072A06D0022AD6
:1071300004D0074ABDE81040FDF710BD20461946AF
:10714000FFF73CFF2046BDE81040FDF7AFBB00BF96
:107150008D1E0808D1E90212FFF712BE036A10B5AE
:1071600004461A8BFFF7FAFE01462046BDE81040A0
:10717000FEF79ABD2DE9F04F884685B004464221BE
:1071800002AA08F10800FDF783F80027236A834666
:10719000BA461E8B5F450AD1D8F80C100B79032B29
:1071A00051D132462046FDF7B4FC054659E0029B1A
:1071B00003AA6C2153F8273003F108000193FDF76F
:1071C00067F8039B054619680A09732A0DD04FF02A
:1071D00001092046FDF79AFDA94528D3019BD968EE
:1071E00069B12046FDF792FD09E0022809D0354635
:1071F000294A2046FDF7B2FC0AF1010A2E46013762
:10720000C8E759680B09412B0DD040F261529342F7
:10721000F2D040F24662934207D040F23F4293429E
:10722000E5D10425E8E70125E6E70325E4E7039B2C
:107230000022606A53F8291009F10109A36A0909BB
:107240001B6D9847C8E7442B17D18F6832462046FC
:107250003946FDF75EFCBA690546D38A43F001035F
:10726000D3820027ABEB0A0ABA450BD82946204641
:10727000FEF71AFD05B0BDE8F08F32462046FFF755
:107280006DFE92E7A36A0121606A0137D3F8BC6002
:1072900000231A46B047E7E7981E08082DE9F34196
:1072A0008D6804460E4605F00F030A2B07D0002D0B
:1072B00031D015F003012ED12B79652B1ED100950D
:1072C000002501AA65216846FCF7E2FF019B002129
:1072D00040F2CA5203EB8000834215D1F26840F2BB
:1072E0001A439A4237D1236A1F78B7B13B4A3146D5
:1072F000204602B0BDE8F041FDF730BC622BEDD175
:10730000AB680093ED68DCE753F8047B97420CBF51
:1073100001310331E0E70021E0E7A36A606A5B6BBB
:107320009847A36A606A05219B6B9847A36A3A460F
:10733000606AD3F8A0300121984701AA2946204667
:10734000FDF702FBA36A02223946DB6A606A02B0DB
:10735000BDE8F0411847A36A0027606A5B6B984755
:1073600006F10C006A466A21FCF792FF0646B74216
:10737000D4E9090313D1D3F8A0300022314698474D
:107380002946002501AA2046FDF7DEFAB542D4E9D8
:1073900009030DD1DB6D984702B0BDE8F081009A7A
:1073A0009B6B52F827200137916809099847DEE75F
:1073B000009ADB6A52F825800122D8F808703F094C
:1073C00039469847D8F80C1029B939462046013576
:1073D000FEF76AFCDAE70909F8E700BFB01E080803
:1073E000836A37B504460D465B6B0021406A9847B7
:1073F000A36A606A0F211B6B98472946204601AAA1
:10740000FDF7A2FA0199204603B0BDE83040FEF72F
:107410004BBC00002DE9F04F9BB09F4D14464FF040
:10742000000BCDE902011020F8F72AFF2B69582242
:1074300000214360064604A841F08EFE4FF0FF3362
:10744000012113A809938DF8104007F011FB039B4D
:10745000012213A8D90041F0020107F03FFB0123EC
:107460000021436016A80BF0EBFC029A95F8343229
:107470000021126804A8FDF752FA054611A800F091
:1074800023FF864B0B9F01900D900E930FB1059C2F
:107490001CB30B9C14B1059B002B3DD059460198A1
:1074A00000F019FF00270B9CDFF8F091DFF8F0A146
:1074B000DDF81480002C00F03981B8F1000F00F0E5
:1074C000F1800C9C04A8E168FDF7BCFAA38A069A37
:1074D0004046039909F060FF2CE13B8B01223946BD
:1074E00004A8042B07D1FEF7A9FA079BBF689B45A8
:1074F00038BF9B46CAE7FFF7F3F83B8D9C42F4D2B6
:10750000FB6A03EBC40113F83430012B02D1384677
:10751000FDF71EF90134F0E7E28A520716D5218DF6
:10752000013913D3E76A4FEAC10E07EBC102507865
:1075300010F0020F25D04BB1D3E9008C92E8030084
:1075400083E8030047F80E80C2F804C04FF0000340
:1075500000272384B4F828C0674518DB00239C4526
:107560004ED1D4F804E0BEF1000F08D00020BEF8E0
:1075700028A00346504553DB002B40F08A80A468C6
:1075800088E7002BCCD1012808BF1346C8E7237831
:107590004FEAC70AD4F82C80012B08EBC70905D1A4
:1075A000D9F804300A2B12D10137D3E718F8373055
:1075B0000DD9012B0BD14FF0030308F83730238B83
:1075C000032B16D0E38A43F01003E38203E018F89C
:1075D0000A30032BF3D018F80A30042B03D099F8A3
:1075E0000130DB07E0D5238C5A1C2284A9F8023035
:1075F000DAE7D9F8040007F0B7F80128EBDCE1E797
:10760000E26A02EBC30112F83320052A06D14A7858
:10761000D7075FBF228C4A800132228401339EE764
:10762000DEF82C2002EBC00912F83020053A012ABE
:1076300014D8002710E0E26A02EBC70812F83720DE
:10764000062A08D1D9F80410D8F80420914204BFC2
:10765000A8F8023001330137BC45ECD1013089E78D
:10766000E06A00EBC20110F83200062802D1487827
:10767000C00702D548881844488001329445EFD1AC
:10768000628B12FA83F26283228C12FA83F32384D0
:1076900075E70022F2E700BF0040022024A6080898
:1076A00028A70808238B042B17D10F9B1BB958461A
:1076B00004F03CFC0F9000230322214604A80D9304
:1076C000494B1093FEF7BAF9059B23B904222146D2
:1076D00004A8FEF7B3F9A468EAE6023B012B21D81F
:1076E00037B95B4607AA05A911A803F07DFD074637
:1076F000CDE90D7A0222214604A8FEF7F1FF059B91
:10770000002BE8D10322214604A8FEF7E9FF059BE0
:10771000002BE0D10422214604A8FEF7E1FF002857
:10772000F8D0D8E7019BCDE90D39E3E7B8F1000FB8
:107730007FF4C7AEDDF81490D5F81080B9F1000FD2
:1077400016D0019800F0CFFD002F41D10F9808B15D
:1077500004F001FC0298FCF789FF2846AD68FCF7AD
:10776000B5FF002DF9D10598002835D0F8F760FD58
:10777000139C1898C4F3DC046400033400EB9400F9
:1077800024F003048000F8F77BFD0444B060F4604B
:10779000DDE9144101F1040CA1450BD1189A002335
:1077A0009342CED0199951F82300F16841F8230093
:1077B0000133F5E751F839303BB1042B1FBF5CF8BA
:1077C0003920DB08521020F8123009F10109E3E7F3
:1077D000384603F02BFDB9E72A46314640461BB038
:1077E000BDE8F04F05F0B0B904A808088842F0B52C
:1077F00007460C462DED028B83B004D1012003B067
:10780000BDEC028BF0BD244B984201D10020F6E77D
:107810009942FBD007F094FB0546204607F090FB09
:107820008542F3D11D4B9D4213D17A6863689A4219
:10783000ECD13E1D043400257B68AB42DED954F800
:10784000041F56F8040FFFF7D1FF0028DED00135E2
:10785000F2E72146384607F033FE0028D6D0104B19
:107860009D42CBD1384609F0F7FEB5EE400BB0EEA5
:10787000408BF1EE10FAC1D1204609F0EDFE18EE72
:10788000900A8DED000B019B00F0004003F00043D7
:10789000C31A58425841B2E740A9080814C1080861
:1078A00034B30808C900012210B541F002010446B2
:1078B000083007F013F943683BB9A368C3F3DC034E
:1078C000013B5B0043F001034360C3F34F0010BD75
:1078D00070B505460E460024EB69A34208D8314630
:1078E00005F114000BF067F9EC69013C204670BD0E
:1078F0002B6A314653F82400FFF778FF0028F5D1B2
:107900000134E9E710B501220446FCF7F9FE0378DB
:10791000012B05D12378012B8CBF04230223037094
:1079200010BD70B505460E46104619461C46FCF7BC
:10793000D7FE03785A1E012A06D873680022214612
:107940002846BDE870401847032B02D17368012216
:10795000F5E73668042B428821462846B4460CBF1A
:1079600000230123BDE8704060474379012B07D015
:107970008368194403695A8C81609142C8BF598455
:107980007047002383714379012B1EBFC26A036ACB
:1079900043F8212070476FF00301FFF7E6BF042191
:1079A000FFF7E3BF6FF00201FFF7DFBF0346426A54
:1079B00040791144032859628ABF586B18468018D1
:1079C0007047827903460AB118467047C26A407907
:1079D0001144032801D8D962F6E7986AD9620244B3
:1079E000586B1044704710B50C460121FFF7E9FFB2
:1079F000047010BD10B51446FFF7B7FF0121FFF763
:107A0000E0FF047010BD53220121FFF7F3BF5422A1
:107A10000121FFF7EFBF57220121FFF7EBBF5822EB
:107A20000221FFF7E7BF59224FF0FF31FFF7E2BF16
:107A30005A220021FFF7DEBF5B220021FFF7DABFE9
:107A40005D224FF0FF31FFF7D5BF19B103215F224F
:107A5000FFF7D0BF5E22FBE7A1F130020021D2B2D6
:107A6000FFF7C8BF62226FF00101FFF7C3BF10B577
:107A700063224FF0FF310446FFF7BCFF0123A371DF
:107A800010BD01F16402494210B5D2B20446FFF7BD
:107A9000B1FF0123A37110BD01F16702494210B586
:107AA0000446D2B2FFF7A6FF2269D38A43F001034E
:107AB000D38210BD38B504461D46FFF79BFF03492E
:107AC0002A462046BDE8384013F0C4BEC3790208F8
:107AD00070B504460D4616461946C068FFF7E2FE2B
:107AE0003246034629462046BDE87040FFF7E2BF14
:107AF0000B4610220121FFF7EBBF11320B4601218B
:107B0000D2B2FFF7E5BF20B40B4602F114055100D5
:107B1000EAB25DF8045BC1F10101FFF7D9BF16328B
:107B20000B464FF0FF31D2B2FFF7D2BF19320B46EE
:107B30000021D2B2FFF7CCBF70B4C4681D462678CE
:107B40006388042E04BF666846F823505D1C658078
:107B500070BCFFF7AFBF03F128011346CAB2002182
:107B6000FFF7A8BF022A02F12A020B46D2B214BFC5
:107B7000C1F101010121FFF79DBF03290AD00429AA
:107B80000AD101210B460A44C94343EA82032F224A
:107B9000FFF790BF0021F5E700210223F3E70B4632
:107BA00030220139FFF786BF10B4144641EA0223A0
:107BB000312221445DF8044BFFF77CBFF8B516462F
:107BC0001F46FFF7D2FE847905460CBB4379022B92
:107BD00026D9C46A442E036AC4F1FF2453F827301F
:107BE00004F57F0404F1FE041C4412D814F1400F84
:107BF00014DB3F2CD4BF00270127E41BB91C284607
:107C0000FFF7DFFE06706FB9442E98BF4034447012
:107C1000F8BD7F2C94BF00270127EEE70127ECE792
:107C20000127EBE7442E6B7998BF04F58044042BC1
:107C300005D1B4F5004F24BF012385F8383064F036
:107C40007F03E41143708470E2E70B464222002177
:107C500010B50446FFF7B2FF0123A37110BDF8B5BC
:107C600005460C4621F400471646CAB90B040ED54A
:107C70005921FFF7B8FE59212846FFF7B4FE5921D4
:107C80002846FFF7B0FE59212846FFF7ACFE3B46D9
:107C9000422200212846FFF791FF0123AB71F8BD76
:107CA0003B4640220021FFF789FF2846210A21F0A8
:107CB0007F013143C9B2FFF796FEEEE70B46B2FAF9
:107CC00082F120B4490902F147054900EAB25DF8A2
:107CD000045BFFF773BF0B464B220121FFF76EBF1A
:107CE0000B464A22002110B50446FFF767FF012327
:107CF000A37110BD264BD3F83032022B2DE9F0478B
:107D0000044689460ED88669B1420BD9C56A8E1BD6
:107D1000436940F2FF77ED1A56EA050304D1E36A9E
:107D2000C4E90539BDE8F087062E01D90F2D1AD90F
:107D30001F2DAA4628BF4FF01F0A1F2D10D8032E53
:107D4000B04628BF4FF0030801212046FFF72EFE62
:107D50004AEA48130370A5EB0A05A6EB0806DBE721
:107D60004FF00008F0E7BE42B0464FF00201204657
:107D700028BFB846FFF71AFEAA464FEA181380F844
:107D8000018003F070032B4363F07F030370E2E78D
:107D90000040022010B5044631B955224FF0FF31A2
:107DA000BDE81040FFF726BE022904D1FFF72BFEE5
:107DB0002046FFF741FE56226FF002012046EFE712
:107DC000134621B143224FF0FF31FFF7F7BE4422A3
:107DD000F9E7134621B145224FF0FF31FFF7EEBE20
:107DE0004622F9E7322938B5044611D0332912D09A
:107DF000002529392046CAB24FF0FF31FFF7FAFDBE
:107E000065B12046D3220021BDE83840FFF7F2BD1E
:107E100001250621EDE701250721EAE738BD012A02
:107E20000B4610B4044608D0022A0ED169224FF046
:107E3000FF315DF8044BFFF7DDBD11461B322046D4
:107E40005DF8044BD2B2FFF743BE4FF0FF31F5E7C8
:107E500070B50D46044611462AB92B461322BDE8DB
:107E60007040FFF735BE022A04D1FFF7CCFD204653
:107E7000FFF7DEFD2B4618226FF001012046EEE7EA
:107E800010B4044643B90F2A06D8503A01215DF8D0
:107E9000044BD2B2FFF7AEBD03F1240120461346D6
:107EA0005DF8044BCAB20121FFF704BE10B40446CA
:107EB0004BB90F2A07D8403A4FF0FF315DF8044B19
:107EC000D2B2FFF797BD03F12601204613465DF8B5
:107ED000044BCAB24FF0FF31FFF7ECBD70B4DDE9DF
:107EE0000365D2B203EB460443EA062315B101321F
:107EF0000134D2B2091B70BCFFF7DCBD07B5CDE978
:107F000000230B4634220021FFF7E8FF03B05DF8A1
:107F100004FB07B5CDE900230B4636224FF0FF31B5
:107F2000FFF7DCFF03B05DF804FB10B50446C06842
:107F3000FFF7CEFC2322034601212046BDE8104076
:107F4000FFF7B8BD01F110033F2B73B506460C4691
:107F500008D8A1F180020121D2B202B0BDE8704080
:107F6000FFF748BD0DF1050501212222FFF742FD73
:107F7000294604F07F00E3B2E4112A4605F8010D1A
:107F8000601C0128F5D8013403F0400314D11BB95B
:107F90007F2305F8013C951E491B3046FFF711FD74
:107FA00001AC6A1E014612F8013FA24208D11044FA
:107FB000401B037002B070BD002BEDD00023E8E73A
:107FC00063F07F0301F8013BEDE770B51446D6B2CC
:107FD000049A054613430B6907BF2022C4F101012F
:107FE000E1432122FFF7A8FD31462846BDE8704055
:107FF000FFF7F9BC1A430B6907BF32220121332274
:108000004FF0FF31FFF798BD0D2910B504460BD195
:108010000949C068FFF75CFC232203460121204682
:10802000BDE81040FFF746BD4231BDE81040CAB27E
:108030000121FFF7DFBC00BFA4BC080838B5044627
:108040000D460F21FFF7E0FF20462946FFF799FC78
:1080500002215C22FFF7CEFC20466FF00301BDE851
:108060003840FFF782BCF8B504460F460F211D4685
:108070001646FFF7C9FF2046FFF7DAFC39462046CF
:10808000FFF7E3FD31462046FFF77BFCFFF7C3FC1B
:10809000012220462121FFF730FD20460821FFF76D
:1080A000A1FE2A4620460021BDE8F840FFF788BE21
:1080B0004379012B70B5044614D0C26B0025436A86
:1080C00005649B1AC3632069038DAB420CD86379A6
:1080D000032B1BD1606AE36AA06223631844F8F79C
:1080E000E8F86063012070BDC36A03EBC50213F8B2
:1080F0003530052B08D1967801212046FFF756FC34
:108100000670236C013323640135DCE7042BE9D1CD
:10811000626AD4E90A138A4202D1216B994203D0E0
:108120000020A2622363DEE794F838301BB10649D1
:10813000064805F049F9E268C38A5268616B006934
:1081400004F0C5FCCEE700BFC21E080828B008082E
:108150002DE9F74F0023164604464171378C8360A2
:108160008371C362436280F83830B6F82490B6F861
:108170001A804FEA8905B6F816A0B6F81EB04FEA85
:10818000590905F004050AF00F0AC0E90423738CAD
:1081900001221F448261B38B9742B8BF174608F093
:1081A00003024FEA9808013F1543FA003F0902F025
:1081B0007802154347EA090242EA0A0242EA080243
:1081C0001A4352EA0B0233D101212046FFF7EEFB9E
:1081D00005706379022B17D9D4E90F787D0008F078
:1081E0000103BF09012105F07E054FEA580820462A
:1081F0001D4358EA070918BF45F08005FFF7D6FB75
:108200000570B9F1000FE9D1636A0025B18AE36313
:10821000E068FFF747FB2B490246204613F01AFBA4
:10822000738BB28B1344AB4248DD318D002241E0A9
:1082300065F07F05012120460193FFF7B7FB05702C
:108240003A01019B4FEA8A1502F03002BF0805F09F
:1082500040054FEA5A0A15430BF001024FEA5B0B47
:108260001543DA005B0802F0080215434FEA880262
:108270004FEA580802F0040215434FEA49024FEA58
:10828000590902F00202154394E7F36A03EBC203B3
:108290005878C0070DD55888A8420AD15968E068B7
:1082A0000135FFF7FFFA07490246204613F0D2FADC
:1082B000B6E701329142E8DC0521F0E703B0BDE802
:1082C000F08F00BFAD79020810B504464420F7F7DF
:1082D000F0FFC46010BD10B50446C1618800F7F717
:1082E000CFFF206210BD10B50446006AF7F7F0FF1B
:1082F0002046BDE81040F7F7EBBF10B5044601611A
:108300008800F7F7BDFF606110BD10B5044611B1DC
:10831000C068F7F7DDFF6069BDE81040F7F7D8BF28
:10832000012938B504460D460BDC02694FF0FF31D8
:108330004069920040F010FF002325706370636075
:1083400038BD4068F7F79CFF6368E060A360F3E71F
:108350000246407810B548B913785468022B21447E
:1083600008BFD368516008BF181910BD0020FCE792
:10837000002343700378012B9EBF4268436943F892
:10838000212070474B1E4268494213440B40436012
:10839000704738B50C461546FFF7DAFF10B10444B4
:1083A000A04200D138BD00F8015B2D0AF8E710B5F6
:1083B0000C460221FFF7CCFF10B10470240A447070
:1083C00010BD38B50D4604211446FFF7C1FF28B192
:1083D00005702D0A8470240A4570C47038BD0129C7
:1083E00070B5054606DC002909DA023921F00104DE
:1083F000FE2606E08B1E012BF7D80024F8E70024A8
:10840000F22646F435412846FFF7D1FF44B17F2CD0
:1084100009D844F43041284641F08001FFF7C7FFF6
:10842000C5E9066470BDA3004FF2AD21A201284644
:10843000DBB202F4E0421A4342F45062FFF7C1FF9C
:10844000EEE7C16910B5044629B17F290BD841F484
:108450003041FFF7ACFFA169204641F43D41BDE842
:108460001040FFF7A4BF8B008A014FF20D21DBB251
:1084700002F4E0421A4342F45062FFF7A2FFEAE737
:10848000114341EAC301FFF792BF072A89BF083AA7
:10849000D200D20042F04002072989BF08391143B7
:1084A000114341F0800141F48C41FFF780BF30B4AB
:1084B000DCB21D0144EA02225C10C3F3033305F46D
:1084C000E04504F480642A43234330BC1943FFF79A
:1084D00078BF38B54369054653F821404368E41A2C
:1084E000043CC4F34A0141F46041FFF760FF2B787C
:1084F000022B0AD1B4F5006F07D36FF30A0414F509
:10850000006F14BF0020012038BD0120FCE7F8B542
:10851000446907461E4654F822404268A41A043CA7
:108520006510BBB9EDB245EA012141F45041FFF7B6
:108530003EFF3B78022B0BD1FF2C09D924F0FF041E
:1085400014F5807F14BF0024012426463046F8BD70
:108550000124FAE76211C5F30A05231202F400525E
:1085600003F400632A43A512C4F3053405F48065BF
:108570001A43254342F4004245EA811141F4704117
:10858000FFF71FFFE2E738B54369054653F821407E
:108590004368E41A043CC4F34F02C4F30A3142F4C2
:1085A000784241F47041FFF70CFF2B78022B0AD17F
:1085B000B4F5800F07D36FF3150414F5800F14BFC3
:1085C0000020012038BD0120FCE7F8B504460D4627
:1085D0001646476813460A464FF24021FFF767FFE9
:1085E0002046330C2A464FF2C021FFF760FF384681
:1085F000F8BD072910B4044609D8FF2A07D842EA73
:1086000001215DF8044B41F40051FFF7D0BEB2F5F3
:10861000803F08D2134620460A465DF8044B4FF2CD
:108620004021FFF744BF20465DF8044BFFF7CDBF64
:108630002DE9F84341EA020706460C461546072F86
:10864000DDF820904AD803FA09F7FF2F0CD89142A1
:1086500001D0FFF71AFF47EA042141F440513046A8
:10866000BDE8F843FFF7A3BEFF2B4FEAC10814D8BB
:10867000914218D043EA012343F40051FFF797FEDB
:10868000304644EA891141EA0801FFF790FE48EAC2
:108690008511214341F4C051E1E7914203D03A46AC
:1086A000FFF7A7FFF3E784F007090125304605FA35
:1086B00009F545F43441FFF77AFE3A46494630461B
:1086C000FFF797FF304644EA891141EA080141F477
:1086D000C051FFF76CFE45F43C41C0E7BDE8F883AC
:1086E00008B50378012B04D9FF2902D9054805F004
:1086F0005BFEC9B241EA0221BDE8084041F41041E5
:10870000FFF755BECD1E080808B50378012B04D924
:10871000FF2A02D9054805F047FED2B242EA0121FC
:10872000BDE8084041F41841FFF741BECD1E0808DE
:10873000D2B242EA012141F42841FFF738BE38B5F0
:1087400043690C46054653F8223042689B1A0A4694
:108750004FF2402143F001030A3BFFF7A8FE2346F6
:10876000284622464FF43241FFF78AFE284621016F
:1087700004F0070401F08001214341F48841BDE881
:10878000384041F07801FFF712BE00001F2B73B58F
:10879000069E05460C4611D8114307290ED81A49E2
:1087A00044EAC202895D41F0010142EAC12141EA85
:1087B000831102B0BDE87040FFF7F9BD03FA06F17E
:1087C000B1F5805F0DD242EA4616284641EA0432EE
:1087D00046F4784141F0900102B0BDE87040FFF7E7
:1087E000F0BD1F3B214628460096FFF721FF064BB0
:1087F000E10028469B5D43F0010341EAC321214388
:1088000041F4F861D5E700BFFCA608081F2B2DE94D
:10881000F7430A9F06460C461546984610D841EA8B
:108820000203072B0CD8204BD95D44EAC12141EA51
:10883000C20141EA881103B0BDE8F043FFF7B7BDBC
:1088400008FA07F2B2F5805F0DD245EA47113046CB
:1088500042EA043241F4784141F0800103B0BDE8BE
:10886000F043FFF7AEBD4FF00109304609FA05F9B4
:1088700049F43441FFF79BFDA8F11F032A4629461E
:1088800030460097FFF7D4FE074B44EAC501304657
:10889000DB5D41EAC32141F4F861FFF788FD49F44B
:1088A0003C413046C7E700BFFCA60808436953F8BF
:1088B00021104368CB1A0131A3F1040310B4C3F3B0
:1088C0004A0204460ED0D91C0CDA23F4FF6121F0D1
:1088D000070111F5006F05D142F460415DF8044BCA
:1088E000FFF765BDC3F30A33204642F438425DF812
:1088F000044B43F47041FFF764BD436953F82220F1
:108900004368D31A0132A3F1040330B405464FEA99
:1089100063040ED0DA1C0CDA23F0FF0212F5807F1C
:1089200007D1E4B244EA012130BC41F45041FFF7E1
:108930003EBD5A11C4F30A04181202F4005200F4A6
:10894000006022439C12C3F3053304F480640243A5
:108950002846234342F4004243EA811130BC41F4EB
:108960007041FFF72EBD37B5144602220B4605466F
:10897000214600920722FFF709FF2846E10041F453
:108980008F4103B0BDE83040FFF711BD07289ABF03
:10899000024B33F8100040F2C720704700A70808C8
:1089A000C36C19440369012BC16404DD436D5A8C07
:1089B0009142C8BF5984704770474FF0FF31FFF7AD
:1089C000EFBFFFF7FABF6FF00301FFF7E9BF704792
:1089D00038B5C36C05461944036A994208D9083171
:1089E000406A21F00304E100F7F765FCC5E908409F
:1089F00038BD70B504460E4601211546FFF7E8FF65
:108A0000E16C626A204602F8316002EBC103012189
:108A10005D605970BDE87040FFF7C2BF70B5044695
:108A20000E4601211546FFF7D3FFE16C626A20462E
:108A300002F8316002EBC103022201215D605A702D
:108A4000BDE87040FFF7ACBF00221146FFF7E6BF5C
:108A50000A460221FFF7E2BF70B50D1E044605DD90
:108A6000FFF7B6FF00231E46AB4205DB2946204632
:108A7000BDE87040FFF794BFE26C012D616A1A44B3
:108A800003F1010301EBC200467014BF002094F80B
:108A9000280001F83200E7E7F8B5D0E90B530446A7
:108AA0000E4601331746AB4206D90435406BA90088
:108AB000F7F701FCE5626063C6F30E01D4E90C3000
:108AC0005A1C00EB8305226341EAC732002120F8DB
:108AD00023204FF6FF733246A06D6B80FFF72FFE09
:108AE000A06D00220321BDE8F840FFF7F9BD024662
:108AF000007D28B1D36C526A5B1A013B12F8330037
:108B0000704737B5456D0B461446ED8AED0708D51D
:108B10000222214600920622806DFFF777FE03B005
:108B200030BD806D03B0BDE83040FFF7D9BD70B5F2
:108B3000002405462646EB6CA34200DC70BD6B6A40
:108B400003EBC4035A78012A07D15E702846B5F8B2
:108B50004A105A682144FFF7D4FF0134EBE7F8B517
:108B600004461E4617460D46FFF7E1FF31463A46DA
:108B7000A06DFFF73EFD2946A06D0322BDE8F84039
:108B8000FFF7F1BE38B504460D46FFF7D0FF0322CC
:108B90002946A06DBDE83840FFF7E5BE10B50821B5
:108BA0000446FFF7EFFF002220461146BDE81040C3
:108BB000FFF71FBFF8B5044617461E460D46FFF7E0
:108BC000B6FF3A46A06D0021FFF713FD3246A06DB7
:108BD0000121FFF70EFD2946A06D0322BDE8F840F4
:108BE000FFF7C1BEF8B5C76C04460E460025BF1A94
:108BF000E36CAB4200DCF8BDBD4211D0636A03EB0D
:108C0000C5035A78012A0BD15A68B24208D1002212
:108C100020465A703246B4F84A102944FFF771FFD3
:108C20000135E5E7002238B50C4611460546FFF749
:108C3000D9FFE2000021A86D42F00202FFF7D9FC43
:108C4000002228461146BDE83840FFF7D2BE13B5D2
:108C5000446D1346E48AE40707D5022200920622F7
:108C6000806DFFF793FD02B010BD806D02B0BDE8CE
:108C70001040FFF749BD0000F8B5C369044615462A
:108C80009E5C602E06D147680A461348134908F0D7
:108C900037FB3860022D0DD8636D9A8C52B9DB8A90
:108CA000DB0707D40E4B5A5D31462046BDE8F8403D
:108CB000FFF79FBE002220461146FFF793FFB4F84E
:108CC0004A20636C002120461A44521B013AFFF7E8
:108CD000BEFF0022E8E700BF74AF0808DF1E0808E7
:108CE00000A80808036873B51A7804465D88022650
:108CF000042A04BF5A6842F825106A1C00215A80D1
:108D0000B0F84820FFF7A3FF002233460096114633
:108D1000A06DFFF73BFD002200962B461146A06D8B
:108D2000FFF734FD02B070BD002273B504460D4656
:108D300011460226FFF756FF626D29462068D38A46
:108D400043F02003D382FEF7C3FDB4F84820054664
:108D500000212046FFF77BFF0022009601231146E9
:108D6000A06DFFF713FD0022009603231146A06DAE
:108D7000FFF70CFD002200962B461146A06DFFF771
:108D800005FD00222046114602B0BDE87040FFF705
:108D900030BE00000D2902D10749FFF7C5BF0F29DA
:108DA00003D100225421FFF739BEB1F10E024FF07A
:108DB000010118BF0122F6E7A4BC0808F8B5C76C8A
:108DC0000546446A07F10053023B04EBC304D4E9AF
:108DD000020184E80300667856B9B5F84A203146A6
:108DE00028463A44013AFFF732FF01236660637078
:108DF00028464FF0FF31BDE8F840FFF7D1BDF8B588
:108E000004461E4617460D46FFF791FE31463A4688
:108E1000A06DFFF7EEFB2946A06D0322BDE8F840E8
:108E2000FFF7A1BD10B402F1290400230A46E1B204
:108E30005DF8044BFFF7E3BF70B504460E461546D8
:108E400062B1037D53B1084605F08EFC021E05DDBC
:108E500020467021BDE87040FFF7E0BD0635324680
:108E600020460023E9B2FFF7CAFF00222046114640
:108E7000BDE87040FFF7BDBD07B513460222009262
:108E80000722FFF783FC03B05DF804FB38B50D46FD
:108E900014463BB9037D2BB1806D5268FFF7A9FBE7
:108EA000207838BD237833B962682946806DFFF792
:108EB000A0FB0020F5E7012B06D1626801322946AC
:108EC000806DFFF7D9FFF4E79A1E012A04D8626883
:108ED000520042F00102E8E7542B01D10022EEE7F4
:108EE000014805F061FA00BFF81E0808F8B5002433
:108EF0000546FFF71CFE2746EB6CA34200DCF8BDDD
:108F00006E6A06EBC4025378022B0ED10121577012
:108F100000232846FFF7BAFF06F83400B5F84A10D8
:108F2000012228462144FFF7ECFD0134E4E738B57F
:108F300004460D46FFF7DAFF2946A06DFFF7B6FCA1
:108F4000A36D01225A7038BDF8B504460E46174687
:108F50000A4619461D46FFF745FEE36C616A9B1BF6
:108F600001EBC30211F833303B705378012B0DD065
:108F7000022B14D0CBB9B4F84A202946E36C204622
:108F80001A44921BBDE8F840FFF761BE5268AA423E
:108F90000BD02946A06DBDE8F840FFF776BA002354
:108FA00029462046FFF772FF3870F8BD10B5044619
:108FB00013460A460121FFF7C7FF20464FF0FF3155
:108FC000BDE81040FFF7ECBC70B5049E04461D469A
:108FD000FFF7ECFF324620462946BDE87040FFF718
:108FE000E5BFF0B5012585B0002204460DF10F0361
:108FF0000DF10E010095FFF7E7FF9DF80F709DF84A
:109000000E602A4639462046FFF7F3FC31462046DB
:109010000022FFF7EEFC2A4639462046FFF7E9FC1E
:1090200000223146204605B0BDE8F040FFF7E1BC24
:109030002DE9F04104461D46089FDDE90686FFF74D
:10904000B5FF294642462046FFF7B0FF3A46314673
:109050002046BDE8F041FFF7A9BF2DE9F04186B0F9
:109060000226012504460DF117030DF1150100221A
:10907000029601930DF116030095FFF7D9FF9DF8B5
:1090800017809DF8167020469DF815100022FFF7F6
:10909000B0FC324641462046FFF7ABFC2A46394633
:1090A000204606B0BDE8F041FFF7A3BC30B587B05D
:1090B0000025044601220DF117030DF1150102955B
:1090C0000193022300930DF11603FFF7B1FF204631
:1090D0001921FFF757FD2A462946204607B0BDE86B
:1090E0003040FFF786BC73B504460E46154672B98C
:1090F00001220DF10701FFF759FF0C35002332461D
:109100002046E9B202B0BDE87040FFF778BE00210A
:10911000FFF7EDFC20B901220DF107012046EAE737
:109120000A4620460DF10701FFF740FF9DF8072092
:10913000204601230421FFF712FD00220121A06D2A
:10914000FFF7A3F9D9E7000037B500220DF10701B9
:109150000446FFF72BFF9DF807302BB165680749E0
:10916000074808F0CDF8286022212046FFF70AFDC5
:10917000A36D01225A7003B030BD00BF061F08085E
:1091800074AF0808022A7FB504460E46154614D867
:10919000436D9A8C8AB9DB8ADB070ED4184B0DF12C
:1091A0000F015A5DFFF702FFE3699DF80F10585D4C
:1091B000602813D1595504B070BD0DF10F01204640
:1091C0000022FFF7F3FE626CB4F84A3020461344E5
:1091D00000225B1B591EFFF794FCE5E78842EAD0AA
:1091E000FFF7D4FB024608460649FFF7CFFB646849
:1091F000134600903246044808F082F82060DAE70F
:1092000000A80808101F080874AF080870B50446C5
:109210000D4616464BB90F21FFF7BCFD32462946D5
:109220002046BDE87040FFF7ADBF70BD03297FB594
:109230000446164613D1182501220DF10F01FFF740
:10924000B5FE3146204600230DF10F02FFF77CFEEC
:109250002946204604B0BDE87040FFF793BC0529BD
:1092600006D101220DF10F011725FFF79FFEE8E758
:10927000022301220DF10E01192500930DF10F03B8
:10928000FFF7A2FEDDE7F0B5044685B00E461546B1
:10929000CAB90223077D0DF10E0102750122009368
:1092A0000DF10F03FFF790FE2B4632462321277561
:1092B0002046FFF7A4FD00222046114605B0BDE878
:1092C000F040FFF796BB012A09D100230DF10F02F0
:1092D0002946FFF739FE2B4632462421E8E70DF1F7
:1092E0000F010022FFF762FE2521204605B0BDE8F0
:1092F000F040FFF747BC10B50446D0E90C3003F14D
:109300008043013B00EB8303DA7822F08002DA70BD
:10931000043B98420BD893F90320002AF8DA1A8804
:109320000021A06DC2F30E02FFF709FA05E059B95A
:109330004FF40051A06DFFF73AF8A06D0022032111
:10934000BDE81040FFF7CCB910BD10B504460121AF
:10935000FFF7D1FF0122A06D0021FFF7D5F9002210
:1093600020461146BDE81040FFF743BB73B5046BC0
:1093700005460E46DCB104F18044436B013C03EB2F
:10938000840292F90120002A20DA33F82430C3F352
:109390000E038B421AD100230DF107020121012493
:1093A000FFF7D2FD00220121A86DFFF799F92846A9
:1093B000FFF79CFD3146A86DFEF7DAFF44B10021AE
:1093C000284602B0BDE87040FFF795BF0024EEE7E5
:1093D00002B070BD38B50D46044611467AB14FF45F
:1093E0000051806DFEF7E3FF00220121A06DFFF721
:1093F00077F929462046BDE83840FFF798BDFFF7CA
:109400007AFFF6E72DE9F04104460D4672B30021DC
:109410001646D0E90C3C0F4603F18043013B0CEBB0
:109420008303184690F901E0BEF1000F09DA90F9C4
:1094300003E0BEF1000F04DA002F08BF0746E1B9D0
:109440000146013EA0F10400ECD1A06D21BB6FF0FC
:10945000030672439E18B44518D94FF40051FEF725
:10946000A6FF00220321A06DFFF73AF925F4004181
:109470002046BDE8F041FFF75ABDB0F80080B1F8D2
:1094800002E068F30E0EA1F802E0D9E79A5AC2F39F
:109490000E02FFF754F9E4E74B8847F6FE7262F3D9
:1094A0000E0325F400424B803146FFF748F932465F
:1094B0001321A06DFFF714F932463146A06DFFF776
:1094C00098F832460121A06DFFF70AF93D88C5F3EF
:1094D0000E05CBE77FB504460E4615468AB90DF159
:1094E0000F01FFF763FD3246204601230921FFF7F4
:1094F00086FC2A462946204604B0BDE87040FFF7A6
:1095000078BA012A35D11146FFF7F1FA024688B937
:1095100002230DF10E01204600930DF10F03FFF71A
:1095200053FD012332460E21204604B0BDE87040B1
:10953000FFF765BC0DF10F02204600230221FFF763
:1095400003FD2B469DF80F2020460421FFF707FB63
:10955000A06D00220221FEF798FF0DF10E012046BA
:109560000022FFF723FD4FF0FF312046FFF718FAE6
:10957000D7E70DF10F010022FFF718FD4FF4085156
:10958000A06DFEF714FFCCE738B50446FFF715FAD7
:1095900001220021806DFFF7B7F822212046FFF756
:1095A000F1FA47F6FF72D4E90C35013B05EB830570
:1095B00023636B88C3F30E03934228D01322002148
:1095C000A06DFFF7A1F84FF42051A06DFEF7EFFE5C
:1095D000A3680021A06D1A68FFF78FF9698847F624
:1095E000FE73C1F30E029A420BD14FF48E41A06D6F
:1095F000FEF7DDFEA36820461968BDE83840FFF796
:10960000B5BEC1F30E012046FFF791FCF2E738BD6D
:109610002DE9F3410E460021174604461D46FFF78B
:1096200066FA024648BB0DF107012046FFF7BEFC73
:109630001DB901212046FFF7B3F910212046FFF79D
:10964000A1FA1DB99DF8073084F828302046FFF7AD
:109650004DFCA06D4FF420515EB3FEF7A8FE3A46D4
:109660000121A06DFFF749F945BB4FF0FF312046BE
:1096700002B0BDE8F041FFF793B90A4620460DF16C
:109680000701FFF793FC1DB901212046FFF788F978
:109690009DF80700431E022BD3D9FFF777F9D4F8C2
:1096A000048002460749084807F02AFEC8F800006F
:1096B000C7E7FEF77CFE3A463146D2E702B0BDE886
:1096C000F08100BF241F080874AF08080023FFF7CB
:1096D0009FBF0123FFF79CBF426D83682DE9F341D3
:1096E000D58A04461E68928C05F01103C6601343A8
:1096F00000F0F98015F0010506F1020721D14FF0C5
:109700000208B0F848202946FFF7A1FA01232A46AB
:109710002946CDF80080A06DFFF738F82A460123CE
:109720002946CDF80080A06DFFF730F805212046CE
:10973000FFF728FAB4F848102A4620460131FFF70F
:10974000E0F9D4E915309A8C002A67D1D98A11F052
:10975000010508D14FF42051FEF729FE3A4629466B
:10976000A06DFFF7CAF80022A06D1146FEF7E0FFDA
:1097700020212046FFF706FA4FF42051A06DFEF796
:1097800016FE3A460021A06DFFF7B7F8636DD98A3F
:1097900011F0010100F08E80022501220021A06D50
:1097A000FEF7B2FF0523062200210095A06DFFF70A
:1097B0002DF8A06D2A460021FEF71BFFA06DFEF7D5
:1097C00040FE39462046FFF7D1FD636DDB8ADB079B
:1097D00040F18980B4F84820204600210132FFF78B
:1097E00036FAA06D4FF48E41FEF7E1FDA06D142214
:1097F000002143682364FEF787FFA06D4FF40451F6
:10980000FEF7D5FDA06D01221421FEF769FF22218C
:10981000204602B0BDE8F041FFF7B4B94FF4005163
:10982000751CFEF7C4FD00221321A06DFEF758FF42
:1098300000220121A06DFEF753FF3A460421A06DDE
:10984000FEF77DFF294620460336FFF78FFD0022F5
:10985000A06D1146FEF76CFF20212046FFF792F91C
:109860004FF42051A06DFEF7A2FD32460121A06DFC
:10987000FFF743F84FF40051A06DFEF798FD00226A
:109880000321A06DFEF72CFF44F22071A06DFEF7BE
:109890008EFD31462046FFF769FD03220421A06DAD
:1098A000FEF732FF4FF43051A06DFEF780FD2A46DF
:1098B000012168E7B4F8482020460132FFF7C7F9D4
:1098C00005212046FFF75EF9D4E91530D98A11F059
:1098D00001017FF461AF0122FEF716FF222120462D
:1098E000FFF750F96DE702B0BDE8F08170B50546AD
:1098F0000C46D0E91560F68AF6070BD544EAC40495
:109900009200FEF776FE44F4CC51A86DBDE870409D
:10991000FEF74DBDBDE87040FEF70ABF2DE9F84FD8
:10992000002504460F469146A846FFF700F94D452D
:1099300010D10026B3464E452BD171422046FFF789
:109940002FF8B4F84A20E36C39461A44BDE8F84FC2
:10995000FFF7CCBFE66CD4F824A0013E761B0AEBDF
:10996000C6025378022B12D10123394682F80180B6
:109970002046FFF78BFA0AF83600B4F84A103A4648
:10998000E36C204619440139491BFFF7BAF8013549
:10999000CDE7E36CD4F824A003F1FF38A8EB060868
:1099A0001AF83820BAB1B4F84A50002120461D44B4
:1099B000013DAD1B2A46FFF74AF901231AF838206A
:1099C00004212046FFF7CBF8002229462046FFF766
:1099D00098F80AF838B00136ADE70000037D37B5D6
:1099E00004460D4613B15F4804F0DEFC426DD38A95
:1099F00043F00103D382FFF779FA012D0BD1A3685D
:109A0000204619680231FFF792FAA36820461968C8
:109A10000131FFF7ABFC012200212046FFF77EFF5A
:109A2000002202212046FFF76CF801220021A06DE0
:109A3000FEF7DFFD00221221A06DFEF751FEA368A4
:109A40000021A06D1A68FEF77AFEB4F848100022D3
:109A500020460131FFF755F8E168A06DFEF726FFBB
:109A6000A368A06D1968FEF783FC236BBBB103F1FB
:109A70008043626B013B02EB83039A420FD893F958
:109A80000310002926DA1A880021A06DC2F30E0205
:109A9000FEF755FE00220321A06DFEF721FE0121F5
:109AA0002046FEF7D9FFBDB914222946A06DFEF766
:109AB0002BFEA06D4FF40451FEF779FCA06D01223E
:109AC0001421FEF70DFE2221204603B0BDE83040F0
:109AD000FFF758B8043BD0E7A36820461968023165
:109AE000FFF744FCA06D14220221FEF70DFEA06DCD
:109AF00000220121FEF77DFDA06D01221421FEF759
:109B0000EFFD0DF1070120460122FFF74FFA002378
:109B10000DF1070220460121FFF716FA2046022226
:109B20000021FEF766FF012220460221FFF7F6FE24
:109B300020463021FFF726F8A06D4FF42051FEF7A4
:109B400036FCA368A06D01211A680132FEF7D5FE2C
:109B500020460121FEF780FF204603B0BDE83040DB
:109B6000FFF72CB93A1F0808F8B5164604460D460B
:109B7000520093B1CB1C02211A44FFF7CFFE012201
:109B800045EA06231D212046FFF714F8002220464F
:109B90001146BDE8F840FEF72CBF8B1C02211A4489
:109BA000FFF7BCFE33462A461C21ECE72DE9F743BC
:109BB0000F4616460121B0F848201D460446DDF840
:109BC00028904FF00208FFF742F80123CDF80080FB
:109BD0001A461946A06DFEF7D9FD55EA09052DD1A3
:109BE0002046FEF7A4FF2A464146A06DFEF701FD80
:109BF00039692046FFF776F803221A21A06DFEF797
:109C0000B2FE32460121A06DFEF7F3FC324602217E
:109C10002046FFF783FE25B16FF001012046FEF7D5
:109C2000BFFEA06D03222B21FEF79DFE00222046E1
:109C3000114603B0BDE8F043FEF7DBBE06F10209B2
:109C4000414620464A46FFF769FE49462046FEF750
:109C5000A7FEFEF76CFFCBE72DE9F34115460F4653
:109C6000B0F8482001211E4604464FF00208FEF7D6
:109C7000EEFF0123CDF800801A461946A06DFEF7CD
:109C800085FD354318D12046FEF751FF2A4641464F
:109C9000A06DFEF7AEFC39692046FFF723F8A06DF2
:109CA00003221A21FEF75FFE00222046114602B071
:109CB000BDE8F041FEF79DBE204642464146FFF713
:109CC0002DFE2046FEF733FFE5E7042A70B5044673
:109CD00086B00E4615462AD102294FF0000518D14C
:109CE00001220DF117010DF116030095FFF76CF934
:109CF0002A463146A06DFFF7BFF826212046FEF721
:109D000041FF00222046114606B0BDE87040FEF734
:109D100070BE0DF1150302220DF11701029501939A
:109D2000012300930DF11603FFF782F9E5E7012AFD
:109D300001D9032A04D1324601212046FFF7EEFD66
:109D40001335002332462046E9B2FEF708FFD8E774
:109D500038B5044604220D460021FFF7DFFD2046FA
:109D60000421FEF71DFE1F21FEF70CFFA06D4FF42E
:109D70002051FEF71CFB2A46A06D0021FEF7BDFD19
:109D8000002220461146BDE83840FEF732BE37B506
:109D900004460D460021FFF7AEFA20464FF0FF3192
:109DA000FEF7FEFDA36819680231FFF7DFFA2046CF
:109DB00000225421FEF732FE204600225421FEF7F5
:109DC0002DFE204600225421FEF728FE20460522C3
:109DD0000221FFF7A3FD0322204600231C21FEF7EA
:109DE000E9FEA36820461968FFF7A1F82946A06D8F
:109DF0000225FEF7BDFA20460121FFF77CFA204636
:109E00000221FEF729FE0122A06D0021FEF77CFC55
:109E1000A06D4FF42051FEF7CAFAA368A06D00218F
:109E20001A680232FEF769FD0023009501211A46E7
:109E3000A06DFEF7ABFC204601220021FEF7D9FD04
:109E4000002220461146FEF7D4FD20460022542170
:109E5000FEF7E4FD294620460522FFF75FFD0023BB
:109E6000032220461C21FEF7A5FE20461021FEF706
:109E700089FEA06D4FF42051FEF799FAA368A06DFA
:109E800000211A680132FEF738FDA36820461968E0
:109E9000FFF76CFAA06D4FF40051FEF788FA00222C
:109EA000A06D0121FEF71CFCA36820461968013152
:109EB000FFF75CFA0121204603B0BDE83040FEF711
:109EC0006FBD0000436D73B5DD8A044615F00106D1
:109ED00013D001220021FFF721FD0022022120469C
:109EE000FEF70FFE0022A06D1146FEF782FB002256
:109EF0001221A06DFEF7F4FB1BE0027D002A47D083
:109F00003146C5F38715FEF7F2FD542825D12046CA
:109F1000FEF753FDADB92A462946A06DFEF7ACFF0A
:109F2000636D9A8C002AE2D1DB8A03F01103002BC7
:109F3000DDD1226B2046E16802B0BDE87040FFF73A
:109F400061BA32463146A06DFEF753FB01232A4623
:109F500004212046FEF703FEE2E70DF10701324639
:109F60002046FFF723F89DF80710A9420DD0284698
:109F7000FEF70CFD024608460849FEF707FD666835
:109F80000346074807F0BCF93060002DC8D0DDE774
:109F90000DF10701FFF70AF8C2E700BF421F0808EA
:109FA00074AF0808F8B51646044600250F46FEF7BC
:109FB000BEFD31462046FEF70BFDE36C2A46B54256
:109FC0000CD1B4F84A20394620461A44FFF78EFCDB
:109FD00029462046BDE8F840FEF7E2BC5819616A00
:109FE000013521F83020EAE773B516460D46002208
:109FF0000DF107010446FEF7D9FF721C022120462D
:10A000002A44FFF7CFFF012345EA062228212046F4
:10A0100002B0BDE87040FEF7A2BD37B504460D465C
:10A0200000220DF10701FEF7C1FF2A46204602215A
:10A03000FFF7B8FF01232A462721204603B0BDE8D9
:10A040003040FEF78CBD37B50D4600220DF10701FB
:10A050000446FEF7ABFF5DB1204604220121FFF765
:10A06000A1FF1E21204603B0BDE83040FEF78ABDA7
:10A070002A46A06D0121FEF7BCFA20461E21FEF7FC
:10A0800081FD2A462946204603B0BDE83040FEF750
:10A09000B0BC37B504460D468AB103220121FFF753
:10A0A0003DFC022201212046FFF77CFF00232A46C7
:10A0B0000B21204603B0BDE83040FEF7A0BE0DF1F5
:10A0C0000701FEF773FF022220461146FFF76AFFE1
:10A0D00001232A460A21ECE77FB5012504460DF14C
:10A0E0000F030DF10E0100220095FEF76DFF9DF8A4
:10A0F0000F609DF80E1020460022FEF77AFC2A46DB
:10A100003146204604B0BDE87040FEF772BCF8B599
:10A1100004460F4601211D461646FEF79DFC2046CB
:10A12000FFF7DAFF0F212046FEF734FE2046FFF747
:10A13000D3FF39462046FEF7FAFE20464FF0FF31A6
:10A14000FEF78AFC31462046FFF710F92046FEF75D
:10A1500034FCA06D01220021FEF7D6FA0022204631
:10A160001146FEF746FCA06D4FF42051FEF71FF993
:10A170002A46A06D0021BDE8F840FEF7BEBB0000F6
:10A18000138B2DE9F34104460161D81E0E46118C54
:10A19000154643426265434123750023E364A36986
:10A1A0008B4205D2E069F6F786F82B8CE061A3615B
:10A1B000626D538B928B1344EA8A510748BF013377
:10A1C00092074FF0000248BF01331146934240F01E
:10A1D000DB80227D002A40F0EB80A2699A4200F2E7
:10A1E000E980226A002360219A4240F0EC80042E2C
:10A1F000A06D14BF01210221FEF792F80023626DC9
:10A20000A4F84830938CD28A02F01101194305D08A
:10A21000D20740F1DD801523A4F848308B4920682F
:10A22000FDF756FB2F8C6B8C064694F814803B444C
:10A23000A06D6364B8F1000F00F00C81626D918C29
:10A24000002940F0CA80D28A12F0010F0CD13946A1
:10A25000032F6F8BA8BF0321032F88BF01F1FF31AC
:10A2600012F0110F00F0BB80B4F84820023292B215
:10A27000A4F84A201A440227511AFEF7B0F8012325
:10A28000002207210097A06DFEF780FA0722032322
:10A2900000971146A06DFEF779FA07223346009722
:10A2A0001146A06DFEF772FA636D9A8C1AB9DB8ABB
:10A2B00003F030032BB10022B4F84810A06DFEF774
:10A2C0000FFA01220021A06D0226FEF7DEF802221D
:10A2D0000121A06DFEF7D9F803220621A06DFEF73B
:10A2E000D4F84FF42451A06DFEF761F8A368012162
:10A2F000A06D1A680432FEF700FB6A8B0221A06D84
:10A30000FEF777F9022300224FF48541A06DFEF796
:10A31000B7F8A3680021A06D1A680532FEF7EDFAC0
:10A32000A368A06D19680431FEF722F86B8B4FF01B
:10A3300002120221A06D00255A43FEF75AF90322AA
:10A340002C21A06DFEF70FFBA368A06D19680531E5
:10A35000FEF70EF8636D5A8BAA4248DC032A0DD92A
:10A360009A8C5AB9DB8ADB0708D4B4F84A20062154
:10A37000636CA06D1A44033AFEF7C6F9204602B09A
:10A38000BDE8F041FFF7A8B9E069815401321DE74B
:10A39000C86A00EBC20001324178CF0741BF47884D
:10A3A0000909E069C155616D088D9042F0DC14E740
:10A3B0000022F8E7227D002AE2690CBF002160211B
:10A3C000D154013309E7606A20F8331001330BE7F9
:10A3D0000BB9132320E714231EE7002144E7EF8A7B
:10A3E000B4F84820BF067FF543AF01323FE72B4664
:10A3F000062200960021A06DFEF7C8F9E3695A5DB8
:10A4000022B1012303212046FEF7A9FB022D12DC15
:10A41000636D9A8C7AB9DA8AD2070CD4022D02D1F4
:10A420005B8B032B07D10A4B0022A06D595DFEF711
:10A430002CF801358EE7B4F84A100022636C2046F0
:10A4400019440139491BFEF75CFBF2E740A90808F3
:10A4500000A80808E26B0421FDF79BFFD4E9153042
:10A46000DF8A17F0010742D0226C0421FDF791FF2B
:10A47000B4F84810A06D0227FDF7B1FF4FF4A023F8
:10A4800042460621A364A06DFDF7FFFF01221421BF
:10A49000A06DFEF725F900970622B4F84830414632
:10A4A000A06DFEF773F90123424641460097A06D67
:10A4B000FEF76CF90323424641460097A06DFEF774
:10A4C00065F90097334642460721A06DFEF75EF915
:10A4D0002046FFF701F9636D9A8C002A49D00023CA
:10A4E00019462A8D9A425BD802B0BDE8F081B4F8D3
:10A4F00048304FF00208616C05339BB21944A4F850
:10A500004A30FDF76CFF3A46CDF800800123A06D7C
:10A510000721FEF73BF90722CDF8008003231146FF
:10A52000A06DFEF733F907223346CDF800801146BF
:10A53000A06DFEF72BF93A46B4F84810A06DFEF76F
:10A54000CFF8626C3946A06DFEF753F8B4F84810A6
:10A550003A4620460331FEF7D4FAB4F8482039468B
:10A56000A06DFEF7E5F804222D21A06DFEF7FBF9A2
:10A57000AEE7DE8A16F00106B1D10F4F2B8CB34245
:10A58000ADDDB4F84A20636C17F8011B1A44A06DC6
:10A59000013A921B0136FEF7B7F8032EEED19EE783
:10A5A000EA6A02EBC30012F833200133052A02BF26
:10A5B0004288E069815494E700A808082DE9F34136
:10A5C0000E4601EB4201044615461F46FEF78FFA80
:10A5D00070288DF8060035D1E26C0021636A2046B0
:10A5E00003EBC20313F80C6CFEF781FA072805464B
:10A5F0000DD888B12046FEF7E1FBE36C626A03F1F7
:10A600000053013B02F8336002B0BDE8F0815428EA
:10A61000F0D01F4803F0C8FE02460DF107012046A6
:10A62000FEF7C4FC2046FEF7C8F932460321012399
:10A63000FEF795FA2A463146204602B0BDE8F041C1
:10A64000FEF7D7B946EA05286FB18A1C20460221D9
:10A65000FFF764F9434600221D212046FEF7AAFABF
:10A6600000221146E8E7354304D00A46204602217D
:10A67000FFF754F90DF1060120460022FEF796FC83
:10A68000012342461B212046FEF769FAE8E700BF96
:10A690004C1F08082DE9F041C66C1546D0F824C0BF
:10A6A0000446013EDDF818800CEBC6077A78012AD3
:10A6B00013D1D7F804E09E450FD0C6450DD01CF845
:10A6C00036300B7079682960FEF78CFA20464FF01F
:10A6D000FF31BDE8F041FEF763B90A462B6801215E
:10A6E0002046FEF731FCF1E77FB5002303AA0DF108
:10A6F0000B01044603934FF0FF330093FFF7CAFFAB
:10A700009DF80B50039E204629463246FEF771F90C
:10A7100032462946204604B0BDE87040FEF769B9CC
:10A72000F7B504460E461546002A57D113460121B7
:10A730000DF10702FEF708FC022220461146FFF742
:10A7400031FC012320460D220A21FEF758FB0DF1B2
:10A75000070120460222FEF729FC0DF107012046E1
:10A760000122FEF723FC2A460DF107012046FEF7E1
:10A770001DFC9DF80770204601223946FEF739F985
:10A78000394620460222FEF734F9022220461146BD
:10A79000FFF708FC012320460C220A21FEF72FFBBD
:10A7A000022220461146FFF7B9F82B462A462046DA
:10A7B0001C21FEF7FFF92A4629462046FEF719F923
:10A7C0002046FEF793FB204601223146FEF764F94E
:10A7D000204603B0BDE8F040FFF786BFFEF786FBDA
:10A7E000AB1E314620465A425A4103B0BDE8F04004
:10A7F000FEF752B970B5044686B00D46164623B929
:10A8000006B0BDE87040FEF7BDBC00221146FEF761
:10A81000E9F9204600220121FEF7E4F932462946F3
:10A820002046FEF729FA002304AA0DF10F01049334
:10A830004FF0FF33204601260093FFF72BFF049DC6
:10A8400005AA0DF10F012B46204600950596FFF74E
:10A8500021FF02232A46059900933346A06DFDF798
:10A86000D5FF06B070BD7FB504460D46164623B928
:10A8700004B0BDE87040FEF7FFB900221146FEF7B4
:10A88000B1F9324629462046FEF7F6F94FF0FF337C
:10A89000002503AA0DF10B01204600930395FFF755
:10A8A000F9FE0223039A294600930123A06DFDF7C8
:10A8B0006DFF2A462946204604B0BDE87040FEF7E9
:10A8C00098B800007FB50E4600210446FEF70FF948
:10A8D000831E05468DF80B00012B38D8002E34D08E
:10A8E000012E19D10B4603AA0391204600910DF1C8
:10A8F0000B01FFF7CFFE039D44F240212B462A4671
:10A90000A06DFDF7BDFD2A469DF80B10204604B052
:10A91000BDE87040FEF76DB8022E0ED10B4603AABB
:10A920000391204600910DF10B01FFF7B3FE039D4B
:10A9300044F2C0312B462A46E2E7104B64689A5D28
:10A940000F49104806F0DCFC206004B070BD70B9FF
:10A9500001220DF10B012046FEF728FB32461121A2
:10A960002B462046FEF7FBF82A462946CEE7FEF79F
:10A970000DF8054902466468E3E700BFCCC108084A
:10A98000541F080874AF08085D1F08082DE9FF412F
:10A9900004460D460121FEF7AAF807468DF80A0085
:10A9A00000212046FEF7A3F8BB1E06468DF80B00DB
:10A9B000012B00F2D480831E012B00F2FB80A5F155
:10A9C00009030C2B9CBF0D35EDB21F2D01D0212D9D
:10A9D00024D1002301220DF10B01204600930DF13B
:10A9E0000A03FEF7F1FA9DF80A30022B07D07B4BE1
:10A9F00066685A5D7A497B4806F082FC30601F2DFC
:10AA000020460CBF2E212F21FEF7BCF80022022188
:10AA1000204604B0BDE8F041FDF7EBBF012602235C
:10AA200003AA0DF10B012046039300960023FFF7C4
:10AA300031FE32460DF10A012046FEF7B7FA1D2D10
:10AA40007ED8DFE805F04C4C4C4C4C4C7D7D7D7D38
:10AA50007D7D7D7D7D7D7D7D7D7D7D7D252D320F87
:10AA60000F374347192DA06D9DF80A604FF0010282
:10AA7000039B06D14FF48141FDF702FD01223146CF
:10AA8000C6E7032E0CBF44F2C0014FF48241F3E746
:10AA9000039B01224FF48641A06DFDF7F1FC11E00C
:10AAA000039B012244F24001F6E7039B01224FF48D
:10AAB0008041F1E7039941F6090343EA8111A06D52
:10AAC000FDF775FC01229DF80A10A1E7039941F6F4
:10AAD0000923F2E7039B012244F24031DCE79DF8B1
:10AAE0000A609DF80B30B34205D067683E493D4887
:10AAF00006F006FC3860032E4FF00002204614BF1B
:10AB0000062600261146FEF76DF80122039B4FF43E
:10AB10008541A06D2E44FDF7B3FC344BA06D33F896
:10AB20001610FDF744FC42F20101A06DFDF73FFC59
:10AB30004FF40051A06DFDF73AFC0022012167E7B8
:10AB400020460121FDF72CFF244B29495A5D254859
:10AB5000646806F0D5FB206004B0BDE8F08157EAD8
:10AB6000000827D101260DF10A0302220DF10B0185
:10AB700020460096FEF728FA322D17D0332D17D035
:10AB8000464600232A4612212046FDF7E8FF56B12B
:10AB900000220121A06DFDF778FC00230322112182
:10ABA0002046FDF7DCFF0022114631E70625E8E7E5
:10ABB0000725E6E720464FF0FF31FDF7F1FE384666
:10ABC000FDF7E4FE024630460A49FDF7DFFE034684
:10ABD0000448646806F094FBBDE700BFCCC10808D8
:10ABE0006D1F080874AF08087D1F080810A7080823
:10ABF000901F08089E1F08082DE9F0430446C1680D
:10AC000085B0FEF7B3FB626DD18A928C01F011031F
:10AC100013432ED011F0010117D1B4F8482020467B
:10AC20000132FEF714F8636D9D8C55B94FF4205135
:10AC3000A06DFDF7BCFBE2682946A06D0132FDF76F
:10AC40005CFE05212046FDF79DFF21212046FDF7F2
:10AC500099FF636DDA8AD20706D49B8C23B9E16829
:10AC600020460131FEF782FB12220021A06DFDF784
:10AC70004BFDA06DFDF7E5FB237D002B5ED1A36DA1
:10AC8000656C5B68013DA3632368EA002D095B885E
:10AC900002F07802E363636D5E8BDF8AB3F81C9089
:10ACA000B3F81E8006F0030307F00F07B6081A4337
:10ACB00045EA0703A06D334343EA090353EA080357
:10ACC00065D10121FDF765FBB4F85060B4F852700E
:10ACD000720007F00103B609012102F07E027F082D
:10ACE000A06D57EA060542EA030218BF42F080024F
:10ACF000FDF74FFB002DEBD1636DA76D998A20689E
:10AD00007E68FCF7CFFD47490246384610F0A2FDA9
:10AD1000626D538B918B108D0B44AB4271DCA36D34
:10AD200000259F88BE1BA4F85060D4E915301A8D09
:10AD3000AA4268DC4368DB1BA4F852302369042B69
:10AD400021D1A36DD3E9027623685868237D5BB9CE
:10AD5000A56BE16B3544002962D001318900F5F71C
:10AD6000AAFAE36B40F82350656D0023217D32463B
:10AD7000CDE902330331EB8AC9B2CDE900033B468A
:10AD8000286901F0ADFE012005B0BDE8F08342F076
:10AD900080020121FDF7FDFABA012B0102F0400209
:10ADA000AD0803F030037F081A4308F001034FEAAF
:10ADB00058081A434FEAC9034FEA590903F0080338
:10ADC0001A43B300760803F004031A4370E7D36A0A
:10ADD00003EBC1035F78FF070ED55F88AF420BD14D
:10ADE0005968A76D01352068FCF75CFD0D490246E6
:10ADF000384610F02FFD8BE701318142E7DB05215A
:10AE0000EFE70021F9E7DB6A03EBC50213F8353001
:10AE1000052B03D152880121FDF7BBFA013584E7E8
:10AE20002846A1E7518302082DE9F04188B0044685
:10AE30000D4607AE002940F0BD800121FDF757FE09
:10AE400007468DF8170078BB01462046FDF74FFEF8
:10AE5000C0B9012231462046FEF7A8F800220DF1C4
:10AE600017012046FEF7A2F804220F2102232046F4
:10AE7000FDF775FE00221146204608B0BDE8F041FE
:10AE8000FDF7B7BD3A4631462046FEF78FF89DF8EC
:10AE90001C20204601230421FDF761FE3A460121D2
:10AEA000A06DFDF7F2FAD9E7E36C626A013B02EBB1
:10AEB000C30032F8332040F202239A422BD14FF0E4
:10AEC000010847682046FDF778FD434632460DF1FC
:10AED0001701CDF800800795FFF7DCFB20462A46D6
:10AEE0002946FDF77FFE9DF8170006280DD007289C
:10AEF0000ED0052854D100953B46079A2946A06DEF
:10AF0000FDF744FC00220221B6E7CDF80080F3E70C
:10AF100002230093F0E72B46324620460791009526
:10AF200006A9FFF7B7FB2A460DF117012046FEF7E9
:10AF30003DF820462A462946FDF754FE9DF81800A4
:10AF4000831E012B08D9FDF721FD65680246A04943
:10AF5000A04806F0D5F928609DF8170006280BD008
:10AF6000072813D005281BD10799890141F4B8415E
:10AF7000A06DFDF71CFAC5E70799A06DC90041F067
:10AF80004201FDF714FA4FF4B541F1E70799A06DBE
:10AF9000C90041F08201FDF70AFA4FF4B141E7E739
:10AFA000FDF7F4FC656802468B498A4806F0A8F96B
:10AFB0002860A7E7012940F0FB80FDF798FD0746D0
:10AFC0008DF8150050BB01462046FDF790FD054663
:10AFD0008DF8180002212046FDF789FD05438DF804
:10AFE0001C0008D0394620460322FEF797FC0321B7
:10AFF0002046FDF7D5FC022306A920460122CDE913
:10B000000163002300930DF11503FEF711F80F21E2
:10B01000204608B0BDE8F041FDF7B4BDE36C626ABC
:10B02000013B02EBC30132F8332040F202239A4283
:10B030003ED12046D1F80480FDF7BFFC0223002258
:10B040000DF115010093CDE906232B4606AAFFF763
:10B0500021FB069F204632463B460DF11701009525
:10B06000FFF718FB9DF81700431E022B08D9FDF7C8
:10B070008DFC656802465949564806F041F928603A
:10B080009DF8150006280FD007280FD0052840F09E
:10B090008580002300933A4643460799A06DFDF74B
:10B0A000B5FB08B0BDE8F0810123F3E70223F1E727
:10B0B000022306AA0DF116012046079300930023F0
:10B0C0000695FFF7E7FA204600220DF11501FDF77E
:10B0D0006DFF9DF81600831E012B08D9FDF756FC65
:10B0E000656802463E493B4806F00AF92860069D1D
:10B0F0000023204632460DF117010095FFF7CAFAEA
:10B100009DF81700431E022B08D9FDF73FFC666827
:10B11000024632492F4806F0F3F830609DF81500DA
:10B1200006280ED0072825D0052837D1079941EAEF
:10B13000851141F4A841A06D08B0BDE8F041FDF7CC
:10B1400036B90126A06DAE4046F43441FDF72FF923
:10B15000A06D45EAC50141F04001FDF728F90799C6
:10B1600041EA851141F4A441A06DFDF720F946F4B0
:10B170003C41E0E70126A06DAE4046F43441FDF7C6
:10B1800016F9A06D45EAC50141F08001FDF70FF900
:10B19000079941EA851141F4A041E5E7FDF7F6FB87
:10B1A000646802460F490B4806F0AAF8206078E769
:10B1B0000025334606A901220095FDF705FF02236D
:10B1C0002A460F21204608B0BDE8F041FDF7C7BC74
:10B1D000C11F080874AF0808B81F0808CB1F08086B
:10B1E000DE1F0808D41F08082DE9F04116468046E6
:10B1F0005C200F461D46F5F75CF88660082604467D
:10B200000662C0E900874020F5F73AF8E66260621E
:10B210002020F5F735F860632020F5F74AF8294635
:10B22000A065FDF76AF82046BDE8F08110B5044638
:10B230000021806DFDF769F8A06DF5F749F8606BA6
:10B24000F5F746F8E069F5F743F8606AF5F740F876
:10B250002046BDE81040F5F73BB8000002F00F03B0
:10B26000022B10B5044608D00A460C490C4806F0DB
:10B2700047F8636A1860002010BD836A1209002035
:10B28000834204D1238C042BF5D10649EEE7E16A11
:10B2900051F820109142EFD00130F1E7E91F080882
:10B2A000E0AF0808F31F080870B50646B2B1900772
:10B2B00014D110792E2811D194687CB1A2070DD138
:10B2C0006568EAB2922A09D12D0A022D06D1A26838
:10B2D00001201A60049BE2681A6070BD0A460448A7
:10B2E000044906F00DF8736A18600020F5E700BF06
:10B2F000E0AF0808032008087FB504460D46104655
:10B3000003A91E46F8F778FD48B92A460B490C48B0
:10B3100005F0F6FF636A1860002004B070BD039862
:10B3200003F0EEFE30EA06020346F6D02A4605494F
:10B330000096034805F0E4FFECE700BF1920080879
:10B34000E0AF08081F200808038C032B70B5C46AFF
:10B3500003D1856A00239D4205D144F82120FDF7E1
:10B3600007F8012070BD54F82360964201D00133E4
:10B37000F1E70020F6E7FDF764B8032910B50446AD
:10B38000018442620FD1826A0021C06A92003DF0BE
:10B39000E3FE01212046FCF7C3FF20460021BDE863
:10B3A0001040FDF71CB8042914BF01210221F1E768
:10B3B00000F00F03022B02D10009F5F78ABE014805
:10B3C000704700BF3752080870B5054610460E4654
:10B3D000FFF7EEFF0378732B19D14378BBB1034617
:10B3E0000A22002013F8014F5CB91F2808D91F2337
:10B3F00032460A490A4805F083FF6B6A186000204C
:10B4000070BD303C092C02D802FB0040EAE732460E
:10B410000449034805F074FFEFE700BF3520080832
:10B42000E0AF080842200808F8B5194C0546104658
:10B430000E461F46FFF7BCFF00220178A446637842
:10B440008B421BD190F801E0A3789E4516D190F86D
:10B4500002E0E378734511D16BB91CF82200B842C1
:10B4600008D93B4632460B490B4805F049FF6B6A49
:10B4700018600020F8BDC378002BEED001320434F0
:10B48000152ADCD132460549034805F039FFEEE7BD
:10B49000B8A8080835200808E0AF08084B200808BD
:10B4A0002DE9F34706460F46002A3CD093073AD1D0
:10B4B00013792F2B37D1926802F00F03022B08D19A
:10B4C00001240F23FFF7B0FF8440204602B0BDE8FF
:10B4D000F08742B312F0030A25D113799F2B22D1B2
:10B4E000D5682B79A12B1ED14FF001090F2392684B
:10B4F000FFF79AFF01AA09FA00F4A22105F108005A
:10B50000F8F7C6FE8046C245DFDA019A0F233946B6
:10B51000304652F82A200AF1010AFFF785FF09FA9E
:10B5200000F00443EFE73A4603490448002405F0DD
:10B53000E7FE736A1860C8E751200808E0AF080802
:10B5400010B50446024805F045FE206010BD00BF5E
:10B55000E0AF080804292DE9F84380460C460DD8D1
:10B56000151F01F1300930264E450DD055F8040F56
:10B5700000F00F03022B0AD00D4900E00D49002412
:10B58000D8F82400FFF7DCFF2046BDE8F883000967
:10B59000F5F79FFD07463DF01DFE0228ECD13B78F4
:10B5A000722BE9D17B78B342E6D10136DCE700BFEC
:10B5B0008B200808622008082DE9F0470F4686B066
:10B5C00004461E4603A938469146F5F78EFD0378DA
:10B5D0000546762B40F01B81B9F1020F40F0C88080
:10B5E000A7F23D67102F00F20981DFE817F0110084
:10B5F00039003C00070107010701070107010701A6
:10B6000007018F00070161003F0034003100BE00D8
:10B610004EF6B4684FF42C69326829462046FFF78D
:10B62000D3FE0746726829462046FFF7CDFEFA0290
:10B6300049EA500902F470424001B90142EA0902A4
:10B6400000F0200001F04001024348EA010129E036
:10B650004EF6B168DEE74EF6B1684FF42469DBE7D9
:10B660004EF6B868D6E74EF6BD68D3E73068FFF708
:10B670009FFEA9493DF0BCFDC0B10F2332682946A9
:10B680002046FFF7D1FE07467068FFF791FEA349F9
:10B690003DF0AEFD002840F0B1803A034EF6F16176
:10B6A00042F421622046FCF78CFEE3E10F27EBE732
:10B6B0003068FFF77DFE03783268722B17D10F23B5
:10B6C00029462046FFF7B0FE294607467268204605
:10B6D000FFF77AFE4EF6106180464FEAC81241EA43
:10B6E0005801D2B242EA073242F42162DAE729462F
:10B6F0002046FFF769FE294680460F2372682046E0
:10B70000FFF792FE4FF46E410746E6E74EF690587B
:10B71000326829462046FFF757FE05AB0746294603
:10B720000093204604AB7268FFF7BEFD002800F0CE
:10B73000A1810723049A29462046FFF775FE059A42
:10B74000064629464FF47F732046FFF7D5FDFA02DF
:10B75000B90102F4704201F0400142EA900241EA6C
:10B76000080142F4206231439CE74EF68058CFE74F
:10B77000B9F1030F42D1DFF8BC81002700F1010AC3
:10B780000322414650463DF04BFD90BB2B7983BBD5
:10B79000634B29463268204613F82780FFF714FED2
:10B7A0007268074629462046FFF70EFEB2688146BA
:10B7B00029462046FFF708FE4FEA081308F0F00874
:10B7C000FA02DBB248F46E4802F47042B90143F465
:10B7D000206348EA590801F0400143EA5003400160
:10B7E00000F02000034313434FEAC912D2B21A43B8
:10B7F0002BE7013708F10408042FC1D14B462A4634
:10B800004849494805F07CFD636A186032E1B9F1A6
:10B81000030FF3D8DFE819F0040015001201C70286
:10B8200040F266539F4205D14FF43F412046FCF75A
:10B83000BEFD1FE140F251639F42DFD14BF63071F4
:10B84000F4E740F24542974210D101463268204663
:10B85000FFF704FD01462046FCF73BFE002840F0C0
:10B8600009813249606AFFF76BFE03E140F24F4203
:10B87000974209D1014632682046FFF7EFFC0146A6
:10B880002046FCF780FEE9E740F25942974209D191
:10B8900001460F2332682046FFF7C6FDC10041F480
:10B8A0008E41C3E7622B47D1039B032B0BD0052BA3
:10B8B00040F08780C3785F2B40F0838003796E2B44
:10B8C00001D0772B7DD169780022194B4FF0FF37DB
:10B8D0005878884205D195F802C09878844508BF09
:10B8E0001F78013203330E2AF2D17B1C86D03268D6
:10B8F00029462046FFF7B2FC039B0246052B09D1DF
:10B900002B79A3F177067342734139462046FCF741
:10B91000FEFDA3E70023F8E7A9200808B3200808E4
:10B9200018A80808C6200808E0AF0808D3200808AF
:10B930007CA8080819A80808692B42D14378742B01
:10B940003FD13068FFF734FDB84B017800221F4625
:10B950005E788E4222D190F801C09E78B4451DD108
:10B960008678DEB9AE1C31460B46013118780028C6
:10B97000FAD1691D8B423FF641AF02EB420208212A
:10B98000013BBF5CFA43F800D20008400A409E42E7
:10B9900009D941EA071141F43F4147E70132033336
:10B9A0000E2AD5D12AE713F801C94908BCF1740F52
:10B9B00001D10143EBE7BCF1650F7FF41FAF1143E9
:10B9C000E5E740F27D439F4202D14BF272612DE7E1
:10B9D00040F27E439F4202D14BF2626126E740F281
:10B9E00099539F4213D1326829462046FFF758FDEC
:10B9F00010F43F4F024607D145044ABFC1B240F49C
:10BA0000344141F4354111E74EF62D114AE6782FC5
:10BA10007FF4F4AE326829462046FFF741FD10F46A
:10BA2000FE4F024607D110044ABFD1B242F43C4156
:10BA300041F43D41FAE64EF6BD0133E6736803F08A
:10BA40000F03022B40F09E8040F257539F4214D1C7
:10BA500001460F2332682046FFF7E6FC074672686E
:10BA600029460F232046FFF7DFFC394602462046D1
:10BA7000FCF70BFD06B0BDE8F08740F26C439F4237
:10BA80001CD14FF6B0294FF280070F2332682946A8
:10BA90002046FFF7C9FC7268804629460F232046DE
:10BAA000FFF7C2FC47EA000249EA000142EA082225
:10BAB000F8E54FF690294FF2A007E6E740F2A353CE
:10BAC0009F42F6D040F25B539F422AD10C2332684A
:10BAD00001462046FFF7A8FC07467068FFF768FCA0
:10BAE0000146064652483DF083FB0346A0B131466D
:10BAF00050483DF07DFB70B12A464F494F4805F054
:10BB0000FFFB636A0022186042EA07224FF2EF311E
:10BB100042F40042C6E5012303EBC303484AD25C6A
:10BB2000F2E7B7F5876F15D14FF4804732682946A1
:10BB300007232046FFF778FC8046726829460723D2
:10BB40002046FFF771FC4246034639462046FCF783
:10BB500097FC8FE7DFF8F080002703224146284654
:10BB60003DF05EFB40B9EB7833B9364B13F82770E4
:10BB70003F0147F48047D9E7013708F104080F2F48
:10BB8000EBD13BE640F25A539F422CD840F2565339
:10BB90009F4220D840F26E439F423DD040F21E5358
:10BBA0009F4200F0888040F22B439F4237D040F202
:10BBB0001C539F4200F0DF8040F21D539F4200F073
:10BBC000DC8040F21F539F4200F0D980972F40F055
:10BBD0009F800323A2E0A7F5AB67022F22D8DFE8FE
:10BBE00007F04C354F0040F209639F4240F08C80D3
:10BBF0004FF460570723326829462046FFF714FCAC
:10BC000029468046FF2372682046FFF775FB47EA06
:10BC1000000141EA082109E64FF42057EAE74FF412
:10BC20004057E7E74FF40057E4E700BF7CA8080857
:10BC3000A7A80808B0A80808B9200808E0AF0808B5
:10BC4000A6A8080840A8080841A808084FF24028FC
:10BC50000F23326829462046FFF7E6FB07464FF6DA
:10BC6000FF73726829462046FFF746FB3A460346B3
:10BC700041462046FCF71BFCFCE64FF2C028E7E7F4
:10BC800001460F2332682046FFF7CEFB29460746C0
:10BC90004FF0FF3372682046FFF72EFB054683B254
:10BCA0003A464FF240212046FCF701FC3A462B0C65
:10BCB0004FF2C021DDE701460F2332682046FFF72F
:10BCC000B3FB05AB074629460093204604AB7268D8
:10BCD000FFF7EAFA00283FF4CDAE0F23049A294675
:10BCE0002046FFF7A1FB059A06462946FF2320467A
:10BCF000FFF702FB46F46841820841F0500142EA36
:10BD0000073242F47062CDE440F205639F4238D0BE
:10BD100040F207639F427FF471AD0523824A2946B2
:10BD2000204632F8237007233268FFF77DFB05AB0E
:10BD3000804629460093204604AB7268FFF7B4FAA8
:10BD400000283FF45BAD049A294607232046FFF7FD
:10BD50006BFBF9040646059A15D51F232946204694
:10BD6000FFF7CAFA47EA0807800147EAC60700F466
:10BD7000F86139435AE50023D0E70123CEE74B466B
:10BD8000CCE70423CAE73B0406D53E2329462046D8
:10BD9000FFF7B2FA4008E5E77C2329462046FFF783
:10BDA000ABFA8008DEE7B7F5A66F21D1002707239D
:10BDB000326829462046FFF737FB81460723726821
:10BDC0002946204647EA0907FFF72EFB2946804609
:10BDD0001F23B2682046FFF78FFA47EA801747EA29
:10BDE000C80123E54FF40067E1E74FF48057DEE731
:10BDF00040F231539F42F5D0B7F5886FF5D040F24D
:10BE00002B439F422BD14FF4C05807233268294659
:10BE10002046FFF709FB072372680746294620469C
:10BE2000FFF702FBB268814602F00F03022B0ED12E
:10BE3000072329462046FFF7F7FA47EAC90141EAF6
:10BE4000080141EA8011F1E44FF4D058DDE70723FF
:10BE50002946204648F48068FFF74EFAEDE740F2A5
:10BE6000D7539F4222D14FF690380F23326829468C
:10BE70002046FFF7D9FA0F238146726829462046EB
:10BE8000FFF7D2FAB268074629460F232046FFF78C
:10BE9000CBFA48EA070140EA092040F4704242F038
:10BEA000F002FFF7FFBB4FF6B038DEE740F22E633B
:10BEB0009F42F8D040F209639F42C5D040F206632A
:10BEC0009F427FF49BAC01460F2332682046FFF768
:10BED000ABFA0F237268294607462046FFF7A4FAFB
:10BEE00005AB804629460093204604ABB268FFF7B5
:10BEF000DBF900283FF4BEAD0F23049A2946204603
:10BF0000FFF792FA06463F02059A2946FF2320468C
:10BF100047EA0837FFF7F0F946F4684147EA90022C
:10BF200041F04001FFF7BEBB28A8080838B5054618
:10BF30003020F4F7A5F90446202200213DF00CF949
:10BF400029462046FCF7D9F9A562A800F4F798F92C
:10BF5000E062204638BD10B50446C06AF4F7B8F96F
:10BF600000212046FCF7D1F92046BDE81040F4F747
:10BF7000AFB92DE9F04F50EA010C85B0074688466D
:10BF8000DDF854B0DDE90F94DDE9136508D0904287
:10BF900071EB030304D31BF0040F13D001340136FB
:10BFA0001BF0020302933BD0002D39D012DB119B12
:10BFB0009D4235DA2E44B44202DC631EF31A12931A
:10BFC00000252DE00A22002352F0B8FB0135074678
:10BFD0008846E5E72B1D23DB6E424FF0000A0A225C
:10BFE00000233846414652F0A9FB1A4371D055440C
:10BFF0005646A41B761B4A462E21731E302502F896
:10C00000025B104689F80110194600296ADC002EEF
:10C010004FF000054FF0FF0608BF002302EB0309B5
:10C02000631E9A460393BAF1000F5FDA731CA342B2
:10C0300074DBFE2ED4BF00220122129B4C443BB184
:10C04000039B2E213020F61A129BF31A9E426CD1CC
:10C05000029B4BB142B123461C4613F8012D302AF6
:10C06000FAD02E2A08BF1C460BF001032B4329D01F
:10C070001BF0040F26D1002D0BF020034FF00A0215
:10C0800043F04503B8BF6D422370B4BF2D232B236B
:10C09000632D6370C9BF6423A11CE11CB5FBF3F3DE
:10C0A000B5FBF2F0C8BF303302FB1055C8BFA37018
:10C0B00030350C46B0FBF2F302FB1303303304F8C7
:10C0C000023B4D700E980023201A237005B0BDE886
:10C0D000F08F0AF1010A07468846B2457FF47FAF28
:10C0E000002586E7013900F8015B8EE756453846A2
:10C0F00041464FF00A02B4BF0AF10103CDF804A093
:10C100000AF1FF3AB8BF0193002352F017FB019BDD
:10C1100030328846074609F8032084E709F101090F
:10C120002E23012209F8063087E716B9012204F808
:10C13000011B013E04F8010B88E70000000000002D
:10C140002DE9F04F2DED068BB0EE408B8A469BB06B
:10C150001C4618EE901A9DF8A830129000292FDA8C
:10C16000B4EE400BF1EE10FA2AD6B1EE408B2D233F
:10C17000DDF848800AF1FF3A08F8013BB0EEC87BD1
:10C1800002F020039FED846BB4EE467BF1EE10FAD3
:10C190001BDD43F0490443F04E0008F1030243F075
:10C1A0004601002388F8010088F8004088F8021052
:10C1B0001370129BD01A1BB0BDEC068BBDE8F08F3C
:10C1C000002BD5D1DDF84880D8E7B4EE488BF1EEEE
:10C1D00010FA07D743F04E0143F0410008F1030283
:10C1E0000C46DEE742F02002662A57D143F00403F2
:10C1F000002CAAF10306099357DA0624A642334617
:10C20000A8BF23461093B5EE408BF1EE10FA5AD03A
:10C2100018EE903AB7EE009BC3F30A53B4EEC98B05
:10C22000A3F2FF33B0EE490B07EE103AF1EE10FA2D
:10C230009FED5B6BB8EEC77B4CBF0127002727EE55
:10C24000067B87F00109FDEEC77B17EE905A09EBDC
:10C25000050000F073FAB4EEC98BF1EE10FA4CBF92
:10C260004FF0FF3B4FF0010BB4EEC80BF1EE10FAAC
:10C2700094BF01230023BB421DD1099B5F074DD50D
:10C28000002D22DD631902339A451EDA099B83F0E3
:10C29000040343F002030993013443E0672A0CBF0F
:10C2A00043F0020343F00103A2E7632CA6D110235D
:10C2B00013241093A7E75D44B7EE000B09EB0500CC
:10C2C00000F03CFAD0E70025D7E7AAF10203A34229
:10C2D000C8BF2646002D1EDA022E15DDAC1C17DA6B
:10C2E0006F42B742A8BF3746023FF41B132C0DDD47
:10C2F000099AA4F11303132412F004020A921CD029
:10C3000004220A92032219E0741C00270023F7E795
:10C31000741C0027EAE76C1C3444FAE7099B980771
:10C32000BAD534B1132C4FF00007E1DC3B460A9735
:10C3300003E0274623460A9401240822AAEB040AB4
:10C34000AAEB020A9A455246A246A8BF1A46102CEA
:10C35000A8BF4FF0100A1792AAEB0503013B1193F7
:10C36000B5EE408B179BE318F1EE10FAA3EB0A032E
:10C37000159300F0E3800A9B002B00F0DB80002D7A
:10C3800080F2D58087B90AF1FF300C97CDF82C8068
:10C390001CE000BFAFF30080FFFFFFFFFFFFEF7F58
:10C3A000FF799F501344D33F434630212E2203F898
:10C3B000021B184688F801203A463CF0CDFE0346A1
:10C3C0000AEB07003B440B93FF230C930A22012343
:10C3D0000F9200220D929A4500F3B680BAF1100F29
:10C3E00040F3C080012840F3BD80BAF1110F00F086
:10C3F000B680022800F0B38002386426B0EE480B05
:10C400004FF0000B00F09AF9B6EE007B30EE077BA0
:10C4100051EC170B52F0C4F9099B00FB0BFB0F9A70
:10C42000CDE906530C9B06FB01BBA0FB06690593F7
:10C43000159BD944304604934946109BCDE902A38D
:10C440000B9BCDE900830D9BFFF793FD18AA0146D6
:10C450000E90404600F0A2F99DED189B39EE489BE6
:10C46000B5EE409BF1EE10FA5AD0BAF1100F4FF032
:10C470000102B0EE49ABC9BF0AEB4A039346303B19
:10C4800002FA03FB0C23CDE91369169319EE903AD7
:10C49000002B69DA16EB0B0649F10009099B4946A6
:10C4A0000F9A3046CDE906530C9B0593159B0493D8
:10C4B000109BCDE902A30B9BCDE900830D9BFFF7F9
:10C4C00058FD18AA01460E90404600F067F99DED10
:10C4D000189B39EE489BB5EE409BF1EE10FA1FD049
:10C4E000B0EEC97BB0EECA6B37EE467B17EE903AE2
:10C4F000002B3EDBB5EE407BF1EE10FA07D10A22AD
:10C5000000233046494652F019F91A4331D0BBF1A5
:10C51000010F33D0169B4FEA5B0B013B1693B5D14D
:10C520000E9B43449B46129BABEB030043E61198E2
:10C530000C952BE70A9B11980C9327E70023CDF865
:10C540002C8018460C9341E70D9A0A210F9E013367
:10C550004A43A6FB011632440F910D923BE7013886
:10C560000A264BE7012649E7B6EB0B0669F10009FD
:10C5700094E7B0EE49ABCDE91369C8E7119BA2453A
:10C5800003F10103119302DA0AF1010AE8E6DDE999
:10C590001332914508BF9E42C2D0099B0F9ACDE944
:10C5A00006530C9B0593159B0493109BCDE902A3A6
:10C5B0000B9BDDE91301CDE900830D9BFFF7D9FC4F
:10C5C0000E90ADE70129136810B522D90178302902
:10C5D0001FD14178841C41F02001782906D133F025
:10C5E000100314D110231360201A10BD6F2904D139
:10C5F00033F008030BD10823F5E7622904D133F0A7
:10C60000020304D10223EEE70BB9012313600446B1
:10C61000EAE7002BFBD10A23F8E70000044608B53F
:10C6200031B1054B4A6B03600023096804F0B4FE86
:10C630002046F3F7FDFD00BFE0AF08082DE9FF41FC
:10C6400004461F46461801922AB1023A222A02D90C
:10C65000374801F0D9FCB442254626D34FF00008F4
:10C66000711B284601AA0024FFF7ACFF0544019B7B
:10C670002846B04201462AD3B8F1000F00D06442E8
:10C68000640044F00104A94204D00D46B5422B4693
:10C6900042D348D0019A2749012A274808BF0022DF
:10C6A00004F02EFE3946FFF7B9FF14F8010BF5F739
:10C6B000EDFA80460028CED12B782B2B01D12546D0
:10C6C000CEE72D2BCAD125464FF00108C8E710F858
:10C6D00001CBACF13002092A0AD9BCF15F0FC8D0F6
:10C6E0004CF02002A2F1610CBCF1190FC4D8573AEA
:10C6F0009342C1D983FB0441B1EBE47F03D11444DD
:10C7000094EA4402B5D5711B424603A8039506F08E
:10C710001EF803990446B6E718780135F5F7B6FA1E
:10C720000028B3D1B6E7204604B0BDE8F08100BFD1
:10C73000DE200808F320080850AF080808B52DEDE2
:10C74000028BE8B1B5EE400BF1EE10FA18D010F103
:10C75000160F53EC102BC3F30A51014461F31E531F
:10C7600043EC182B0FD34342B1EE040B01EE103A09
:10C77000B8EEC11B3BF0CCFDB0EE407B88EE070B62
:10C78000BDEC028B08BD07EE900AB1EE040BB8EECB
:10C79000E71B3BF0BDFD28EE000BF1E700232DE980
:10C7A000F74F9C4600EB010E044601921F461A46C5
:10C7B000184619461D460093744577D2264616F84A
:10C7C000019BA9F13008B8F1090F57D8022D07D104
:10C7D000454CA74202DC0A2404FB07873446EBE7FA
:10C7E000B8F1000F25D0DFF80891DFF800A1484527
:10C7F00071EB0A041DD20A2412BB6246DFF8F090E6
:10C800003A4C4FF00A0C42BB484571EB040432D25B
:10C810004FF00A0C012DA0FB0C0408BF03F1FF33FD
:10C820000CFB014110EB080041F100014FF0000C3E
:10C83000D4E70DB90132D1E70CF1010C0125CDE7A8
:10C84000484502F1FF3271EB0A0B37BF04FB01FBD5
:10C850000133A0FB04015944CEE7484502F1FF3201
:10C8600071EB040A3FBF0CFB01FA03F1FF33A0FB9D
:10C870000C015144C7E78DBB0133D7E78DB9B9F13E
:10C880002E0FDBD049F02008B8F1650F0BD1B6456B
:10C8900003D965782B2D1BD1A61C764522D0022505
:10C8A0009CE7022DEED1B9F15F0F97D0009DBDB985
:10C8B0001A44174451F0BCFE41EC100B3846FFF708
:10C8C0003DFF019B83ED000B204603B0BDE8F08FD8
:10C8D0002D2DE4D1A61C01240094DEE79446ADE79B
:10C8E0007F42E5E70024EFE76466660699999919A7
:10C8F00098999999000000002DE9F04F2DED068BD5
:10C900009FED678B83B0054690461F46B0EE489B6F
:10C91000DDF8489046184FF0000A9FED63AB8DEDAF
:10C92000009BB5422C466DD34FF0000BA31C9E42DA
:10C9300040F28A80237843F02003692B74D1637816
:10C9400043F020036E2B7FD1A37843F02003662BA6
:10C950007AD1574B0022E01CCDE90023E31D9E4213
:10C960001AD9E37843F02003692B15D1237943F0DA
:10C9700020036E2B10D1637943F02003692B0BD178
:10C98000A37943F02003742B06D1E37943F020030D
:10C99000792B01D104F10800B8F1000F0FD0B0429B
:10C9A0000DD2037843F020036A2B08D1844203D1CF
:10C9B0000022404BCDE9002301304AF0020ABBF1CE
:10C9C000000F05D09DED007BB1EE477B8DED007B28
:10C9D000844240D00446B442254643D348D1BAF1FC
:10C9E000010F38D09DED000BBAF1000F4AD0B0EE28
:10C9F000401BB0EE480B03B0BDEC068BBDE8F04F1A
:10CA000003F0BCBB15F8010BF5F740F9834600288D
:10CA100087D123782B2B01D12C4687E72D2B83D16F
:10CA20002C464FF0010B81E76E2B0DD1637843F05C
:10CA30002003612B08D1A37843F020036E2B03D190
:10CA4000E01C8DED00ABA7E76A46311B2046FFF7DF
:10CA5000A5FE0028A0D11849184804F0BBFB4946A0
:10CA6000FFF7DCFD28780134F5F710F90028B2D182
:10CA7000002FF0D0BAF1000FEDD14FF0010A9DED7B
:10CA8000008B4CE717B19FED061BB4E703B0BDEC7C
:10CA9000068BBDE8F04F04F073BD00BFAFF300801C
:10CAA0000000000000000000000000000000F87F0F
:10CAB0000000F07F0000F03FFF20080850AF08089A
:10CAC00008B51020F3F7F5FB0123837008BD10B5FE
:10CAD00003F001030224C3708470C0E9011210BD89
:10CAE00070B51C1E11DD02F01F032344BFF34F8FEE
:10CAF000144E14461344C6F8684220341D1B002D02
:10CB0000F9DCBFF34F8FBFF36F8FBFF34F8FBFF3CE
:10CB10006F8F0C4B0024C3F85042BFF34F8FBFF30D
:10CB20006F8FBDF81430426003F00103079A8170E3
:10CB3000C370049B8360069B0373C36862F31F2367
:10CB4000C36070BD00ED00E070B504460D461046B0
:10CB50002388CBB10A460023214605F0C7F82346B7
:10CB6000002213F8011B1D1B090605F1FF3503D434
:10CB7000D30725D51C4B19E013F8011BC1F3801610
:10CB800006FA05F52A43EEE7A3786668042B0FD072
:10CB9000052B16D0032B0A46A36831461DD105F09C
:10CBA000A5F8124B0360E37853B1114B036007E023
:10CBB000A46810200F4902F0B7F9C660C0E901541B
:10CBC00070BD257B1020E4680B49C4F3172402F0E4
:10CBD000ABF9C0E90156C460F2E705F087F8E378E5
:10CBE000002BEDD0C6E700BF20B50808D8B3080871
:10CBF00004B50808C0B30808A8B3080838B5144637
:10CC000012F480721D4618BF1A46FFF79DFF620995
:10CC1000E1B202F008022A44BDE8384003F048BA05
:10CC2000D0E90003184770B505460C468E18B4428B
:10CC300000D170BDD5E90003984704F8010BF6E771
:10CC400038B504460025D4E90003984700F07F0377
:10CC500043EAC5150306F6D4284638BD2DE9F04150
:10CC600086B00546FFF7DCFFC4B2042C06D8284B7B
:10CC700053F82440204606B0BDE8F0812846FFF76F
:10CC8000DFFF064630B9062C04D12846214CFFF7B9
:10CC9000C7FFEFE70A2C10D10021304609F06EFFE4
:10CCA0000027044600F10408B742E3D028460137C4
:10CCB000FFF7D4FF48F8040FF6E7314602A8F4F76F
:10CCC000F1FA324604992846FFF7ADFF631F012BA6
:10CCD0000CD82846FFF7A4FF052C02A803D108F0C2
:10CCE0006FF80446C6E708F071F8FAE7072C4FF032
:10CCF0000003DDE9031003D10A22FFF79FFCF0E7F0
:10CD0000093C009362426241FFF7F6FDE9E700BF8C
:10CD10000CA90808FCBC08082DE9F84304460F4696
:10CD200090460025294E2068FFF77AFF5FFA80F9C8
:10CD3000B9F1FF0F01D1BDE8F883C1070CD5206818
:10CD4000FFF77EFFC2074FEA500548BFA3684FEACE
:10CD5000850554BFED19ED184FEA5903082B21D86A
:10CD6000DFE803F0050505050505171B1E00DB07B9
:10CD70000DD52068FFF764FF5FEA990923D0B9F168
:10CD8000010F0CBFA368E3680246294616E00120A4
:10CD9000F2E763689B680120F6E76368DB68FAE7FF
:10CDA0003346F8E703F18043084A093B52F8233041
:10CDB000F1E751F804CB9C4441F804CC013AF8D295
:10CDC00005EB8005AFE74346DEE700BF40A9080852
:10CDD0002DE9F04F8FB080460991FFF731FF00F049
:10CDE000030300F004099A1C0492C2080792002B66
:10CDF0003FD14FF0000A1046F3F742FA079A574620
:10CE00005446014606464046FFF70DFFCDF820A0E8
:10CE10005546CDF814A0B9F1000F00F098804046B7
:10CE20004FF0000BFFF70CFF049B8146032B08BF5C
:10CE300001308000F3F724FA0690CB457DD1FFF74F
:10CE40003FFE049B8346022B40F08C803246002339
:10CE500012F8011B901B090600F1FF307AD49BB237
:10CE6000069A31465846FFF732FE58460FB0BDE8E5
:10CE7000F08F0798F3F704FA079A014606464046F2
:10CE8000FFF7D1FE049B4046032B18D1FFF7D8FED5
:10CE9000044630180027335D411C0A1A1D0602F1B2
:10CEA000FF3204D44FF0000ACDF820A0B0E711F80B
:10CEB000013BC3F3801505FA02F21743EDE7FFF7D4
:10CEC000BFFE049B0746052B0BD140460024FFF70D
:10CED000B7FE08904046FFF7B3FE8246254605940C
:10CEE00099E710F0200B23D04046FFF7A9FE8246B9
:10CEF00017F0400002D04046FFF7A2FE1AEB0004F4
:10CF000018D0C51C25F003050AEB0500F3F7D1F98D
:10CF100005440590BBF1000F04D052462946404617
:10CF2000FFF781FE4FF0000A5446CDF820A072E7CB
:10CF3000DA46DDE7A2460894D0E709994046FFF7B4
:10CF400047FF069B43F82B000BF1010B75E7CDF86B
:10CF5000189074E712F8011BC1F3801404FA00F072
:10CF6000034377E7099BCDF82880CDE90B35059B76
:10CF70000D93FB0610D5154DD5F8D40020B9014608
:10CF800006F0A6F8C5F8D400314605F014FE324686
:10CF900031460AA8FFF7C0FE049B032B06D1344498
:10CFA000B9F1000F03D0069B43F82940069C089B6B
:10CFB000BFB23246049902935846079BCDF80CA0A5
:10CFC000CDE90047FFF78CFD4FE700BF004002208E
:10CFD0002DE9F047836886B004460F460493036842
:10CFE00002A83F490593F3F7E9F8042220460DEB28
:10CFF0000201FFF718FE9DF806509DF80420AB08CB
:10D000004D2A03F02F030CD19DF80520062A08D1E4
:10D010001BB105F00302032A03D19DF807201F2A44
:10D0200002D9304800F0F0FF23B1043B042B01D9B2
:10D030002D48F7E715F04005F3D12046FFF700FE35
:10D04000814620464FEA4906FFF7FAFD804603363F
:10D05000D7F800A000EB960026F003068000F3F757
:10D060000FF9CAF808003044CAF80C004D450DD13C
:10D070000025454539682AD12046FFF7A9FE78608A
:10D080000120F3F7A3F806B0BDE8F0872046FFF7CC
:10D09000D7FDC3074FEA500613D43046F3F7F0F834
:10D0A0003246014682462046FFF7BDFD2046FFF787
:10D0B000B7FD31465046F3F747FF06465046F3F7B3
:10D0C00007F93B689B6823F815600135CEE7CE6809
:10D0D0002046FFF7C3FD46F825000135C9E700BF2C
:10D0E00003D2020805210808112108081FB50C46C3
:10D0F000014601A819F0CAFE214601A8FFF768FF02
:10D1000004B010BD8268024B1A61C268DA607047D1
:10D11000004002208388024603F4C071B1F5C07F4D
:10D120000FD0190604D5C37B00EB8302106970474A
:10D1300013F4807006D0D37B02EB83021369586826
:10D1400070470148704700BFE584030870B5F3F7E6
:10D15000A1FE264C01230025E561A4F83C32D4F859
:10D1600040320BB1A4F83C52A4F8485203F0BAFF85
:10D170001F4B03211F4E2048A564C4F8305284F889
:10D180003452C4E910351D4BE36403F02FFD012137
:10D19000304603F02BFDAA22BA21304603F030FEC0
:10D1A000002125670846C4F8D450C4F8BC50C4E92F
:10D1B0000366C4E92D55C4E9715505F089FF0A21BC
:10D1C000C4F8500105F0F7FC40F2E261D4F85001D8
:10D1D00005F0F1FC002106F1440005F031FE40F2BB
:10D1E0001A7240F2DA63C4E9552370BD0040022090
:10D1F000B0B208086040022050400220D8C00808A1
:10D200007047D0E90230184708B5074B186F08B9C6
:10D21000064808BD002242F28A01043001F05EFC9B
:10D220000028F5D04068F4E700400220D0C7080885
:10D23000C000034B0A4640F00201D86803F0E0BD8D
:10D2400000400220C100034B41F00201D86803F006
:10D25000E5BD00BF00400220C000034B0A4640F07D
:10D260000201186903F0CCBD00400220C100034B4D
:10D2700041F00201186903F0D1BD00BF0040022057
:10D28000F8B51C46930707460E46154608D11368A5
:10D290009A88910615D5520610D5B3889B0501D5FD
:10D2A0002560F8BD50B9114B9E4207D010490C20A3
:10D2B00001F03AFEC0E901652060F2E7C4E90057D9
:10D2C000EFE70C4A934202D16B682360E9E70A4A10
:10D2D0009342E5D130B101F033FE084B834214BFD5
:10D2E00006463E466B68C4E90036DAE77CB80808B3
:10D2F00020A9080860C1080848C10808A8C1080892
:10D3000000232DE9F0410E4607461446C2E90033DA
:10D3100001F016FE0A2E054602D12060BDE8F0811C
:10D32000192E07D1838803F4C0731BB1144BC4E9D1
:10D330000037F3E76B7B5BB105EB83032246314695
:10D3400038461B6998476368042BE7D10023636064
:10D35000EB7C002BE2D005EB83030022F10018697F
:10D3600041F00201043001F0B9FB0028D6D0234679
:10D37000426829463846BDE8F041FFF781BF00BF4B
:10D3800044C70808F0B593B005460E4617466846F0
:10D390001C46F2F735FF40B93A4631462846FFF7BA
:10D3A000AFFFF2F703FF13B0F0BD002CFBD1019BE0
:10D3B000044918680AF0C6FB0028F4D10198F2F776
:10D3C00037FF00BF6CB1080808B519B903F0FDFEBE
:10D3D000F2F72EFF03F0FEFEFAE70EB403B503AA40
:10D3E00052F8041B019203F023FFF2F721FF000023
:10D3F00070B5C400114E05460022306944F00204A5
:10D400000430214601F06AFB0246A0B9306F30B10A
:10D410002146043001F062FB08B1406870BD002273
:10D420002146074801F05AFB024620B92A46054921
:10D430000548FFF7D2FF5068F0E700BF0040022028
:10D4400080C308081D21080870B008080A4B10B5F1
:10D450000446D3E90303984207D0E10000220430D8
:10D4600041F0020101F03AFB20B92046BDE810402E
:10D47000FFF7BEBF406810BD00400220032837B54B
:10D4800005460C4607D1084601F07AFF00B30E248A
:10D49000204603B030BDCA072FD54B1008282AD824
:10D4A00001A252F820F000BF91D40208D9D402089A
:10D4B000F7D40208F7D40208CDD40208F7D4020842
:10D4C00091D40208D5D4020891D40208002BDED0F2
:10D4D0001E24DDE7002BDBDAB3F1404F06D14FF01D
:10D4E000804003B0BDE8304005F00CB95B425B0002
:10D4F00043F00104CCE7DB43F9E7062825D101F02E
:10D500000703022B10D08B071FD10B681A7BE2B1E7
:10D5100003EB82031A69204B9A4216D1486840B93E
:10D520008B68C86801930CE0CC082046F3F7BAFD7D
:10D5300018B1400040F00104AAE701A92046F3F722
:10D54000D4FD0199F3F796FCF3E7204601F0F8FCCF
:10D55000C37ABBB100EB8300214603692846984794
:10D56000B0B9042DB4D0A5F10803022B12D90B4B8E
:10D5700020465D5D01F0F0FC094903462A46094852
:10D58000FFF72BFF062DECD1640044F001047FE788
:10D5900004467DE700247BE7C9550308FEC108085F
:10D5A0002921080898AF08082DE9F04105460E46E4
:10D5B0001746984601F0C4FC847A54B100EB840409
:10D5C00043463A46314624692846A446BDE8F04120
:10D5D0006047284601F0C0FC024902460248FFF7B6
:10D5E000FCFE00BF3221080898AF080800231A4645
:10D5F0001946FFF7D9BF0000F0B51546124A87B0AB
:10D600000C461169064602A80491D16805910F499C
:10D61000C2E90335F2F7D2FD224631466846376843
:10D62000F6F74AFEB4FA84F2684639465209F9F729
:10D63000F1FE044615B1FFF7D9FF04460120F2F7C9
:10D64000C5FD204607B0F0BD0040022005D102080C
:10D6500007B50022019101AB0121FFF7A5FF03B03F
:10D660005DF804FB07B5CDE900126B4600220221EC
:10D67000FFF79AFF03B05DF804FB30B45568144619
:10D68000003D18BF0125C5F1020302EB83030A46E2
:10D690002918206830BCFFF787BF000010B504468A
:10D6A00003F03CFE30B1002320461A461946FFF72E
:10D6B0007BFF0446204603F04BFE28B9034904488B
:10D6C000BDE8104003F086BD204610BD3821080893
:10D6D00098AF08087FB5C000104B059240F00200DB
:10D6E0000190186902900620CDE90301186F78B106
:10D6F000002242F2BA01043001F0F0F940B101AB6E
:10D70000002205214068FFF74FFF07B05DF804FBDA
:10D7100001A905200BF00CFBF7E700BF0040022039
:10D7200070B5164604460D46FFF7EAFD336893B917
:10D73000A30709D12268084B9A4205D12B46E288FB
:10D7400006490748FFF749FE204601F005FC2B4635
:10D7500002460449F5E770BDA8C108085921080828
:10D760006CB108086221080807B56A46FFF7D8FFC0
:10D77000DDE9000109B102F03BFC03B05DF804FBF8
:10D780002DE9FF41174606460C461D4601F0D8FB21
:10D79000374A904208D12B463A462146304604B0DB
:10D7A000BDE8F04104F064BB818811F4C07812D068
:10D7B000062C2DD100232F4F3B62FFF7ABFC034615
:10D7C000304698472860D8B93B6A002B18BF1C46E2
:10D7D0002C60002015E0062C1AD101AA1921304630
:10D7E000FFF78EFD019B7BB901AA8A213046FFF726
:10D7F00097FF039401AA00210120FFF73EFF286054
:10D80000012004B0BDE8F08101AA41464046F4E79A
:10D81000002CE9D1384601F093FB17490AF092F940
:10D8200001AA60B147213046FFF76AFD019B73B141
:10D8300001AA21462046FFF720FF2860C9E79B2167
:10D840003046FFF75DFD019B0BB10397D2E70B4913
:10D85000384603F091FD30B109490A4803F0BAFC9B
:10D8600028600220CDE73846FFF718FFF8E700BF31
:10D8700090B40808004002208CB2080820B20808C2
:10D880006A21080828B008087FB540F20E4102AAB4
:10D890000546FFF735FD029CDCB12046002401AAB5
:10D8A000694601F0D1FC009BA34201D804B070BDD1
:10D8B000019B53F82400013407F0DEFD06460146C3
:10D8C00002AA2846FFF72CFF02993046FFF7B0FC6A
:10D8D000E9E7284602AA40F21441FFF721FF029D22
:10D8E000AB68A342E2D9EB68E60053F8340080B19C
:10D8F00004280ED007F0D8FD03785F2B09D0EB6821
:10D9000053F8340007F0B8FDEB6833445968FFF76B
:10D910008FFC0134E4E7000073B505460C4616465B
:10D9200001F00EFB437B5BB104222146CDE90026CA
:10D9300000EB8302284613696A469847009B43B16F
:10D94000284601F009FB2346024603490348FFF736
:10D9500044FD02B070BD00BF622108086CB1080828
:10D9600073B50C46064601F0EBFA838805461906A6
:10D9700032D4C37BB3B14CB900EB83031A69174BA4
:10D980009A4203D01020F2F77BFC0446EB7B214641
:10D99000AA88304605EB8303D2051B6948BF1B6884
:10D9A000984778B96A460F213046FFF7A9FC009BDB
:10D9B00053B11CB91020F2F763FC044621466846B7
:10D9C00004F046FB02B070BD304601F0C5FA0449D0
:10D9D00002460448FFF701FD3046F3E7D16F030824
:10D9E0008121080898AF080837B5044601F0A8FA65
:10D9F000818811F4C0750AD0104B00221A62FFF71B
:10DA000089FB0346204603B0BDE8304018476A460C
:10DA100019212046FFF774FC009B3BB9204601F01A
:10DA20009BFA074902460748FFF7D7FC6A46294692
:10DA30002846FFF722FE03B030BD00BF00400220A1
:10DA40008E21080898AF080830B5054695B000F05B
:10DA500047FF284601F074FA848814F4C0740AD091
:10DA60001B4B00221A62FFF755FB0346284615B0F0
:10DA7000BDE8304018476A4619212846FFF740FCA8
:10DA8000009BE3B102A8F2F7BBFB014640B96A462E
:10DA9000FFF7F3FD0446F2F789FB204615B030BDD1
:10DAA000039B0C4918680AF04DF80346039823B10C
:10DAB00003F05CFB064B1862EFE7F2F7B9FB284670
:10DAC00001F04AFA044902460448FFF786FC00BF09
:10DAD0000040022020B208088E21080898AF0808EC
:10DAE0002DE9F04F13688DB004460293002857D1FA
:10DAF00002F10408C1F30729CFB24FEA490353FAF0
:10DB000081F158F821604FEA810B76105ED13546DD
:10DB1000BB0008EB870A039308EB8703009308EB2D
:10DB20000B034FF0000B0193019B9A4552D1D9444E
:10DB300007F1010A4FEA490B002E5FD10BEB0A05F2
:10DB4000A800F2F79DFB814614B1574601260460F8
:10DB50003C46039A414609EB86003BF0B9FAA344E0
:10DB6000AB4506D948464FEA8B01F2F7A4FB5D4668
:10DB700081462646DFF800A2DDE90032934240F0FC
:10DB80008A80321B21464B4602985208FFF70CFD53
:10DB900004464846F2F79CFB20460DB0BDE8F08FE6
:10DBA00002F108085468A5E726FA0AF3D80708D551
:10DBB00058F82A0001F0C6FB18B101F095FA0138B7
:10DBC00005440AF1010A5745EED1A1E74FF0000ADA
:10DBD0005546F8E7DAF800206AB9DAF8040050B1DF
:10DBE000810708D1026864498A4204D10BF1FF3BE6
:10DBF00003F003F983440AF1080A95E755445D44AC
:10DC0000A800F2F73DFB81460CB1046001244FF0FF
:10DC1000000A5745A3D026FA0AF358F82A00DA0773
:10DC200035D5830716D10368544A934202D0544A2B
:10DC300093420FD108AA07A901F006FB079A09EB46
:10DC40008400089992003BF043FA079B1C440AF1B8
:10DC5000010ADEE708A9FFF783FEA7EB0A0303909A
:10DC600004930398FFF7F0FE03460028EFD0049AD0
:10DC70002244954207D8E900484605936D00F2F723
:10DC80001AFB059B814649F824300134E9E749F83D
:10DC900024000134DBE7009BD3E9002B002A62D18A
:10DCA0001BF0030726D1DBF80030534522D1DBF807
:10DCB00008309F4203D3009B083300935CE7DBF8F6
:10DCC0000C304FEAC70853F8370088B104280FD04A
:10DCD00000F00703022B01D008F0E4FB49F826000E
:10DCE000B200DBF80C3002364A4443445B685360B0
:10DCF0000137DCE708AA6A215846FFF711FD002129
:10DD000008AA0846FFF7B9FC0021FFF729FE039097
:10DD10000398FFF799FE07460028CCD0731CAB424E
:10DD200007D34FEA45084846E900F2F7C4FA4546EA
:10DD3000814607F00703022B03D0384608F0B2FBF8
:10DD4000074608AA0F215846FFF7EAFC08AA002157
:10DD500001200A97FFF791FCB30049F826700236BC
:10DD60004B445860D4E7B30049F8262002364B44B0
:10DD7000C3F804B09FE700BF8CAE080814C10808C0
:10DD8000CCB60808830770B50C4686B015461BD183
:10DD900003681D4A934202D01C4A934214D102AA3E
:10DDA00001A901F051FA019BA34227D319D8029B84
:10DDB000043D03EB84049C4201D106B070BD54F8CD
:10DDC000042D45F8042FF6E702A9FFF7C9FD00234B
:10DDD00006469C423046019306D8FFF735FE0028E0
:10DDE000EBD022460A490BE0FFF72EFE019B28B13B
:10DDF000E21A0133013A45F82200EAE7019A05499F
:10DE00000548FFF7EAFA00BF14C10808CCB60808B5
:10DE1000B12108089C21080850AF08082DE9FF41EE
:10DE200083071546CFB2C1F3072436D10368384AB9
:10DE3000934202D0374A93422FD1029003AA02980C
:10DE400001A901F001FA01983B1983425AD80399BC
:10DE5000002601EB8003A64214D1C01B01EB870111
:10DE6000BC00801B05EB860805F032F90399424699
:10DE700045F826000B198B420AD10023029304B007
:10DE8000BDE8F08153F8042D45F826200136E2E77D
:10DE900053F8040D42F8040FEDE70021FFF760FD91
:10DEA000002380469F42019317D80021084605F0C1
:10DEB0000FF906464046FFF7C7FD0146C0B9B368F3
:10DEC000A3421FD305EB840245F8246005EB8301D0
:10DED000AA4211D11B1BB360D1E74046FFF7B4FD46
:10DEE000019B78B1FA1A0133224445F82200D9E7A0
:10DEF000304604F060FEDDE7881AF768385842F8CB
:10DF0000040DE5E7019A04490448FFF766FA00BFEB
:10DF100014C10808CCB608089C21080850AF0808AE
:10DF20002DE9F04F85B005460C4600AF07F1080219
:10DF3000FFF7E6F9D7E9020129B102F059F81437E1
:10DF4000BD46BDE8F08F0028F9D107F108024FF473
:10DF500083612846FFF7D4F9BB6823B922461E49DE
:10DF60001E48FFF73AFA07F1080228461721FFF783
:10DF7000C7F9391DB86807F005FB82462046F3F75C
:10DF80009DF8D7F80490514609F101064A468519D3
:10DF9000EB1D23F00703ADEB030D6B4668466E44A3
:10DFA0004FEAD30B3BF094F82E23204609F83B3080
:10DFB000F3F78FF881462046F3F780F8494602468A
:10DFC00030463BF085F829466846F2F7BDFF01224E
:10DFD0001E21FFF77FFBB2E7CB21080824B1080818
:10DFE00008B50446F2F778FA18B104490448FFF777
:10DFF000EBF9224603490248FFF7EFF9D12108085F
:10E0000094B00808F82108080146024808B5FFF74F
:10E01000DBF900BF50AF0808831E2DE9F043054629
:10E0200087B088461746062B3BD8DFE803F0093A4D
:10E030003A093A040F00B94212D04FF00E09EBE052
:10E040003A4607B0BDE8F04301F0C2B9384603F0E4
:10E0500065F940B13946404603F08EF90028ECD00E
:10E060004FF01E09D8E017F0030440F0FF803A6833
:10E07000A34B9A4240F0FA8007F104097B68A3425F
:10E08000DBD959F8046F304603F048F9002800F056
:10E090005F813146404603F06FF90028E0D101343A
:10E0A000ECE711F0010F00F0FE804E10F90740F18F
:10E0B000CD807C10232800F2D980DFE800F0B1B5D4
:10E0C000D7B9BDD7D7D7D7121D20233D46484AD749
:10E0D00050586A72121D20233D46484AD750586A4C
:10E0E000729346EA040090EA40034FEA400900F1C7
:10E0F000A78049F001098FE086EA0400F3E706EA09
:10E100000400F0E7002C02DA7E48FFF77DFF1F2CA9
:10E1100009DC6FF040432341B34204DB4FF040433E
:10E120002341B34205DD3046F11704F0DBFA8046A7
:10E13000BFE006FA04F0D6E7002CE5DB1F2C2046F2
:10E14000A8BF1F2046FA00F0CDE73019CBE7301BFF
:10E15000C9E786FB0404B4EBE07FC4D0E3E7002CFE
:10E1600000F0F880214630460DF0BEFFBBE7002CE2
:10E1700000F0F08007EE906AB8EEE70B07EE904AE9
:10E18000B8EEE77B80EE070B07B0BDE8F04303F085
:10E19000F7B9002C00F0DE80214630460DF096FFE6
:10E1A000A1E7002C1BDA07EE906A3946B8EEE70BC0
:10E1B00007B0BDE8F04303F053BA33460120E2074D
:10E1C00006D580FB0302B2EBE07FACD1012C8AD0F4
:10E1D00083FB03326410B2EBE37FF0D0A3E7ECD112
:10E1E000012080E7002C00F0B5800021022008F01B
:10E1F000C5FC2146814630460DF076FF21464000A1
:10E2000040F00100C9F8080030460DF05FFF400003
:10E2100040F00100C9F80C00484607B0BDE8F083A3
:10E22000A642FFF61DAF08E7A6423FF719AF04E785
:10E23000A6427FF715AF00E7A642BFF611AFFCE696
:10E24000C11707B0BDE8F04304F04CBABB072AD1B0
:10E250003B682D4A934219D107EE906A3946B8EED1
:10E26000E70B03F0FDF981460028D5D1274B404646
:10E270005D5D00F071FE0446384600F06DFE2A46F2
:10E280000090234622492348FFF7A7F8224A9342E9
:10E2900009D107EE906A39469FED171BB8EEE70BE0
:10E2A00002F04AF8DFE7062D03D143462425B8469D
:10E2B0001F46404600F044FE037B33B9A5F1090335
:10E2C0000C2B0DD80D35EDB2F3E700EB83003A4689
:10E2D000414603692846984781460028EED09BE7CF
:10E2E000A5F116030C2B19D843460F35B846EDB2ED
:10E2F0001F46DEE7AFF300800000000000000000D2
:10E3000014C108082622080834B30808CCC108083C
:10E310003B22080898AF0808A0AC0808242D04D9AF
:10E3200043460F3DB846EDB21F46242D9ED102A9AB
:10E330004046FFF715FB04462046FFF785FB002803
:10E340003FF47BAE394601F0BBF80028F4D087E6F5
:10E3500037468BE701490248FFF736F84E22080896
:10E36000B4B108080146024808B5FFF72DF800BF10
:10E3700098AF08082DE9F041044617461E460D46A1
:10E3800041B1186800F0DCFD6368834202D00548A3
:10E39000FFF7E8FF33463A462946A068BDE8F0415A
:10E3A000FFF702B95A2208080146024808B5FFF7EC
:10E3B0000BF800BF04B0080807B5002201AB0191BB
:10E3C000012102F023FEF1F733FF0000014603486C
:10E3D00008B509B9FEF7F8FFFFF7EEFF20B208080D
:10E3E00008B500F0B9FD024902460248FEF7F5FF04
:10E3F0006422080898AF08084100034841F0010171
:10E4000008B5FFF7D9FF00BF4CB0080842F6D2119B
:10E41000014808B5FFF7D0FF28B0080830B593B021
:10E4200004460D466846F1F7EBFE48B920462946FA
:10E43000FFF70EF90446F1F7B9FE204613B030BDE0
:10E4400001990024014800F0B5FDF6E7949E080804
:10E45000054BD861B3F83C2212B2012A02D1002246
:10E46000A3F83C22704700BF00400220EFF3108168
:10E4700072B6084AB2F83C321B0408D5B2F83C32F6
:10E48000013B1BB2A2F83C3281F3108870474FF673
:10E49000FF73F7E700400220EFF3108172B60C4BD8
:10E4A000B3F83C22013212B2A3F83C2252B9DA6925
:10E4B0002AB9D3F8402212B993F848222AB100228F
:10E4C000A3F83C2281F3108870470122F8E700BFCF
:10E4D0000040022070B5EFF3108572B60F4B93F831
:10E4E0004822082A18D0B3F83C4224B2012C02D1A9
:10E4F0000024A3F83C4293F84942561C224483F876
:10E50000486202F007022B3203EBC203C3E90101A8
:10E51000012085F3108870BD0020FAE7004002203A
:10E520000228F8B503462C4C10D0E26972B1EFF323
:10E53000108272B6E06938B10021012BE16103D18C
:10E5400082F31088F1F774FE82F31088B4F83C323D
:10E550001BB243B9EFF3108272B6B4F83C6236B224
:10E5600016B182F31088F8BD4FF6FF73D4F84472E9
:10E57000A4F83C3297B1D4F840526B68C4F84032EA
:10E580000BB9C4F844322B682E6082F310882846F9
:10E590009847EFF3108272B6AF42ECD194F848522C
:10E5A000BDB194F84932013D03F12B01013384F8E8
:10E5B000485204EBC10103F00703D1E9010184F8DB
:10E5C000493282F31088FFF729FFBDE8F840FFF7D2
:10E5D00063BF82F31088F8E7004002200120FFF7B4
:10E5E0009FBF08B5FFF7FAFF30BF08BD08B5FFF7BA
:10E5F000F5FF30BF08BD000038B1044A13699842E6
:10E6000002D0106118467047002070470040022079
:10E6100001F00F0108290DD8DFE801F011050A0CFF
:10E620000C0C0C0C0E0000280CBF0E201E20704796
:10E6300004F068B804F081B8C00040F002007047F0
:10E6400000F0AEBD08B500F0ABFDB7EEC00B08BDE5
:10E6500002F096BFB7EEC00A02F092BFF0B593B0D9
:10E6600005460F46144668461668F1F7C9FD78B9A5
:10E67000002E2346324628460CBF39460021FFF7BC
:10E680007FF80546F1F792FD012D0CD1284612E0E6
:10E69000019B23601049206802F06EFE034620684B
:10E6A0005BB9F1F7C5FD2368002DF3D10BB9062343
:10E6B000236036B9002013B0F0BD02F057FD206092
:10E6C000F7E70649304602F057FE0028F2D0304600
:10E6D000FEF7E4FFE5E700BF20B208088CB20808A7
:10E6E000036803B94068FFF7AFB91346C1F30722C7
:10E6F000C9B2FEF759BF1FB501F00F030446012B45
:10E700000CD011F00E0F0BD0023B012B0AD90122C5
:10E7100001A900F01DFF50B1019801E000F030FEAA
:10E7200004B010BD04B0BDE8104000F0E9BC2046C4
:10E7300000F0E6FCF4E708B528B1062803D0FEF7A0
:10E74000ADFFF1F775FD08BD10B50C4619B9BDE870
:10E750001040FFF705B9FFF703F984421CBF0023FF
:10E76000C4E90030002010BD40F29553984217D8FC
:10E7700040F29153984209D85E281DD075281DD0CB
:10E780003E2814BF4FF0FF3001207047A0F2935095
:10E79000022815D8DFE800F00C0E020005207047B3
:10E7A00040F22F63984214BF4FF0FF3003207047B0
:10E7B00006207047072070470220704700207047EE
:10E7C0000420704738B5034614460D4661B152B176
:10E7D00011462846984760B16B683BB96C6045F0BC
:10E7E0000103AC60E3602C46204638BDAB68DC60BA
:10E7F000F5E76368EB606560002BF5D144F0010339
:10E80000A560EB60F0E7F8B5064631B1002511F0E0
:10E81000010304D000232946EB600846F8BDCC680C
:10E82000CB6014F0010307D1E7682246E36030466D
:10E83000FFF7C8FF3C4601460A4630462946FFF727
:10E84000C1FF21460546E2E78A4284462DE9F041B0
:10E850000F4606D100235168BDE8F0415360FFF731
:10E86000D2BFD66896B11446E468E307FCD524F01D
:10E87000010406F0010851686368934216D1002331
:10E8800039B9984518BF1E466660D1603846BDE864
:10E89000F08160465360D360FFF7B5FF05466060C6
:10E8A000EE60B8F1000FF1D0A560EFE71D46DB6820
:10E8B0009342FBD1002260465A60DA60FFF7A3FF63
:10E8C0000028EDD0E8600546EAE7000082B0034B7F
:10E8D000186801ABC01A02B0704700BF00400220A8
:10E8E00007B5064A01A9136852685B1A9A4201D813
:10E8F000FFF78CFD03B05DF804FB00BF0040022071
:10E900000346500C10B51446C2F34F0221B1E10783
:10E9100002D40C48FFF726FD904206D198420FD052
:10E92000024609490948FEF758FD984204D9C21A1F
:10E9300007490648FEF751FD9A4201D20549F1E721
:10E9400010BD00BF6B2208087522080898AF0808A0
:10E95000872208088F2208082DE9F74F0024064671
:10E960008B461546A046A1460193DDE90CA7019B05
:10E970009C4204D1B1453CD22248FFF7F3FCB4429B
:10E9800010D2BAF802209205F6D409F101095BF819
:10E9900024009AF80220012A24D100F0F1FC07F8A3
:10E9A000240017E0BAF8001000222846C90041F000
:10E9B000020100F093F888B9BAF80220D30505D512
:10E9C000BAF8002010491148FEF707FDDAF80420D4
:10E9D00047F8242001340AF1080AC8E708F10108C1
:10E9E0004068D6E7022A01D100F07EFB47F82400F8
:10E9F000F0E72B68B8EBD30F01D20548BDE703B0B1
:10EA0000BDE8F08FAD220808A822080898AF0808D2
:10EA1000B722080870B586B00446154602EB80029E
:10EA200003A81E4600F031F80B9B03AA2946019368
:10EA300020460A9B00933346FFF78EFF06B070BD59
:10EA4000014808B5FFF7B0FCC12208080346074992
:10EA5000002231F8020B984206D20132222AF8D164
:10EA600003EB530343F00100704700BF9CAA080862
:10EA700010B50446416019B90123A160236010BD9F
:10EA8000C800F1F716FC0146F6E74160C900826054
:10EA900041F007010160704703789B0710B50446F9
:10EAA00002D48068F1F714FC0022236862F3DF03CC
:10EAB0006260236010BD03789B0710B5044602D442
:10EAC0008068F1F705FC236803F0040343F00103B9
:10EAD00023600023C4E9013310BD0000022A2DE9A0
:10EAE000F04F044685B00E46904612D0426882B17F
:10EAF000C1F38601904B0B4493F84A32B3FBF2F119
:10EB000002FB1133826802EBC30552F83330B34283
:10EB100013D0237813F00102019213D006F00702FC
:10EB2000022A0FD016F0030203D1306883498842CD
:10EB300007D0B8F1010F05D00025284605B0BDE883
:10EB4000F08F01925B076AD52768A56827F0070751
:10EB50002F44BD4232D3B8F1010FEDD1D4E90032D8
:10EB6000B2EBD30FC3F3DC0111D10431A0686160B3
:10EB7000C900F1F7A0FB0021A060D4E90032A2EBAC
:10EB8000D30223F00703D20018443AF0E5FA2368D1
:10EB9000A168C3F3DC02501C01EBC20560F3DF0384
:10EBA000236041F8326006F007060022022E6A60F8
:10EBB000C3D0237862F300032370BEE72868B04215
:10EBC00024D1B8F1020F17D123687A1BD5F804803D
:10EBD00005F10801083B083A284623603AF0A8FAF4
:10EBE0002568A3680021C5F3DC0225F007051D4454
:10EBF00043F83210C5F804804F4BC6F386061E4416
:10EC0000A368EB1ADB1086F84A3296E7019B23B91A
:10EC1000314600F055FC0028D3D1083599E76368E8
:10EC20002BB9B8F1010F87D1204600F089F806F022
:10EC3000070BBBF1020F2CD1F008F2F733FA814633
:10EC400063680025B9FBF3F203FB129A5746A268EA
:10EC5000FB0052F83700029302EBC70300BBB8F188
:10EC6000010F7FF469AF2268002D18BF2B46BBF15E
:10EC7000020FC2F3DC0101F1010161F3DF02226046
:10EC8000C3E9006003D0227860F3000222701D46C1
:10EC900053E731460620FEF7F1FB4FEA6009CFE764
:10ECA00004281AD1002D08BF1D4601376368B7FB41
:10ECB000F3F203FB1277BA45C9D1B8F1010F7FF423
:10ECC0003BAF002D33D023680022BBF1020F03F1CC
:10ECD000080323602E606A606AE7B04218D1B8F179
:10ECE000020F0ED12168606808392160791CB1FBE0
:10ECF000F0F500FB1511A06850F83110A9B9F80023
:10ED00001150C6F386060C4A164486F84A72BEE7CE
:10ED100001990029C9D13146CDE9023200F0D0FB7A
:10ED2000DDE902320028C0D0D9E70421E7E7204618
:10ED300000F006F884E700BF00400220CCBF0808BE
:10ED40002DE9F041466804464FF00008701CFFF7BB
:10ED50007DFE0546C000A768F1F7ABFA2368656041
:10ED60003D1D03F00603A06043F001032360B0459E
:10ED700004D13846BDE8F041F1F7AABA55F8041CB1
:10ED800039B1042905D001222046FFF7A7FE2B68E0
:10ED9000436008F101080835E9E7002310B504468F
:10EDA000016043608800F1F784FAA06010BD036839
:10EDB0002DE9F74F04460F46934623B912F0010F91
:10EDC00065D000F067F839460620FEF757FB4FEA9A
:10EDD000600A23684FF00008BAFBF3F603FB16A69F
:10EDE0003546A168AA0051F8259001EB8503B9F1D9
:10EDF000000F0CD11BF0010F49D06268B8F1000F71
:10EE000018BF4346013262601F60B94633E0B9F172
:10EE1000040F17D1B8F1000F08BF984601352368D9
:10EE2000B5FBF3F203FB1255AE42DAD11BF0010F32
:10EE30002DD0B8F1000F26D0636801336360C8F8A5
:10EE40000070E2E739464846019200F039FB019A2A
:10EE50000028E3D01BF0020F0DD063682068013B4F
:10EE6000A16863606B1CB3FBF0F400FB143351F832
:10EE7000233023B98B50484603B0BDE8F08F0423FC
:10EE800041F82530F7E7204600F004F8A1E74FF0FD
:10EE90000009F0E7F8B50768044600258668781C85
:10EEA000FFF7D4FD656020608000F1F702FAA060F2
:10EEB000BD4204D13046BDE8F840F1F709BA56F832
:10EEC000251029B1042903D001222046FFF76FFF46
:10EED0000135EDE702460168002370B5994201D182
:10EEE000002015E094689E0054F8230001330028A8
:10EEF000F4D00428F2D05568013D5560B3FBF1F21F
:10EF000001FB123354F82330002B18BF0423A35104
:10EF100070BD10B504468068F1F7DAF90023C4E942
:10EF20000033A36010BD704710B50C46F1F7A8F987
:10EF3000046010BD10B50C46F1F7B0F9046010BDC7
:10EF400083070FBF006800F00F00024B53F820004A
:10EF5000704700BFE0AA080808B5FFF7F1FFC088B6
:10EF6000BDE80840F2F7B5B870B50D460446164640
:10EF7000FFF7B6FC2846FFF7E3FF437A43B100EB07
:10EF800083033246294620461B69BDE87040184776
:10EF9000C28820460249BDE87040F2F729BE00BF92
:10EFA000E62208080A4601460148FFF7DDBF00BF18
:10EFB00040CF0808F7B5044608460E4602F0C8F9E7
:10EFC00070B101AA6946304602F024FA009B3BB1B9
:10EFD00016492046F2F75FFA009D033D002D0BDA3B
:10EFE000314620460222FFF7BFFF1149204603B0F9
:10EFF000BDE8F040F2F74FBA019A20460D49AF0044
:10F0000002EB850352F825205B68F2F7F1FD019BC6
:10F010003B449A6822B906492046F2F73CFADCE7FD
:10F0200005492046F2F7E4FDD7E700BFEB220808C8
:10F030009F5408080F2308082423080808B502462F
:10F04000FFF77EFF837A53B100EB830306491B6908
:10F050008B4204D11046BDE8084008F047BD181E99
:10F0600018BF012008BD00BF0D790308830710B544
:10F07000044603D10268084B9A4208D02146082072
:10F08000FEF7FCF910B92046FFF7AAF9044620461E
:10F09000BDE8104003F0C8BCB4B508080E2838B568
:10F0A00003460C4604D1002323600125284638BDC1
:10F0B0001E2801D10123F7E710F0010501D043100C
:10F0C000F2E7820707D10168064A914203D103F0B3
:10F0D0005DFB2060E9E719460820FEF7CFF900281C
:10F0E000F5D1E3E7B4B5080813B501A90446FFF765
:10F0F000D5FF10B92046FFF773F9019802B010BD93
:10F10000C20705D4830705D10268034B9A4201D197
:10F1100003F035BBFFF7E8BFB4B5080800000000F6
:10F120000E2838B503460C4629D01E282AD010F0E8
:10F13000010508D0431000EE103AB8EEC00B0125CF
:10F1400084ED000B19E081070CD1026812498A4254
:10F1500002D103F081FCF2E710498A4202D102F0A9
:10F160007BFAECE719460920FEF788F928B18207F7
:10F1700003D10268094B9A42F1D0284638BD9FED71
:10F18000040BDCE7B7EE000BD9E700BFAFF300805C
:10F190000000000000000000B4B5080834B30808FF
:10F1A00013B569460446FFF7BBFF38B92046FFF7A1
:10F1B000D3FE044902460448FEF70FF99DED000B0B
:10F1C00002B010BD2D23080898AF0808F8B5044612
:10F1D0000F461646FFF7A4FF054630B10022002374
:10F1E000C6E9002301252846F8BDA10709D12268F8
:10F1F0000B4B9A4205D132463946204601F090F831
:10F20000F0E721460A20FEF739F90028EBD0820703
:10F21000E9D10268024B9A42E5D132463946EDE720
:10F22000A0AC080810B50446FFF7D0FF38B9204657
:10F23000FFF792FE024902460248FEF7CEF810BDE3
:10F240003823080898AF0808830710B50FD1036862
:10F250000A4CA34204D1436808300B60106010BD13
:10F26000074CA34203D18368C0680B60F6E7FFF741
:10F2700073FE044902460448FEF7AFF814C10808BB
:10F28000CCB608083F23080898AF080813B50C4609
:10F2900001A9FFF7D9FF019BA34204D022460349ED
:10F2A0000348FEF79AF802B010BD00BF48230808D3
:10F2B00050AF0808F7B51F46D30706460D4614465B
:10F2C0000DD5541001940198002823DA2844B7B1D1
:10F2D00000281DDBA84228BF284603B0F0BD01A9C5
:10F2E0001046FFF7DBFE0028EDD1F5882046FFF73A
:10F2F00033FE0A4903462A460948FEF76EF80028FD
:10F3000001DBA842E9D3F28806490748FEF765F811
:10F310000020E2E7002FDDD1F3E700BF5A23080801
:10F3200098AF080871230808DCB00808820701D0EC
:10F3300003F0E8B9002801DA03F0FFB9400040F01B
:10F34000010070478307014610B508D102680B4BD6
:10F350009A4204D18068400040F0010010BD084688
:10F36000FFF7EEFDC37A33B100EB8300BDE8104038
:10F370000369052018471846F0E700BF9CBF08083E
:10F380000E2810B5044620D01E281CD006281CD0FC
:10F39000C20703D5013818BF01200EE0FFF7D0FDEA
:10F3A000C37A5BB100EB83002146036904209847D0
:10F3B00020B1A0F11E035842584110BD2046FFF76E
:10F3C000C1FF0138E7E70120F7E70020F5E700007B
:10F3D00005282DE9F04707BF4FF00E084FF01E0932
:10F3E0004FF01E084FF00E09914207460C46154695
:10F3F00007D1C8075FD40846FFF7A2FD83885907E5
:10F4000059D504F00703022B05D0A20717D12268B3
:10F410002A4B9A4213D105F00703022B05D0AB0704
:10F4200012D12A68254B9A420ED12946204605F072
:10F43000DCFF00283FD14B461846BDE8F08714F0AA
:10F44000010623D0EE07F6D401262846FFF778FD03
:10F45000027B82465AB38188080704D42046FFF70E
:10F460006FFD824523D1052F14D09AF80C30224627
:10F47000294602200AEB83031B6998470346B0B173
:10F48000022FD9D0FFF77CFFD3E701262B46254674
:10F490001C46DAE7CB06E8D50AEB82022946384655
:10F4A00013692246984703460028DED0C4E7002EA1
:10F4B000EBD0AC42BFD14346BEE700BFCCBF08088B
:10F4C0000A460146022008B5FFF782FFBDE8084062
:10F4D000FFF756BF10B50446FFF734FF38B9204692
:10F4E000FFF73AFD024902460248FDF776FF10BDDC
:10F4F0007823080898AF080838B50446FFF720FDC0
:10F50000837B15462BB100EB8300036920469847A7
:10F51000A0B9204635B9FFF71FFD09490246094841
:10F52000FDF75BFF042D04D1FFF716FD06490246E7
:10F53000F5E7FFF711FD05490246F0E738BD00BFCA
:10F540008523080898AF080898230808AA23080804
:10F5500038B50546FFF7F4FC037C14461BB914F0DC
:10F5600004000BD138BD00EB830302F003022846F0
:10F570001B6998470028F2D10120F3E70148FEF704
:10F58000F1FE00BFB5230808042803D0052807D0E2
:10F59000002070478B68002B0CBF0E201E20704788
:10F5A0008868400040F00100704700000346084AA8
:10F5B0000846C1E900230022C1E902221968054A70
:10F5C000914202BF5B68C3F317238360704700BF9B
:10F5D00028AB080874AB0808F8B50D460179044655
:10F5E000164601F07F010022402008F08BFFA26840
:10F5F000E368424327682B606A60227902F07F014A
:10F60000A96009498F4201D00020F8BD110601D43C
:10F61000B20706D46268C2F3172200FB02332B60E4
:10F62000F2E70120F1E700BF74AB0808F8B500224B
:10F6300005460E460146402008F064FF07461020AC
:10F64000F0F71EFE094A0A4B04460571012D08BF5A
:10F6500013460360436803F0FF03C0E9013606FB6D
:10F6600007F0F0F70DFEE0602046F8BDB4AB0808E7
:10F6700040AB08084268C36891688B4230B40AD234
:10F6800014795D1CD1688268C56004F07F001A445B
:10F6900030BC08F0ABBF002030BC70474368FF2B84
:10F6A00070B504460E461AD800220179402008F0B1
:10F6B00029FFA168054608314143E068F0F7FBFDEA
:10F6C00063680822E060002162F31F23C5EBC502D6
:10F6D0006360A36803FB0553184439F03DFD3346CE
:10F6E0002079D4E9022109F0AFF9A368062001339B
:10F6F000A3606368A3F58073636070BD70B50E7915
:10F7000005460C46012E0ED11949F1F7C4FE3346C9
:10F710002846D4E9022105F005F928461549BDE837
:10F720007040F1F7B8BE32461349F2F761FAA368A8
:10F73000002BF2D0002611492846F1F7ACFEA36851
:10F74000B34204D80E492846F1F7A5FEE5E71EB1FD
:10F750000C492846F1F79FFE3246E16820790136D0
:10F7600008F044FF012201462846FFF7FDFBE6E7CB
:10F77000C3230808766F0808CF230808DA2308088F
:10F78000EF420808DE2308082DE9F04F044689B04F
:10F790000D4616460AB90025DEE011F00307806821
:10F7A000DFF848A240F0ED800B68884A934240F0B1
:10F7B000E88002AA08F010FB10B98548FEF7F4FDB6
:10F7C0002179042E3A464FF0400001F07F0100F00D
:10F7D000A48008F097FE16F00302054663D1316855
:10F7E0008B7B002B50D001EB83031869794B984237
:10F7F0004AD13179402001F07F0108F083FEA84210
:10F8000002D07548FEF700FC33685345D6E9029BE9
:10F8100046D17368C3F3172805FB08F82268E76828
:10F820005245DDE90203A3EB0003A9EB03063CD13B
:10F8300094F90420002AAEDA002EE2D16268C2F305
:10F84000172205FB027705FB09F20BEB080105FB0C
:10F850000070019339F06CFC0399A2680298521A67
:10F8600005FB017148446A4305FB007039F060FCF8
:10F87000019BA0680021A3EB090230446A4305FB09
:10F88000007039F069FC3BE0544B99420BD1012DDB
:10F89000B7D1052205A93046FFF75AFEDDE905B9C3
:10F8A0004FF00008BAE74E4888E7002ECBDD6368CA
:10F8B000B6EB132F2FD9A168384631446943F0F7CE
:10F8C000FAFC63688246BB4508BF834666F31F2384
:10F8D000E06063600298A26848440399324401FBE7
:10F8E00005A1121A05FB00A06A4339F021FC029819
:10F8F00005FB09F20BEB080100FB05A039F018FC31
:10F900006368C6EB132262F31F236360A36833446A
:10F91000A360062520E0BA46DCE708F0F3FD226884
:10F920000646029B52451BD1B3F1807F03DB2D4974
:10F930002D48FDF749FD1020F0F7A2FC054694E89C
:10F940000F0085E80F00029A02EB112363F31F21D9
:10F950006960039B9B1AAB60284609B0BDE8F08F35
:10F9600003992079C91AFFF761FEE1680546C0686E
:10F97000DDE90232D21A06FB0311724339F0A8FB0B
:10F98000EAE700232A4601462068FFF793FC236834
:10F990000246207953450ED16368042E02EB1322F0
:10F9A0000BD003067FF5F7AE3346E16800F07F0029
:10F9B00009F04AF8ADE7042EF6D1E16800F07F00C7
:10F9C00009B0BDE8F04F08F011BE00BFC4BC080884
:10F9D000E123080889F70208052408089CBF0808E5
:10F9E000202408083B240808D8B1080874AB08088C
:10F9F00001282DE9F043074685B00E4608D08B0755
:10FA000024D10B68254A934202D0254A93421DD146
:10FA1000012201A93046FFF79BFDB8B1002239460B
:10FA2000402008F06FFD029E0546B6FBF0F6384612
:10FA30003146FFF7FBFD06FB05F204460199C0685D
:10FA400039F046FB204605B0BDE8F0833046FFF7AD
:10FA500079FC054600B1451029463846FFF7E6FD1A
:10FA6000002104463046FDF77BFF4FF000080646B4
:10FA70003046FDF7E9FF03460028E3D025B91946D3
:10FA80002046FFF70BFEF3E708F101094246E16863
:10FA90003846C84608F0D8FFEAE700BF9CBF080810
:10FAA000B4AB080838B50C46114606221D46204660
:10FAB000FEF726FF2CB921460120BDE83840FFF7AC
:10FAC000B5BD2968CA0705D48B0708D10B680C4A55
:10FAD00093420DD10846FFF707FB0146ECE701F022
:10FAE0000703022B07D1012C05D10648FEF73AFC8B
:10FAF000054A9342F6E70120BDE83840FFF778BF9A
:10FB0000B4B5080850240808CCBF080838B50D461D
:10FB10001C461146094A2846FEF7F2FE206805F009
:10FB2000C3FC012D007804D10021BDE83840FFF767
:10FB30007DBD6168BDE83840FFF75ABF0400020090
:10FB4000F0B50F4685B00446012201A93846FFF7FB
:10FB5000FFFC014678B93846FDF702FF0546284606
:10FB6000FDF772FF014610B9062005B0F0BD204632
:10FB7000FFF794FDF3E700222179402008F0C2FC52
:10FB8000029D63680646B5FBF0F5B5EB132FC3F392
:10FB900017221ED9A16829444143E068F0F78BFB86
:10FBA0006368BC42E06003F0FF03636004D1052298
:10FBB00001A92046FFF7CCFC05FB06F20199D4E928
:10FBC000020300FB063039F083FAA3682B44A360DC
:10FBD000CAE7521B62F31F236360EDE71B28F0B5F1
:10FBE00006468DB00C46154626D005D804286BD99C
:10FBF0000E2850D000244BE02428FBD1012203A979
:10FC00002846FFF7A5FC00284ED0A1075AD122684C
:10FC1000474B9A4256D1012209A92046FFF7DCFC46
:10FC20000123DDE909010093DDE9032304F040FF2E
:10FC3000002847D01E242BE00A683E4B9A42D9D0B8
:10FC4000012206A92046FFF7C7FC052209A928467C
:10FC5000FFF77EFC9DF8207000224020394608F016
:10FC600051FC0A9EA1680546B6FBF0F638463144C1
:10FC7000FFF7DCFC079F044606993A46C06839F056
:10FC800027FAE06806FB05F20999384439F020FAB2
:10FC900020460DB0F0BD0A68264B9A42AAD02946EC
:10FCA0002046FFF74DFFF3E7EA0702D50020FEF7F5
:10FCB0007BFBAB0706D12B681F4A9342F6D01F4A45
:10FCC0009342F3D00E24E3E7012206A92046FFF772
:10FCD00083FC012209A92846FFF73AFC0028F1D04D
:10FCE000089A012A1DD05A2A1DDC203201460B9B9E
:10FCF000012B1AD05A2B01DC203301469342D5D177
:10FD000023F00203642BD1D0022E01D00029CDD0E4
:10FD10000A9B30460093099BDDE9061208F09BF828
:10FD200086E74222E1E70021E1E74223E4E700BF62
:10FD3000B4AB080874AB0808B4B5080834B30808B5
:10FD400070B50646102014460D46F0F799FA054A9C
:10FD5000067102604268C46002F0FF02C0E901253A
:10FD600070BD00BF74AB08087FB51D46084611463C
:10FD70004FF00212FEF7C4FD052201A92868FFF723
:10FD8000E7FB9DF80C40029E00222146402008F02F
:10FD9000B9FB019AB6FBF0F12046FFF7D1FF04460C
:10FDA0002868FFF7CDF80D4B834209D12A686168B6
:10FDB0005368C3F3172363F31F216160D368E360C3
:10FDC000032201A92868FFF7C3FB18B1237963F068
:10FDD0007F032371204604B070BD00BF74AB0808D8
:10FDE00070B505460E4601460120FFF71FFC04468C
:10FDF0002A463146C06839F06BF9204670BD0000D4
:10FE000038B505460C4610200349FFF78DF801224E
:10FE1000C460C0E9012538BDB4AB0808136870B5EB
:10FE20006BB94468A51C50F825509C4207D055F882
:10FE30002360B14204D1023350F82330136070BD07
:10FE40000133F2E72DE9F041164600250F4611492E
:10FE500006F104080446F1F71EFB7368AB4205D8AF
:10FE600020460D49BDE8F041F1F715BB1DB10B4926
:10FE70002046F1F710FB57F82520204608490135A8
:10FE8000F1F7B6FE012258F8041F2046FFF76CF880
:10FE9000E3E700BF67260808766F0808DE23080836
:10FEA000642408084B680A46023351F82310FFF710
:10FEB000C9BF0E3918BF0121490041F00101FEF709
:10FEC000ABB8052807D00E3918BF0121490041F011
:10FED0000101FDF7D3BA002070470000032A05D1C5
:10FEE0000E2914BF04490549F1F7D5BA0E2914BFEC
:10FEF00003490449F8E700BF7C1B0808811B080878
:10FF00002C0408085AF7070838B50C461146022297
:10FF10001D462046FEF7F4FC1CB12868FFF730FAB6
:10FF200008B90E2038BD1E20FCE7062801BFD1E924
:10FF300001305840400040F0010018BF00207047D9
:10FF400002280AD188689368984208D148685368A3
:10FF500098420CBF1E200E207047002070470E20D4
:10FF60007047136813B94068FDF7CAB970472DE9A7
:10FF7000F84F984602EB430300AF82465D1C042B0A
:10FF80008B4616464FEA85051FD8EB1D4FF000093A
:10FF900023F00703ADEB030D6C4620462A1FB96A18
:10FFA00040F804BB39F094F823464246711C504691
:10FFB000FDF7FAFA0446B9F1000F02D04846F0F70F
:10FFC00087F92046BD46BDE8F88F2846F0F763F96B
:10FFD00004460028D9D08146DFE707B500931346D1
:10FFE0000A46D0E90101FFF7C2FF03B05DF804FB48
:10FFF00038B505460C460C200249FEF795FFC0E9CE
:020000040803EF
:10000000015438BD38AC080810B504460249082030
:10001000FEF78AFF446010BD5CAC08082DE9F04F84
:100020008668044601EB420987B006EB010A0F46D9
:10003000154698460AEB420004F10C0B4FEA890979
:10004000052816D801AFB60059463246384639F071
:100050003FF84A464146B81939F03AF860683B46DD
:100060002A465146FDF7A0FA0446204607B0BDE8EF
:10007000F08F8000F0F704F9A26859460646920016
:1000800039F026F8A0684A46414606EB800039F070
:100090001FF8A16833462A4639446068FDF784FAA0
:1000A00004463046F0F714F9DFE74068FDF728B959
:1000B0002DE9F041CD1C174680460E46AD0008499B
:1000C0002846FEF731FF0446A5F10C023946C0E987
:1000D00001860C3038F0FCFF2046BDE8F08100BFFF
:1000E00070AC080891ED027B73B5B5EE407B044619
:1000F0000D46F1EE10FA24D01349F1F7CCF94FF088
:10010000FF3363206721114ECDE9003000232046E4
:100110001A4695ED020BF1F753FB02224FF0FF3325
:1001200063212046CDE900310023672195ED040BC2
:10013000F1F746FB3146204602B0BDE87040F1F7CA
:10014000AAB90022024EE9E76726080868240808D1
:100150006B240808136810B514463BB9B1F5B76FA6
:1001600005D190ED020B01F00BFA206010BD40F2BA
:10017000FB439942FAD190ED040BF4E708B52DED5D
:10018000048BB0EE409B0649B0EE418B1820FEF781
:10019000CBFE80ED029B80ED048BBDEC048B08BD93
:1001A000A0AC080808B5072841D8DFE800F01326FE
:1001B00040400440153291ED027BB5EE407BF1EEFC
:1001C00010FA36D191ED047BB5EE407BF1EE10FADA
:1001D0002FD10E21084608BD91ED047BFDEEC77BB3
:1001E00017EE903A91ED027BBDEEC77B17EE102A19
:1001F00053405B0043F00101ECE791ED041B91EDEE
:10020000020BBDE80840B1EE411BB1EE400BFFF719
:10021000B5BF91ED040B91ED027B20EE000BA7EE34
:10022000070B38F051FFBDE8084001F0A9B90021E3
:10023000D0E71E21CEE7000030B50C46114604225F
:100240001D4620462DED048B87B0FEF759FBF4B117
:10025000012C286826D082074DD102682E4B9A4285
:1002600049D190ED028B90ED049B6868830749D1DA
:100270000268294B9A4245D190ED047B90ED021B18
:1002800038EE478B39EE011BB0EE480B03E09FEDD3
:10029000201BB0EE410B07B0BDEC048BBDE8304035
:1002A000FFF76CBF00F007020346022A05D0810762
:1002B00016D1026819498A420FD104A905F062F9E2
:1002C00000230499009301231A46FCF715FB03460B
:1002D000184607B0BDEC048B30BD0F498A42F7D0F9
:1002E00004AA02A9FEF79EFF9DED041B9DED020BE3
:1002F000FFF744FFEBE7FEF753FFB0EE408B9FEDB7
:10030000049BB2E7FEF74CFF30EE091BBCE700BFD1
:100310000000000000000000A0AC0808CCBF0808E6
:1003200030B5D0E90245C1E90045D0E90401C2E990
:10033000000130BD0000000010B52DED088B84B029
:1003400004460846B0EE40AB02AA6946B0EE418BC7
:10035000FEF73CFF002800F0CB80A01E202800F212
:10036000CB80DFE800F0B5C9C9C9C9C9C9C9C9C9C5
:10037000C9C911205BC9292CC968C9C9C9C9C91112
:10038000205BC9292CC968009DED009B9DED027B77
:100390003AEE099B38EE078BB0EE481BB0EE490BE6
:1003A000FFF7ECFEA4E09DED009B9DED027B3AEE95
:1003B000499B38EE478BEFE75348FDF7D3FF9DEDA0
:1003C000027B9DED006BB5EE407BF1EE10FAB5EED1
:1003D000406B0BD1F1EE10FA03D14C494C48FCF7BD
:1003E000F3FF8AEE069B88EE068BD5E7F1EE10FA56
:1003F00006D1B1EE4AAB88EE079B8AEE078BCBE7BE
:1004000027EE075BB1EE477BA6EE065B86EE054B5B
:1004100087EE056B8DED004B8DED026B9DED007B46
:100420009DED026B28EE469B27EE088BA7EE0A9BFC
:10043000A6EE0A8BB0E728EE080BAAEE0A0B38F0FE
:1004400043FEB5EE400B9DED02BBF1EE10FA18D164
:10045000B5EE40BBF1EE10FA11D19DED007BB5EE8B
:10046000C07BF1EE10FA0ADBB5EE407BB7EE009BE5
:10047000F1EE10FA9FED227B09FE079B8CE72549E0
:10048000ACE737F055FDB0EE4A1BB0EE409BB0EE46
:10049000480B36F0BDFDB0EE408B2BEE400B9DEDD2
:1004A000007B27EE088BA7EE090B37F029FAA9EE9F
:1004B0000B8BB0EE40ABB0EE480B36F091FE20EE69
:1004C0000A9BB0EE480B38F0ABFA20EE0A8B63E7DC
:1004D0009DED007BB4EE4A7BF1EE10FA0ED19DED5E
:1004E000027BB4EE487BF1EE10FA0CBF1E200E200A
:1004F00004B0BDEC088B10BD0020F9E70E20F7E733
:1005000000000000000000006D2408088224080894
:10051000B4B108088F2408080B46114693ED041B5C
:1005200093ED020BFFF708BFD0E902120346C8683B
:1005300082420AD00869496850F8220001328A4292
:10054000DA6003D10022DA607047002070470000B3
:100550000346084603499A6801600349C260C0E93E
:10056000011370472CB908082905030870B5C56840
:1005700042686B1C466984689A4208BF0023F607EC
:1005800005D5A34203D108490848FCF71DFF0669B9
:10059000A34246F82510C36004D101339A4208BF34
:1005A00000238360062070BD522B0808DCB00808C9
:1005B000836810B553B14469013BC268E40707D5AD
:1005C000934205D108490948FCF7FEFE4368F2E76B
:1005D00004699342836044F8231003D103B943684C
:1005E000013BC360062010BD522B0808DCB0080890
:1005F00030B585B0054608466946FDF7B1F90446B1
:100600002046FDF721FA014610B9062005B030BD9D
:100610002846FFF7ABFFF3E770B504460E461546D4
:10062000C2B10068D4E90223991A324644BF636814
:10063000C9180023FEF73EFEA3681844636883428E
:1006400098BFC01A042D23691ABF43F8205006250D
:1006500053F82050284670BDF8B50F461E46114687
:100660000446134A3846FEF74BF97068FEF73CFD26
:10067000051E02DA0020FDF7C7FC21461820FEF710
:1006800053FC00230446681CC4E902336060800008
:10069000EFF70FFE022F206103D9B068FEF724FDAB
:1006A000606131682046FFF7A3FF2046F8BD00BF18
:1006B0000600040008B5D0E902239A4203D1074995
:1006C0000748FCF781FE03B94368013B026900213A
:1006D000C36052F8230042F8231008BD9C24080888
:1006E000DCB00808042803D0052808D00020704793
:1006F000D1E9020398420CBF0E201E207047D1E9B9
:100700000230C01A44BF4B68C018400040F00100DE
:1007100070470000D0E9023102468B4210B503D188
:1007200008490948FCF750FE0169002451F82300EC
:1007300041F82340013351688B4208BF2346936040
:1007400010BD00BF9C240808DCB00808042803D0B2
:10075000052807D0002070474B68082B34BF0E20B7
:100760001E2070474868C0F3DC00400040F00100E4
:10077000704700000346054A08460A601A7A0A7163
:100780005B688B600023CB60704700BFF4AD080846
:10079000062802D10B7A022B02D04968FFF7D6BF98
:1007A000490041F001007047044B886008460B6027
:1007B00001230B710023CB60704700BFF4AD080824
:1007C00010B5044904460C20FEF7AEFB022244603B
:1007D000027210BD0CAE080808B503799B0702D55C
:1007E0000020FDF7BFFD08BDF8B506460D460F68B1
:1007F000144612B13846FFF7EFFF22466968381DEC
:10080000FEF76CF9034608B1406870B9022E05D1B5
:10081000022C08D169680748FDF7CEFDA868012CB5
:1008200000D15860F8BD0620F9E7022C04BF002271
:100830005A60F7E7B8B008080122FFF7D5BF0222D7
:10084000FFF7D2BF0022FFF7CFBF10B50446FFF776
:10085000C3FF201DFEF72FF9062010BD30B502465C
:1008600085680B68AB4201D300200AE0D46804EB32
:10087000C30054F833400133002CF3D0042CF1D0E2
:100880000B6030BD13B5044600F10C018068FFF722
:10089000E5FF60B12379012B0BD0022B43680AD00E
:1008A000026869460220CDE9002306F067F902B02C
:1008B00010BD0068FBE71846F9E700007FB5174B4D
:1008C00004460A7A0D46012653F82210F0F7E3FD9C
:1008D00013492046F0F7DFFD124B00932B7A8DF879
:1008E00004306B680293002303936846FFF7CAFF46
:1008F000054630B90C49204604B0BDE87040F0F719
:10090000CABD1EB909492046F0F7C5FD0122294696
:1009100020460026FEF728FBE7E700BFE8AD080801
:100920009F240808F4AD0808A2240808DE2308085C
:100930001FB50446FFF750FF6368072B03D8114922
:100940001148FCF741FD002220460192227951070F
:1009500001A942BFC3F3DC0303F1FF330193FFF7A7
:100960007DFF6368042202A9083B63600368029369
:10097000436803930023C0E90023022006F0FEF839
:1009800004B010BDA5240808B8B008082DE9F74F39
:10099000032A0B68DFF8EC9015461EBFDFF8E8B0BD
:1009A0000125DFF8E8A00446884608BFD0E902AB7D
:1009B0004B4505D0032D03D0DA882C49F1F718F9FF
:1009C0002B492046F0F767FD01270023019301A979
:1009D0004046FFF743FF064680B926492046F0F718
:1009E0005AFDD8F800304B453CD0032D3AD022496F
:1009F000204603B0BDE8F04FF0F74DBD1FB951469A
:100A00002046F0F748FD032D2AD1336803F0070292
:100A1000022A25D013F0030708D11B681A7B2AB1DC
:100A200003EB82031A69154B9A4204D0012714493B
:100A30002046F0F730FD2A4631682046FEF794FA4A
:100A40001FB10F492046F0F726FD59462046F0F722
:100A500022FD2A46716820460027FEF785FAB6E790
:100A60000027E8E703B0BDE8F08F00BFBE24080808
:100A7000C224080860200808766F0808C9550308D2
:100A8000792E08088CAE08083A5F0808DE230808AB
:100A900010B5044904460C20FEF746FA00224460D3
:100AA000027210BD0CAE080810B5044904460C20B3
:100AB000FEF73AFA01224460027210BD0CAE08083B
:100AC00010F003030CD10268117A31B102EB8102FC
:100AD0001369044A9A1A5342534103F001007047C4
:100AE0000023FAE7150C03082DE9F3470C681646B6
:100AF00007460D462046FFF76FFE3168314A3846FB
:100B0000C908FDF7FDFE022F12D16F683846FFF7C6
:100B1000D7FF0146E8B12B689F4209D0002304F1BA
:100B20000408019301A96868FFF798FE074640B9D9
:100B3000002504347368AB4233D8062002B0BDE808
:100B4000F087012239684046FDF7C8FF7B684360A3
:100B5000E8E7384604F1040AFCF702FF81464846FC
:100B6000FCF772FF0028E3D00021FCF7F9FE804675
:100B7000FCF76AFF07464046FCF766FF054640461D
:100B8000FCF762FF17B91048FDF73EFA002DFAD0C6
:100B90000028F8D1012239465046FDF79FFF4560F5
:100BA000DDE7B36853F8351003EBC50739B1042905
:100BB00005D001222046FDF791FF7B684360013597
:100BC000B8E700BF05000200C424080810B50022E1
:100BD00004300C46FDF782FF18B921460248FDF7A4
:100BE000EBFB406810BD00BFB8B00808024B40F8EE
:100BF000043BFDF73DBF00BF8CAE080838B5054685
:100C00001020EFF73DFB04462946FFF7EFFF204693
:100C100038BD00002DE9F041804686B000200D4629
:100C200016461F46FFF7EAFF0F4B0446C0F8008048
:100C3000984502BF037943F00403037155EA0603A4
:100C40000DD03B6807EB85023146019003A8029363
:100C5000FDF71BFF03AA01A9681CFFF745FF20460B
:100C600006B0BDE8F08100BFBCAE0808F8B50C4680
:100C7000064600216068FCF773FE022E0546606898
:100C80008CBFA6680626FEF75DFB50B9FFF7B6FFDE
:100C90000446071D2846FCF7D7FE014618B9204632
:100CA000F8BD4010F2E701223846FDF717FF466015
:100CB000F0E738B504468068FFF7A0FF05462368D3
:100CC00062680360237922F0070203F005031343EF
:100CD0004360A268E168D200C06838F0F9F928469C
:100CE00038BD00001628F0B50C4685B0154663D017
:100CF00005D8022810D0092862D0002409E0242851
:100D0000FBD100222946201DFDF7E8FE00282ED148
:100D10000E24204605B0F0BD02F003038A0728D157
:100D20000A682B498A4224D1002BF1D129689142CB
:100D300021D1CDE9013301A92046FFF78FFD0746F8
:100D400002A92846FFF78AFD064677B10028DFD0C2
:100D500031683868FEF7B4FB0028D9D0716878682C
:100D6000FEF7AEFB0028E6D1D2E70028D0D11E2442
:100D7000CFE7002BCCD12A68164B9A42C8D16368C2
:100D80006A685340072BC3D800230435029302A995
:100D90002046FFF763FD06460028E8D000223168B0
:100DA0002846FDF79BFE0028B2D041687068FEF728
:100DB00087FB0028EBD1ABE70846FFF77AFF044634
:100DC000054A02A90220CDE90245FFF78DFEA0E702
:100DD000BCAE08088CAE0808F4AE080810B40C7A53
:100DE000012C06D1242804D149685DF8044BFFF793
:100DF00079BF00205DF8044B70474068C008704719
:100E000070B504460E461546FFF7E6FC0122314652
:100E1000201DFDF763FE4560204670BD022213B51C
:100E20000446CDE9000169461046FFF7DDFC204687
:100E300002B010BD38B50C461AB9FFF7EFFF062017
:100E40000BE0042A0AD100220430FDF747FE18B94E
:100E500021460448FDF7B0FA406838BDFFF7D0FFDF
:100E6000EDE700BFB8B0080813B504464068FCF7CA
:100E7000EBFD58B1A36869465A1C5B0043F00103BF
:100E8000A260CDE90030022005F078FE02B010BD6E
:100E90001FB50446084611461A4602AB01930A4B99
:100EA00000930223FDF7B6FD21460C20FEF73CF827
:100EB000044600210298FCF753FD039B6060204626
:100EC000A36004B010BD00BF00AF0808C3685A6833
:100ED000012A70B506462AD19D68AB0727D12A683A
:100EE000154B9A4223D1EC682378FF2B20D14A205E
:100EF000EFF7D1F9044638B9104AD2F83832343B0A
:100F0000492B12D9D46B3434E9682046F0F756F9EE
:100F10002046EC6038F05EF90023A8606B60A96899
:100F20002046EFF7A7FF686001E0054BF36070BD56
:100F30006B68002BFBD1F2E7CCBF08080040022011
:100F4000D8C00808F8B5164602F07F0705460C46DB
:100F500032060AD47B1E012B0DD80B68D888F0F717
:100F6000B8F801462846F0F796FA022F03D1234934
:100F70002846F0F790FA2046FFF7A8FF16F07D0705
:100F800034D1E3680BB15A682AB928461C49BDE838
:100F9000F840F0F780BA20681A4988421FD1022A27
:100FA0001DD89868C3071AD509F0DAFB0346B0B11B
:100FB000E2682846144992685210F0F719FEE36877
:100FC0005B68012B19D90D492846F0F764FAE368EC
:100FD0003A46D9682846BDE8F840FDF7C5BFE36842
:100FE0005A68012A02D100229968F3E73246E16883
:100FF0002846BDE8F84005F047BDF8BD3A5F08084F
:10100000375208084CB00808FA2408082DE9F843BC
:101010000D46044611461A4F1A4A28469846FDF7CF
:101020006FFC1020EFF737F90023002814BF81462A
:10103000B946C9F80040C9F808302DB9124C4846E5
:10104000C9F80C40BDE8F883AE1CB6003046EFF797
:1010500022F9044640B9D7F80C2206F118032C3FB8
:101060009A42EBDBFC6B1834084BA6F108024146B0
:1010700004F10800C4E9003538F02AF8DFE700BFC2
:101080002C400220FEFF0100D8C0080814C1080847
:10109000F8B515460F460446D0E901325119994278
:1010A0000FD30178D9B105F110060122C0681E44A2
:1010B0003146EFF70BF978B96568A368013D2070F8
:1010C000ED1A2A463946D4E90230184438F000F8BF
:1010D000A3682B44A360F8BD6660E060F1E7013BC4
:1010E0009D1AEEE7024B0022C3F83822DA637047FC
:1010F0000040022010B5FDF7F7FF041E11DDEFF7E9
:10110000BFF80346084AD06BEFF3108172B6C2F8FD
:101110003842D36381F3108808B1EFF7D9F806207D
:1011200010BD0023EEE700BF0040022038B50546A1
:10113000FDF706FF007A70B12846FDF701FF04466F
:101140002846FDF7FDFE037A04EB8304024B206979
:10115000C31A5842584138BD0D10030810B5044653
:10116000FFF7E4FF00B92469204610BD10B5FFF772
:10117000F5FFC36804465B6823B1FFF7A7FEE36889
:10118000986810BD0620FCE738B51368054614467C
:1011900053B140F21D43994205D15368062B02D149
:1011A0000023C380236038BD3D2903D1FFF78EFEA5
:1011B000EB68F7E7A22903D040F2B5439942F2D198
:1011C0002846FFF7D3FF2060EDE700231A461946B3
:1011D000FFF71CBF73B5054610200E46EFF75BF80E
:1011E000044630B9104BD3F83822332A12DDDC6BB9
:1011F00024340E4B3046236037F0ECFF002201AB65
:10120000012162600194C4E902062846FFF7FEFE50
:1012100002B070BD034602460146284602B0BDE852
:101220007040FFF7F3BE00BF00400220CCBF0808AB
:101230002DE9F0430D469BB0064610201746EFF708
:101240002AF80446284637F0C5FF00F10109804618
:101250004846EFF720F80CB1002848D12549D1F8CD
:101260003822432A29DDC86BA2F13409012100F19B
:101270002404343003AB81F001010022CDF810903A
:1012800001931D4B8DF80C1002932B78FF2BCDE9A9
:10129000052004D1294607AD07A8EFF78FFF3A468E
:1012A000294601A8F0F700FB0021DDE90532D15401
:1012B000059BA360069BE3600CE044B923462246ED
:1012C000214630461BB0BDE8F043FFF79FBE70B922
:1012D000C4E90285094B002201213046236007AB97
:1012E00062600794FFF792FE1BB0BDE8F083002117
:1012F000C0E700BF0040022091100308CCBF0808DF
:101300000EB403B503AA52F8041B0192FFF790FF35
:1013100002B05DF804EB03B07047000083070BD107
:101320000268084B9A4207D1037A2BB100EB830382
:101330001A69054B9A4202D0044906F003BC012009
:10134000704700BFA8C108080D100308F8B20808CC
:1013500010B50446FFF7EAFE50B92046FDF7F0FD50
:10136000FFF7DCFF20B12069024BC01A18BF012033
:1013700010BD00BF0CC2080838B504460D46FFF783
:10138000E7FF18B12046FDF7DBFD0446294620465D
:10139000BDE8384006F0D6BB2DE9F0418846174637
:1013A0001E46FFF7DBFE04468068E0B90C20EEF72E
:1013B00072FFA060A8B9164BD3F83822172A0EDDA9
:1013C000D86B0623A060A3800023E380E38800EBB2
:1013D0008302D91CE18040F82380C2E90176BDE890
:1013E000F0810323EFE7E388A5880233AB42EDDB0E
:1013F000074BDB6B9842F2D003350122A900EEF7D0
:1014000065FF0028EBD0A388A0600333A380DDE74D
:101410000040022038B50D461446FFF79FFE836852
:101420001BB1C2882A60236038BD1A46FAE737B577
:101430000446A068FCF708FB019068B16568062DBA
:1014400005D001AB002201212846FCF7ADF8FDF7DD
:1014500097FF0028EDD0019803B030BD38B50446A1
:101460001D46084611464FF00412FDF749FA214681
:101470000C20FDF759FD2B68044600214360686885
:10148000FCF76EFAA060204638BD13B54FF0FF336D
:101490000C4663226721CDE9003294ED020B002354
:1014A0004FF48072F0F78CF902B010BD000000001C
:1014B00038B52DED048B90ED009B91ED008B05462A
:1014C0000C46B0EE490BB0EE481B36F03DFCB5EED5
:1014D000400B39EE407BF1EE10FA87EE086B1FD11E
:1014E00018EE903A9FED220B9FED237B002B20FE00
:1014F000070BB5EE406BF1EE10FA28D189EE087BB0
:101500009FED1D6B53EC172B9FED197B002B27FED6
:10151000067BBDEC048B85ED007B84ED000B38BDB4
:10152000B5EEC00BF1EE10FAB5EEC08B4CBF012248
:101530000022F1EE10FA4CBF012300239A42D8D0CA
:10154000B7EE007B30EE080B36EE476BD1E7B6EE18
:10155000005BBBFE467B36EE476BB4EEC56BF1EE2F
:1015600010FAD6DDB7EE006B37EE067BD1E700BF91
:1015700000000000000000000000000000000080EB
:1015800008B52DED028BB0EE408B1020EEF778FE03
:10159000034A80ED028BBDEC028B026008BD00BFE8
:1015A00034B308080000000030B50D4687B011467E
:1015B000022228461C46FDF7A3F935B99FED100B12
:1015C00007B0BDE83040FFF7DBBF012203A9206868
:1015D000FDF7BEFF40B10023DDE903011A46009389
:1015E000FBF78AF907B030BD2068830703D1026892
:1015F000054B9A42F6D0FDF7D3FDFFF7C1FFF1E7A7
:10160000000000000000000034B3080891ED020B58
:1016100007281DD8DFE800F00A181C1C041C0C1455
:10162000B5EE400BF1EE10FA14D01E2108467047BB
:10163000BDEEC00B10EE103A590041F00101F5E784
:1016400010EE903A002BF1DAB1EE400BFFF798BFA5
:101650000021EBE70E21E9E790ED020B7047000057
:1016600030B50C4605462DED028B87B0204602A909
:101670008DED000BFDF754FD002800F0C180232DF7
:1016800000F21E81DFE815F0E000EC00F800040134
:1016900010011C011C011C011C011C011C011C016E
:1016A0001C011C0124002D0034001C013B004F00D4
:1016B0005D008E001C011C011C011C011C0124008A
:1016C0002D0034001C013B004F005D008E00C50062
:1016D0009DED007B9DED026B37EE067B8DED007B73
:1016E0001CE09DED007B9DED026B37EE467BF5E740
:1016F0009DED007B9DED026B27EE067BEEE79DEDF9
:10170000027BB5EE407BF1EE10FA03D174497548C7
:10171000FBF75AFE02A96846FFF7CAFE9DED000BD3
:10172000FFF72EFF6CE09DED027BB5EE407BF1EE06
:1017300010FAEBD09DED005B85EE076B8DED006B35
:10174000ECE79DED028BB5EE408BF1EE10FADDD0AB
:10175000B0EE481B9DED000B36F0F6FAB5EE400BEF
:10176000F1EE10FA09D118EE903A9FED577B9FEDFC
:10177000586B002B27FE067BB0E7B5EEC00BF1EEF1
